:10000000000001204DFF000075FF000077FF000099
:1000100079FF00007BFF00007DFF00000000000072
:100020000000000000000000000000007FFF000052
:1000300081FF00000000000083FF000085FF00003A
:1000400087FF000087FF00000505010087FF000013
:1000500041A9000087FF000087FF000087FF000024
:1000600087FF000087FF000087FF000087FF000078
:1000700087FF000087FF000087FF000087FF000068
:1000800087FF0000C908010087FF000087FF00000C
:1000900087FF000087FF000087FF000087FF000048
:1000A00087FF000087FF000087FF000087FF000038
:1000B00087FF000087FF0000000000000000000034
:1000C00087FF000087FF000087FF000087FF000018
:1000D00087FF000087FF000087FF0000000000008E
:1000E0000000000000000000000000000000000010
:1000F0000000000000000000000000000000000000
:1001000000000000000000000000000000000000EF
:1001100000000000000000000000000000000000DF
:1001200000000000000000000000000000000000CF
:1001300000000000000000000000000000000000BF
:1001400000000000000000000000000000000000AF
:10015000000000000000000000000000000000009F
:10016000000000000000000000000000000000008F
:10017000000000000000000000000000000000007F
:10018000000000000000000000000000000000006F
:10019000000000000000000000000000000000005F
:1001A000000000000000000000000000000000004F
:1001B000000000000000000000000000000000003F
:1001C000000000000000000000000000000000002F
:1001D000000000000000000000000000000000001F
:1001E000000000000000000000000000000000000F
:1001F00000000000000000000000000000000000FF
:1002000010B5054C237833B9044B13B10448AFF350
:1002100000800123237010BDA00200200000000018
:10022000309B010008B5034B1BB103490348AFF3F2
:10023000008008BD00000000A4020020309B0100E7
:10024000154B002B08BF134B9D46A3F5803A0021A8
:100250008B460F461348144A121A12F066FE0F4BD3
:10026000002B00D098470E4B002B00D09847002061
:10027000002104000D000D48002802D00C48AFF307
:10028000008012F09BFD2000290010F05DFB12F0B1
:10029000E3FB00BF00000800000001200000000098
:1002A00000000000A00200207C09002000000000E7
:1002B00000000000002070470020704700207047B9
:1002C000F0B5044685B00E46684611461F4609F053
:1002D00031FF23686A469D6A31463B462046A8475F
:1002E00005B0F0BDF0B5044685B00E46684611462F
:1002F0001F4609F02EFE23686A469D6A31463B463A
:100300002046A84705B0F0BD70B590B00C46154624
:100310001E4605F0F9FC48B364B321464022684606
:1003200013F0D7FD2F21684613F06AFD28B9234644
:1003300003224021684609F07FFE3F22314668468D
:1003400013F0A1FD0C480EF0C9FC78B10B4B93F9EA
:100350000030062B0CD10A4B93F9003043B901232E
:100360002A46694604480EF016FF012010B070BD01
:100370000020FBE72046F9E7E0030020D803002037
:10038000B003002007B5002300931A46194603481E
:100390000FF014FC03B05DF804FB00BFBC020020AA
:1003A00007B5002300931A46194603480FF006FCD0
:1003B00003B05DF804FB00BFC402002082B002ABB2
:1003C000012003E9060002B07047002070470020BA
:1003D0007047406818B1006808B1007C0009704798
:1003E00043682BB11B681BB11A7C61F307121A74A6
:1003F0007047406808B508B101F0B4FF012008BD9E
:1004000013B5002204461146684604F041F96068BD
:1004100001F0A8FF052807D8DFE800F01103110656
:100420000611012002B010BD61684FF400726846E9
:1004300004F020FD0021684604F0ECFBF2E7002008
:10044000F0E713B5002204461146684604F020F98F
:100450002046FF22694604F058FC204602B010BD39
:1004600007B5002300931A46194603480FF0A6FB70
:1004700003B05DF804FB00BFCC0200207047436866
:100480003BB1B0F90A00012806D002DB033802288C
:1004900001D9002070470220704700002DE9FF417C
:1004A00002AC84E8060006463B493C489DF828809B
:1004B0009DF82C501F460FF0C9FB204604F064FE47
:1004C000204604F063FA50BB204604F0C5FC052822
:1004D00004D8DFE800F01524170303170546304958
:1004E0002E480FF0B3FB0A2229462C480FF017FCC8
:1004F0002A480FF0BBFB204604F046FE00200BE02C
:100500004FF00108CDE90085336894E806005D6C82
:1005100030463B46A847012004B0BDE8F0812046A4
:1005200004F0E4FB012812D0022831D01D491B48F9
:100530000FF08CFB204604F0D9FB0A220146174835
:100540000FF006FC15480FF091FB0125C7E70021CD
:10055000204604F0B1FA13280ED81E21204604F0DC
:100560001BFB71684FF40072204605F061F94FF4EF
:100570009051706802F08CFD01953368012500955B
:10058000D3F8448094E806003B463046C047C2E7B3
:1005900000230393F0E700BF6479010068030020A3
:1005A0007A7901006D79010008B511B9B0F9080038
:1005B00008BDB0F90A208A4203DC0089084400B271
:1005C000F6E7406801F078FFF9E7000007B500237F
:1005D00000931A46194603480FF0F0FA03B05DF88D
:1005E00004FB00BFD40200200A460068022100F08C
:1005F00099BD000070B503680546F3B17221FFF79D
:10060000F3FF28680E4E03680021DB699847002439
:100610002868042C03680CD0DB689847A35D9842D7
:1006200005D0286803685B6A9847002070BD0134D4
:10063000EEE75B6A98470120F8E71846F6E700BF47
:10064000DC7901002DE9F041036804461BB900265E
:100650003046BDE8F081FFF7CDFF07460028F6D011
:10066000254672212046FFF7BFFF55F8100B03689F
:100670000421DB69984704F1160800262068036806
:10068000DB689847C0B205F8010B0138C0B2FD28FD
:1006900098BF3E46A845F1D1206803685B6A984739
:1006A000D6E7F8B5036804460F4613B90025284677
:1006B000F8BDFFF79FFF05460028F7D072212046BE
:1006C000FFF792FF206803682646DB6904219847FC
:1006D00056F8100B036806225B68394698473B685A
:1006E0002361BB88B380206803685B6A9847DEE7B4
:1006F00070B5036804460D46164613B90025284612
:1007000070BDFFF777FF0028F8D072212046FFF771
:100710006BFF206803684021DB699847731E2A46F7
:10072000002120680FF076FD06B2206803685B6A3E
:100730009847002EE2D00023AB55E0E738B50368B8
:1007400004460D460BB9002038BDFFF753FF0028C3
:10075000F9D0284613F08FFB0F28F4D872212046D9
:10076000FFF742FF206803684021DB69984729466C
:1007700020680FF074FA2068036800211B6898470E
:100780000546206803685B6A9847281C18BF01204B
:10079000DAE738B5036804460D460BB9002038BDCA
:1007A000FFF728FF0028F9D0284613F064FB0F2834
:1007B000F4D872212046FFF717FF20680368502104
:1007C000DB699847294620680FF049FA20680368DA
:1007D00000211B6898470546206803685B6A9847B4
:1007E000281C18BF0120DAE770B5036804460D46DF
:1007F000164613B90025284670BDFFF7FBFE0028FA
:10080000F8D072212046FFF7EFFE20680368202110
:10081000DB699847731E2A46002120680FF0FAFC16
:1008200006B2206803685B6A9847002EE2D0002376
:10083000AB55E0E738B5036804460D460BB9002018
:1008400038BDFFF7D7FE0028F9D0284613F013FB78
:100850001F28F4D872212046FFF7C6FE20680368DF
:100860002021DB699847294620680FF0F8F92068B5
:10087000036800211B6898470546206803685B6A87
:100880009847281C18BF0120DAE773B503680546AE
:100890000E461BB90024204602B070BDFFF7AAFE29
:1008A00004460028F6D072212846FFF79DFE2868EE
:1008B00003681021DB69984704220DEB02012868C8
:1008C0000FF093FC019930460FF095F92868036802
:1008D0005B6A98473379002BDCD0FF2BDBD173792F
:1008E000FF2BD8D1B379FF2BD5D1F479FF3C18BFBA
:1008F0000124D0E773B5036805460E461BB90024F2
:10090000204602B070BDFFF775FE04460028F6D001
:1009100072212846FFF768FE286803681C21DB69FE
:10092000984704220DEB020128680FF05EFC019944
:1009300030460FF060F9286803685B6A984733799E
:10094000002BDCD0FF2BDBD17379FF2BD8D1B3790F
:10095000FF2BD5D1F479FF3C18BF0124D0E773B544
:10096000036805460E461BB90024204602B070BD40
:10097000FFF740FE04460028F6D072212846FFF714
:1009800033FE286803681421DB69984704220DEBC5
:10099000020128680FF029FC019930460FF02BF96D
:1009A000286803685B6A98473379002BDCD0FF2BFB
:1009B000DBD17379FF2BD8D1B379FF2BD5D1F47963
:1009C000FF3C18BF0124D0E773B5036805460E4607
:1009D0001BB90024204602B070BDFFF70BFE044691
:1009E0000028F6D072212846FFF7FEFD286803682C
:1009F0001821DB69984704220DEB020128680FF0EB
:100A0000F4FB019930460FF0F6F8286803685B6A3A
:100A100098473379002BDCD0FF2BDBD17379FF2B88
:100A2000D8D1B379FF2BD5D1F479FF3C18BF01247D
:100A3000D0E737B54B6801930368044613B900202B
:100A400003B030BDFFF7D6FD0028F8D07221204654
:100A5000FFF7CAFD206803681021DB69984720680A
:100A6000036804225B680DEB020198470546206885
:100A700003685B6A9847281C18BF0120E0E737B578
:100A80004B6801930368044613B9002003B030BDDE
:100A9000FFF7B0FD0028F8D072212046FFF7A4FD33
:100AA000206803681C21DB699847206803680422DA
:100AB0005B680DEB020198470546206803685B6A96
:100AC0009847281C18BF0120E0E737B54B68019311
:100AD0000368044613B9002003B030BDFFF78AFD58
:100AE0000028F8D072212046FFF77EFD20680368B9
:100AF0001421DB6998472068036804225B680DEBCA
:100B0000020198470546206803685B6A9847281CDD
:100B100018BF0120E0E737B54B680193036804462E
:100B200013B9002003B030BDFFF764FD0028F8D0F2
:100B300072212046FFF758FD206803681821DB6901
:100B400098472068036804225B680DEB0201984710
:100B50000546206803685B6A9847281C18BF012077
:100B6000E0E713B57723009303680446A3B1FFF7CA
:100B700041FD88B172212046FFF736FD20680368E9
:100B80000C21DB6998470422694620680FF02DFB91
:100B9000206803685B6A9847009B0020DAB262F322
:100BA0000700C3F3072262F30F20C3F3074262F387
:100BB00017401B0E63F31F6002B010BD37B50191E3
:100BC0000368044613B9002003B030BDFFF712FDDF
:100BD0000028F8D072212046FFF706FD2068036840
:100BE0000C21DB6998472068036804225B680DEBE1
:100BF000020198470546206803685B6A9847281CED
:100C000018BF0120E0E707B5FFF7ABFFC043C0F313
:100C1000C01003B05DF804FB37B505460C46FFF77E
:100C2000A0FF84F00104019064F3C7108DF8040064
:100C30000199284603B0BDE83040FFF7BFBF07B5B4
:100C4000FFF78FFFC0F3002003B05DF804FB37B55A
:100C50000D460446FFF785FF0190C0F3072065F3BA
:100C600000008DF805000199204603B0BDE8304032
:100C7000FFF7A4BF07B5FFF774FF80F00800C0F3CB
:100C8000C00003B05DF804FB37B505460C46FFF71E
:100C900068FF84F00104019064F3C3008DF8040040
:100CA0000199284603B0BDE83040FFF787BF37B54C
:100CB0000D460446FFF755FF019065F302008DF8DD
:100CC00004000199204603B0BDE83040FFF776BF2D
:100CD00037B50D460446FFF744FF019065F3061053
:100CE0008DF804000199204603B0BDE83040FFF7BD
:100CF00065BF07B5FFF735FF00F0070003B05DF8EB
:100D000004FB07B5FFF72DFFC0F3021003B05DF839
:100D100004FB000070B51E4D0C468AB00646043434
:100D20001C4928460EF092FF214607A80FF0AFFCA1
:100D300007A928460EF08EFF2846174D0EF096FFA5
:100D400007A80FF014FC294601A80FF055FC01A9D3
:100D500004A80FF09CFC214604A80FF0D8FC2946FB
:100D6000044607A80FF048FC07A920460FF0CFFC67
:100D7000014630460FF08BFC07A80FF0F8FB04A8E3
:100D80000FF0F5FB01A80FF0F2FB30460AB070BD82
:100D900068030020E1790100EC7901007FB50D4680
:100DA0000446222128460FF007FD22210646284648
:100DB0000FF01CFD002E034604F1040422DB002882
:100DC00020DD721C294601A80FF014FD01A9204660
:100DD0000FF067FC01A80FF0CAFB0D490D480EF09B
:100DE00035FF214601A80FF052FC01A909480EF079
:100DF00031FF08480EF03AFF01A80FF0B8FB0120C0
:100E000004B070BD294620460FF032FCE5E700BF74
:100E1000EE790100680300207FB503680446002BCB
:100E200039D07721FFF7E0FB206803680021DB69F8
:100E300098470025206802690368954204D21B6820
:100E4000002198470135F5E7DB69144E00219847EA
:100E500000252068715D036801351B689847042DE3
:100E6000F7D1206803685B6A98470D4901A80FF025
:100E7000C3FB01A92046FFF791FF01A80FF077FB04
:100E800007212046FFF713FF07212046FFF720FF29
:100E9000012004B070BD1846FBE700BFDC790100FB
:100EA000E69501007FB50368044613B9002004B03D
:100EB00070BDFFF79FFB0028F8D0E3681F2BF5D823
:100EC000264672212046FFF78FFB56F8040B036875
:100ED0006021DB699847314620680EF0BBFE206830
:100EE000036800211B6898470546206803685B6A11
:100EF00098478DB10A490B480EF0A8FE314601A86B
:100F00000FF0C5FB01A907480EF0A4FE05480EF03E
:100F1000ADFE01A80FF02BFB281C18BF0120C6E76F
:100F2000067A01006803002030B5036885B00446E6
:100F300013B9002005B030BDFFF75CFB0028F8D0E6
:100F4000254672212046FFF74FFB55F8040B036836
:100F50006021DB6998470022216801A80FF074F92D
:100F600001A928460FF09DFB01A80FF000FB2068A7
:100F700003685B6A98470B490B480EF067FE2946E9
:100F800001A80FF084FB01A907480EF063FE064894
:100F90000EF06CFE01A80FF0EAFAE068003018BF0E
:100FA0000120C7E7F97901006803002007B5002395
:100FB00000931A46194603480EF000FE03B05DF890
:100FC00004FB00BFDC02002007B5002300931A4693
:100FD000194603480EF0F2FD03B05DF804FB00BFB4
:100FE000E402002001207047C08A7047027D1AB1D8
:100FF0000368FF211B68184770470369994228BF9F
:101000001946816108467047037D10B5044633B91F
:10101000A069236998422CBF0020012010BD0368FD
:101020001B699847FF28F3D10020F7E7036810B544
:1010300004461B699847A3690133A36110BD70473B
:1010400008B502698369934205D2C169034819440E
:101050000EF003FC08BD4FF0FF30FBE7EC02002070
:1010600010B5D0E906345A1C82610A460248E118DC
:101070000EF0F5FB012010BDEC02002008B590F841
:101080002020772A0BD10368DB6A9847044905487A
:101090000EF0DCFD0348BDE808400EF0E7BD08BDDA
:1010A0002B7A010068030020F0B50D4685B0044698
:1010B0003F21284617460FF07FFB031E0BDB002263
:1010C000294601A80FF096FB01A928460FF0E9FA7E
:1010D00001A80FF04CFA114928460FF024FB0646F0
:1010E00060B10023A3614FF4FA43236101208423FC
:1010F000E361207584F8207005B0F0BD08492846EA
:101100000FF011FB0028F7D08423C4E906662361A1
:10111000267584F820700120EEE700BF127A0100E6
:101120001F7A010001294FF0000303D002290CD0DF
:101130001846704783614FF4FA4303618423C36107
:10114000017580F82020012070478421C0E9063312
:1011500001610375F5E7000007B5002300931A4607
:10116000194604480EF02AFD034803B05DF804EB6D
:101170000EF070BBED020020EC02002038B5002319
:1011800083608380036804460D46002B47D0274ABE
:101190001268002A43D0002908BF1D462B7C03F0AB
:1011A0000F03062B10D1224A224829460DF045FA9A
:1011B00008B143692371204A1E4829460DF03DFAC3
:1011C00000282DD0436963711C4A216819480DF02D
:1011D00034FA054608BB1A491A480EF037FD0A22B0
:1011E000617918480EF0B4FD174916480EF02EFD2F
:1011F0000A22217913480EF0ABFD12480EF036FD9D
:101200002B460E4A21680B480DF05FFA0B4A216805
:1012100008480DF012FA054608B11435A56038BD2E
:10122000286811F0FCFB6071CEE700BF300400209D
:10123000249501006C070020707A0100D67A010025
:10124000D97A0100680300209B86010010B504468E
:1012500001601146FFF792FF204610BD41790C4A0C
:10126000002352F82300884203D10A4A52F823008F
:10127000704752F8230028B942F82310054A42F873
:10128000230070470133052BEBD10020704700BFCE
:10129000040300201803002010B50A4A40790023F7
:1012A00052F82340844203D1074A42F8231010BD6C
:1012B00052F8234014B952F82320F5E70133052BE7
:1012C000EED1F4E70403002018030020F0B52DED63
:1012D000028B9BB00446FFF7C1FF05460FF0B2FA40
:1012E0000023014643F69822284608F039FF0028DB
:1012F00000F0E78006231622617905A80EF0A4F815
:10130000372105A80EF0B0F80022114605A80EF00E
:10131000C7F9002108EE900A05A80EF059FA6B49AA
:1013200008EE100A6A480EF091FC0A2261796848BA
:101330000EF00EFD674966480EF088FC18EE900A24
:1013400010F0ACFF022502460B46009560480EF0F7
:10135000BBFD61495E480EF079FC18EE100A10F0F2
:101360009DFF00950B46024659480EF0ADFD5B49C6
:1013700057480EF06BFC56480EF078FC584A21682E
:1013800058480DF05AF9584A2168074655480DF05B
:1013900054F9F4EE688AF1EE10FA06460FD60AAD5B
:1013A00018EE901A284603F080F90023CDE90033A7
:1013B0004FF0FF3195E80C00384608F0EBFEB4EE34
:1013C000488AF1EE10FA0FD60AAD18EE101A284628
:1013D00003F06BF90023CDE900334FF0FF3195E8BE
:1013E0000C00304608F0D6FE404A21683D480DF01A
:1013F00024F9054600285ED0037C03F00F03042B7C
:1014000059D1F5EE408AF1EE10FA54D0B5EE408A8B
:10141000F1EE10FA4FD0F4EE688AF1EE10FA4AD1EC
:10142000B4EE488AF1EE10FA45D100213C220BA817
:101430000A9111F07AFD696940220AA812F049FD6B
:101440002F210AA812F0DCFC28B96B690322402185
:101450000AA808F0F1FD26490AA812F0C2FC02A869
:1014600018EE901A08F075FD22480DF037FC40B1D7
:10147000214B93F9003023B902AA0AA91D480DF0A7
:1014800075FE0AA812F0F7FC1AAB1844482300F8BE
:10149000413C18EE101A02A808F05BFD15480DF04B
:1014A0001DFC40B1144B93F9003023B902AA0AA9DC
:1014B00010480DF05BFE0FF0C5F901462046FFF71E
:1014C000EBFE1BB0BDEC028BF0BD00BFD27A010079
:1014D00068030020DE7A0100EE7A0100F57A01004F
:1014E000F77A01006C070020FC7A0100007B010004
:1014F00024950100E0030020B00300202DE9F04F07
:101500000546006887B00F46904640B1A86830B1E4
:101510000378FF2903F0100335D11BB9012007B070
:10152000BDE8F08F032AF9D047789C499C480EF01B
:101530008DFB0A2269799A480EF00AFC994998486D
:101540000EF084FBAB68964859780A2201F00F012F
:101550000EF0FEFB3F09944991480EF077FB0A22FA
:1015600039468F480EF0F4FB8D480EF07FFBAB68D8
:101570005A7802F00F02BA4207D11A786FF30412B8
:101580001A700020CBE7002BFBD100220DF10809D7
:101590001146484603F07CF8AB685B7803F00F0314
:1015A000BB4223D0B8F1030F20D080497C480EF015
:1015B0004DFB0A2269797A480EF0CAFB79497848CE
:1015C0000EF044FBAB68764859780A2201F00F010F
:1015D0000EF0BEFB744972480EF038FB0A22394601
:1015E0006F480EF0B5FB6E480EF040FB29680C2FDB
:1015F00000F2AF80DFE807F0073A94A1A394739458
:10160000A5A784A9AB00AB685B7803F00F03023B8E
:10161000082B24D8DFE803F00523239D230F232381
:101620001900634A63480DF008F8AB681C78064659
:1016300004F001042DE0604A5E480CF0FEFFAB6848
:101640001C780646C4F3400423E05C4A59480CF079
:10165000F4FFAB681C780646C4F3800419E0584ACE
:1016600054480CF0EAFF0646002412E0554A51485F
:101670000CF0E3FFAA681378D94303F0010461F387
:1016800000031370064620B90122494604A803F05E
:10169000DCFB4D4A296847480CF0CFFF4B4A2968CC
:1016A000824644480CF0C9FF834638B9BAF1000FAE
:1016B00004D15246494604A803F0C7FB002E4BD183
:1016C000484603F063F9002846D1AB685A7867F3BF
:1016D00003025A701A7866F304121A701EE73C4A25
:1016E00034480CF0AAFFA9680B7883F00202C2F319
:1016F0004002C3F34004064662F341030B70C8E79F
:10170000344A2C480CF099FFA9680B7883F0040246
:10171000C2F38002C3F38004064662F38203EDE75E
:10172000274A24480CF089FF064600289CD1022253
:10173000494604A803F089FB96E7274A72E7274A3F
:1017400070E7274A78E7274A76E7274A7EE7274A5D
:101750007CE7002426469CE7AB68B8F1030F5A7873
:101760000FD067F303025A701A786FF304121A70DD
:10177000CDE900AB214699E80C00304608F00AFD9F
:10178000CCE602F00F01B9423FF4C8AE67F307128E
:101790005A701A7842F010029FE700BF687A010081
:1017A00068030020147B0100727A0100707A010046
:1017B000767A01006C070020757A01007C7A0100BE
:1017C000837A0100887A0100BE7A0100007B010063
:1017D0008D7A0100937A0100997A01009E7A0100C6
:1017E000A47A0100AA7A0100B17A0100B77A010057
:1017F0002DE9F0435D4A95B00746884601685C488C
:101800000CF01BFF5B4A3968814659480CF015FF04
:101810000646B9F1000F01D100287AD0564A39683E
:1018200053480CF00AFF554A3968054650480CF0F9
:1018300004FF5349044653480EF008FA0A22797906
:1018400050480EF085FA50494E480EF0FFF90A2232
:1018500041464C480EF063FA4A480EF007FA5EB370
:10186000337C03F00F03042B26D14022716904A8B6
:1018700012F02FFB45480DF031FAE8B1444B93F9D3
:101880000030CBB92F2104A812F0BAFA28B9736935
:101890000322402104A808F0CFFBB8F1000F41D08B
:1018A00025B12B7C03F00F03042B35D0394A0123DB
:1018B00004A936480DF06FFCB9F1000F29D099F852
:1018C000103003F00F03042B23D1D9F8141004A80F
:1018D00000F0E0FF04A800F01BFFB8B1B8F1000F62
:1018E00034D025B12B7C03F00F03042B25D002ACA0
:1018F00001220021204602F0CBFE01220023CDE987
:10190000002304A894E8060001F024FC04A800F0D9
:101910001FFD15B0BDE8F0836A691378002BCBD0AA
:101920000123C5E724B1237C03F00F03042B02D06D
:101930000123194ABCE76269EFE769690B78002B5C
:10194000E4D0002204A802F0A7FADFE724B1237C48
:1019500003F00F03042B02D002AC0222C9E7616935
:101960000B78002BD2D04246ECE700BFBE7A0100D4
:101970006C070020007B0100887A0100837A010057
:10198000CB7A010068030020F37A0100E003002015
:10199000B0030020268F0100318F010070B598B090
:1019A000054602AC84E8060039483A490EF04EF983
:1019B0000A22697936480EF0CBF9374934480EF0DF
:1019C00045F9204603F0E0FB2968344A34480CF01E
:1019D00034FE0023CDE900334FF0FF3194E80C00D2
:1019E00008F0D8FB29682F4A2D480CF026FE2968FC
:1019F0002D4A06462A480CF020FE054660B3037CBB
:101A000003F00F03042B27D14169402208A812F0EC
:101A100060FA2F2108A812F0F3F928B96B690322A4
:101A2000402108A808F008FB0023102200930DEBCA
:101A300002014FF40073204603F092FA1B480DF0A8
:101A40004DF948B11A4B93F900302BB9012304AA80
:101A500008A916480DF09FFBC6B1337C03F00F03B5
:101A6000042B13D1716908A800F014FF08A800F036
:101A70004FFE40B101220023CDE9002308A894E8DD
:101A8000060001F067FB08A800F062FC18B070BD0A
:101A900068030020D27A0100F37A0100C77A0100BE
:101AA0006C070020BE7A0100007B0100E0030020EB
:101AB000B003002010B503788B42044604D143786C
:101AC000402B01D1408810BD40232170637008462F
:101AD0000EF0B0FF80B26080F5E7000083682DE96A
:101AE000F04104460D46002B00F05A81AD4F3B7883
:101AF0000133DBB20A46FF213B70FFF7FFFC63793D
:101B000026790E3B072BC6F3400830D8A64A216839
:101B1000A6480CF092FD064648B3037C03F00F0381
:101B2000052B24D16179A248FFF7C4FF002280462B
:101B300031469E480CF077FD436998451FDA002630
:101B4000032D60D0A3685A7802F00F02013A0B2AE5
:101B500059D8DFE812F01F00ED0042006A00ED00E6
:101B60007200ED009100A200AA00D300E5006079A8
:101B70000FF090F8A8EB00035E425E41E0E73146CB
:101B800001228A480CF04FFD4669B045CCBF0026C3
:101B90000126D5E7B3F802800EF054FE4FF6FF732E
:101BA00081B24FF47A72404608F0DAFA58B3814AAB
:101BB00021687E480CF041FD28B12A4603212046C9
:101BC000FFF79CFC1FE07C4A216878480CF035FD4B
:101BD0000028F2D12A460D21F1E7B3F802800EF079
:101BE00031FE4FF6FF734FF4967281B2404608F013
:101BF000B7FA40B12A4604212046FFF77FFC0EF0D9
:101C000021FEA3685880A2681378C3F3C001B142D3
:101C100000F0468113F0E00F00F09C80C3F3421106
:101C2000013961F347131370B6E0B3F802800EF088
:101C300009FE4FF6FF739622D7E7B3F802800EF045
:101C400001FE4FF6FF7381B24FF47A72404608F0FE
:101C500087FA0028D7D0594A216854480CF0EDFC87
:101C600010B12A460821AAE7554A21684F480CF0CE
:101C7000E4FC0028F5D1ADE7B3F802800EF0E2FDF8
:101C80004FF6FF734FF4967281B2404608F068FA3F
:101C90000028B8D02A460921AEE7B3F802800EF03A
:101CA000D1FD4FF6FF739622EEE7B3F802800EF0F7
:101CB000C9FD4FF6FF7381B24FF47A72404608F0C7
:101CC0004FFA00289FD03F4A216838480CF0B5FCF5
:101CD00010B12A460B2172E73B4A216833480CF0C9
:101CE000ACFC0028F5D1394A216830480CF0A5FC3D
:101CF00000287FF46FAF2A46062160E7B3F8028020
:101D00000EF0A0FD4FF6FF734FF4967281B240467D
:101D100008F026FA00283FF476AF2A460C216BE73C
:101D2000B3F802800EF08EFD4FF6FF739622EDE7BA
:101D3000B3F802800EF086FD4FF6FF7381B24FF4C8
:101D40001672404608F00CFA00283FF45CAF2A46B1
:101D5000002134E70EF076FDA36858805B7803F02D
:101D60000F03002E51D0072B11D8DFE803F04810E5
:101D700004101004104B164A21680C480CF05DFC4E
:101D800040B32A4606212046FFF7B8FB20B1A368DE
:101D90001A7866F3C3021A703B78013BDBB23B70E2
:101DA000BDE8F08100030020C37A01006C07002029
:101DB0002C030020997A01009E7A0100A47A010088
:101DC000AA7A0100B17A0100B77A0100937A010082
:101DD0008D7A0100334A216833480CF02EFC00282C
:101DE000CFD1324A216830480CF027FC0028C8D1F6
:101DF0002F4A21682C480CF020FC0028C1D12A462B
:101E00000121C0E72A460A21BDE7013B0C2BBED8C1
:101E100001A252F823F000BF4D1E00008F1D0000EC
:101E2000531E0000531E00008F1D0000591E0000AD
:101E30008F1D00009B1E00009B1E00009B1E0000CB
:101E40009B1E00009B1E0000531E00002A4602211C
:101E500099E72A46052196E7164A216812480CF0B0
:101E6000ECFB10B12A4607218DE70E4A21680E4887
:101E70000CF0E3FB0028F5D10C4A21680A480CF06D
:101E8000DCFB0028EED12168094A07480CF0D5FB9D
:101E900001460028E6D12A4675E72A46002172E766
:101EA0000221BEE6A47A01006C070020AA7A010094
:101EB000757A01008D7A01002DE9F047032986B07B
:101EC000804669D00168624A62480CF0B6FB98F817
:101ED000051006466048FFF7EDFD05B2002E69D0FB
:101EE000337C03F00F03052B64D1314659480CF0C5
:101EF00090FB032853D90022314656480CF093FB3F
:101F000001224469534831460CF08DFB0222D0F87F
:101F100014A0504831460CF086FB43694D480A270F
:101F20000322314607FB03F90CF07DFB43695F4355
:101F3000214600974B46524628460EF00EFB0446BB
:101F4000314644480CF065FB052830D10422314667
:101F500040480CF068FBB0F914A03E48BC42C4BF36
:101F60003C4640F2FF3531464C45BCBF4C4600254F
:101F70000CF04FFB022826D10022314635480CF0E8
:101F800052FB4369AB4251DC0122314631480CF02F
:101F90004AFB4369AB4258DB06B0BDE8F08705EB6E
:101FA000850464004FF000094FF42057C8E74FF054
:101FB000010AD2E705EB850464004FF000094FF4F5
:101FC00020574FF0010AD8F80830B3F902002A1A56
:101FD000002AB8BF5242524507DC1A785109052938
:101FE00007D8013161F3471202E01A786FF3471204
:101FF0001A701B789F2B03D94C4501D0BC42CBD122
:10200000A842C9D00022114604AE02A802F040FB4B
:10201000224602A9304602F0A4FE96E80600404699
:10202000FFF7BCFCD8F808305D80B5E70024D8F88D
:102030000830B3F90230A342AED021464046FFF744
:10204000D7FBD8F808305C80A6E70124EFE700BF93
:10205000C37A01006C0700202C03002008B58368B8
:102060000246F3B1012916D00ADB032908DC037903
:10207000402B0CD006D8032B02D81046FFF72EFDBC
:10208000002010E0422B02D0FAD3803BF3E7104649
:10209000FFF712FFF4E70379042BF1D1FFF716F9EC
:1020A000EEE74FF0FF3008BD7FB5037C03F00F0370
:1020B000062B054623D10146124A13480CF0BDFAFF
:1020C00090B1037C03F00F03052B0DD1C4680026EB
:1020D000ACB1294601A80194FFF750F8039B1E609C
:1020E0000EF006FC6468F3E704AC002144F80C5DD4
:1020F0002046FFF743F802212046FFF7AFFF04B068
:1021000070BD00BFC77A01006C07002038B5836836
:102110000446BBB1124B1B68A3B10068FFF7C4FFB4
:10212000A36800251D602379032B0CD8012B94BFD5
:102130000221294660790EF073FDA3685A7865F391
:1021400003025A7038BD402B03D0422BFAD12946E6
:1021500000E002216079BDE838400EF061BD00BFAB
:1021600030040020002303807047000013B50024D2
:10217000234600942246214603480DF01FFD034BE1
:102180001C8002B010BD00BFF80200202C0300200C
:1021900010B5044670B3204911F03FFE58B31F49F3
:1021A000204611F03AFE40B31D49204611F035FE9D
:1021B00028B31C49204611F030FE10B31A492046BE
:1021C00011F02BFEF8B11949204611F026FEE0B1BE
:1021D0001749204611F021FEC8B11649204611F0DA
:1021E0001CFEB0B11449204611F017FE002814BFA0
:1021F0000020152010BD0120FCE70220FAE7052091
:10220000F8E70620F6E71320F4E71420F2E70E20A3
:10221000F0E70F20EEE700BF247B01003F7B0100C9
:10222000667B0100537B01006B7B01005C7B01003E
:10223000577B01001B7B01002F7B010010B504467A
:1022400000284AD00378002B48D0314911F0E5FD31
:10225000002845D02F49204611F0DFFD002841D04D
:102260002D49204611F0D9FD00283DD02B492046AC
:1022700011F0D3FD002839D02949204611F0CDFDB9
:10228000002835D02749204611F0C7FD90B32649D4
:10229000204611F0C2FD78B32449204611F0BDFD5F
:1022A00060B32349204611F0B8FD48B321492046C8
:1022B00011F0B3FD30B32049204611F0AEFD18B344
:1022C0001E49204611F0A9FD00B31D49204611F01A
:1022D000A4FD002814BF00200D2010BD1846FCE707
:1022E0000220FAE70920F8E70120F6E70820F4E7E2
:1022F0000520F2E70620F0E70720EEE70A20ECE7EA
:102300000B20EAE70C20E8E70320E6E70420E4E7F7
:102310004B7B0100617B0100277B0100707B01008A
:10232000377B0100437B0100337B01003B7B0100D5
:10233000477B0100757B01004F7B01002B7B010077
:102340007A7B0100406910B103685B6918477047E8
:1023500010B50446406910B103685B689847204691
:1023600010BD000008B50322016804480CF05BF9B9
:1023700008B1007D08BDFF20FCE700BF6C0700200E
:1023800010B503220C46016810480CF04CF9E0B17E
:10239000037C13F00D0F18D1022262F303030374C0
:1023A00043690B4923F07F4323F0FF032343436139
:1023B00008480DF04BFC21460A2206480DF0C8FCE7
:1023C0000448BDE810400DF051BC10BD6C07002062
:1023D000FD7D01006803002010B503220C46016852
:1023E00008480CF020F960B1037C03F00F03022BC6
:1023F00001BF24F07F41406921F0FF01084018BF70
:10240000002010BD6C07002010B503220C460168A7
:1024100009480CF008F970B1037C13F00D0F0AD1D4
:10242000022262F30303037424F07F41436921F025
:10243000FF011943416110BD6C07002010B504462F
:10244000406968B103689B69984718B1606903687F
:102450005B69984760690368DB68984708B90120A1
:1024600010BD2046FFF77EFF20B14FF4807120465B
:10247000FFF7CAFFA368002BF1D04FF4007120468C
:10248000FFF7C2FFEBE7000010B503220C4601681E
:1024900008480CF0C8F858B1037C13F00D0F07D1B1
:1024A000E143436941F07F4141F0FF01194041613F
:1024B00010BD00BF6C07002038B50C4641680546CA
:1024C00009B9002038BD0B7C03F00F03022B03D1A8
:1024D000002CF6D14869F5E7052BF2D105480CF040
:1024E00098F88442EDDAE2B2696802480CF09BF891
:1024F0004069E7E76C07002038B50D46416804469F
:1025000021B9DFED1A7A17EE900A38BD0B7C03F083
:102510000F03052B15D116480CF07BF8854210DA15
:10252000EAB2616812480CF07EF80028E9D0037C1A
:1025300003F00F03022B0FD1D0ED057AF8EEE77A06
:10254000E1E7002DDDD16268137C03F00F03022B5D
:1025500007D1D2ED057AF1E7032BD2D1D0ED057A80
:10256000D1E7032BCDD1D2ED057ACCE700000000F6
:102570006C07002008B5416869B10B7C03F00F03BC
:10258000022B06D0052B06D104480CF042F800B20D
:1025900008BD0120FCE70020FAE700BF6C0700201F
:1025A00008B5816809B9002008BD087C00F00F0358
:1025B0009A1E012A00D90BB90009F5E7052BF2D1C3
:1025C000002203480CF02FF80028ECD0007CF3E741
:1025D0006C070020826810B5BAB1137C03F00F03BA
:1025E0009C1E012C00D983B9516183681A7C022199
:1025F00061F303021A748268137C03F0F00160290E
:1026000002BF0A2161F30713137410BD826810B56D
:10261000BAB1137C03F00F039C1E012C00D983B9BF
:10262000516183681A7C032161F303021A74826882
:10263000137C03F0F001602902BF072161F3071347
:10264000137410BD836853B11A7C02F00F02901E00
:10265000012800D91AB91A7C61F307121A7470475D
:1026600008B5C16809B9002008BD0B7C03F00F0351
:10267000022B01D14869F7E7052BF4D1002203486A
:102680000BF0D1FF0028EED04069EDE76C07002089
:102690002DE9F041C36804460E46A3B90168194804
:1026A000184F0BF0B6FF0546042D0CDC3846D4F865
:1026B00000800BF0F4FF41460246E06038460BF024
:1026C000CBFF0135F0E7E268CAB1137C13F00F01CC
:1026D00013D1022161F303031374E3680A495E61B5
:1026E0000A480DF0B3FA31460A2208480DF0F5FA0F
:1026F0000648BDE8F0410DF0B9BA0229EDD0BDE8B9
:10270000F08100BF6C070020057E010068030020F7
:10271000006828B1007C00F00F00431F5842584168
:1027200070470000F8B50446FFF7F2FF002832D0EA
:1027300021683748364F0BF06CFF0546032D26689D
:1027400009DC38460BF0ABFF3146024638460BF049
:1027500083FF0135F2E7002231462D480BF063FF7D
:1027600002F0DDFB01222074216829480BF05BFF99
:1027700002226060216826480BF055FF0422A06009
:10278000216823480BF04FFFE060207C0C282CD000
:1027900002D803280ED0F8BD102830D01228FAD164
:1027A0000C200EF0E5F81B4B44600360054606F074
:1027B000FFFB18E010200EF0DBF8174B0360054616
:1027C000446000212046FFF777FE03B2002BB6BF1E
:1027D00040422B8128816868FFF7CCFE0F4B2B60AD
:1027E00000236881AB816561D5E714200EF0C0F845
:1027F0000B4B44600360054606F04AF8F3E70EF021
:10280000B7F8084B44600360054606F0FDFDEAE7B3
:102810006C070020B88F010094790100109001002E
:10282000D48E0100B890010010B500230446016069
:10283000436103768362FFF775FF204610BD0000F9
:1028400070B5056806462F21284611F063FB044643
:1028500098B1002300F8013BFFF7F0FC0B49054657
:102860000B480DF0F3F90A22294609480DF057FAF2
:1028700007480DF0FBF9284670BD2846FFF7DEFC3F
:1028800005460028F7D03460F5E700BF057B01005E
:10289000680300202DE9F04389B0002400F11808F6
:1028A0000546CDF804804461047684620E46002912
:1028B0003BD01F4B1F68002F37D02F21304611F01F
:1028C0009FFA814650B3234602AAF05C19B238B190
:1028D0002F2805D0142B02D0D0540133F5E7194628
:1028E00008AB1944002301F8183C124839460BF094
:1028F000A4FE0F22286009F10101404611F0E9FA17
:1029000001A8FFF79DFF019BA86203B92B7628461B
:10291000FFF708FF284609B0BDE8F0833246394684
:1029200004480BF08AFE2860F1E700232B60EEE7F5
:10293000D40300206C07002008B543693BB9007C34
:10294000052809D014280CBF0020FF2008BD1A68F4
:102950001846D26B9047F3E75020F7E708B50522F9
:10296000016805480BF05FFE20B1037C13F0F00016
:1029700018BF180908BD00BF6C0700202DE9F743F8
:102980006D4685E80600016881461F4619B900209A
:1029900003B0BDE8F0833448DFF8CC800BF039FE9B
:1029A0000446052CD9F8006009DC40460BF077FEA0
:1029B0003146024640460BF04FFE0134F1E7052256
:1029C000314629480BF02FFE04460028DFD0284668
:1029D00002F08CF90F28DAD8284602F023F80028F4
:1029E00007DD237C13F00D0F10D003F00F03072B2E
:1029F0000CD0237C1D491E486FF3071323740DF080
:102A000025F91B480DF032F90120C1E70DF01AFF3E
:102A10000646284602F006F8002F237C0CBF02224F
:102A2000072262F30303304460612374284602F0F6
:102A30005DF9237C0F4960F3071323740C480DF0F4
:102A400005F9284601F0EEFF0A22014608480DF07C
:102A500044F9094906480DF0F9F80A226169044869
:102A60000DF03BF9CDE700BF6C070020B37B010000
:102A700068030020BD7B0100C87B0100F0B587B072
:102A80006F4687E80600054697E8030002AC84E835
:102A9000050038461E4602F029F901380C2838D8BE
:102AA000DFE800F0424B959E8C0739373754627E41
:102AB00070004EBB0722214604A802F0C6F949491E
:102AC00049480DF0C3F8204602F010F90A220146E9
:102AD00045480DF03DF9454943480DF0B7F820460B
:102AE00001F0A0FF0A2201463F480DF0F6F83E48EB
:102AF0000DF0BCF89DF8303094E806002846FFF74A
:102B00003DFF012007B0F0BD2846FFF727FF002852
:102B1000D0D10020F6E70EB10622CCE72846FFF719
:102B20001DFF0028F8D1F4E70EB90222C3E72846BA
:102B3000FFF714FF0028F8D1EBE70EB10122BAE746
:102B40002846FFF70BFF0028F8D1E2E74FF4803169
:102B50002846FFF741FC08B10B22ACE72846FFF7F7
:102B6000FDFE0028F8D1D4E74FF480312846FFF766
:102B700033FC08B90A229EE72846FFF7EFFE00283B
:102B8000F8D1C6E74FF400312846FFF725FC08B915
:102B90000C2290E72846FFF7E1FE0028F8D1B8E7BD
:102BA0004FF400312846FFF717FC08B10D2282E7E9
:102BB0002846FFF7D3FE0028F8D1AAE70EB103227A
:102BC00079E72846FFF7CAFE0028F8D1A1E70EB939
:102BD000052270E72846FFF7C1FE0028F8D198E7E4
:102BE000042268E7E27B010068030020F67B010015
:102BF00018B1034903480DF029B80349FAE700BFAB
:102C0000117B010068030020167B01002DE9F043D1
:102C10009FB04FF0000802AC84E806000646102280
:102C200041460AA81D46269FCDF8248010F07DF964
:102C30002046CDE906888DF8208002F0A5FAEA0545
:102C40001AD5204602F052F8172800F2CD80012351
:102C500003FA00F0964B18420AD1964B0340002B22
:102C600040F0C68010F0240F00F0BE80924900E0D2
:102C7000924906A811F0DBF891480CF02FF80028D3
:102C800000F0AA808F4B93F900209846002A40F06C
:102C9000A380002F44D13B46032240210EA807F019
:102CA000CBF933683F2219680EA811F0ECF8AB0598
:102CB00040F1AD80204602F019F8022800F0A7800C
:102CC000204602F013F8052800F0A180204602F00B
:102CD0000FF8012840F08F804FF001094FF4007386
:102CE000142209A9CDF80090204602F039F94B468C
:102CF00009AA0EA972480CF04EFA734973480CF0F9
:102D0000A5FF0EA971480CF0AAFF71496F480CF09D
:102D10009DFF09A96D480CF0A2FF6C480CF0A6FFBE
:102D2000204601F044FE05F4005908B1A90503D47A
:102D3000B9F1000F00F09C800023032240210EA86F
:102D400007F07AF933683F2219680EA811F09BF852
:102D500047B160490EA811F044F83F2239460EA849
:102D600011F091F85B490EA811F03BF8B9F1000F92
:102D700067D059490EA811F034F8204601F0B8FF89
:102D8000043801285FD81722214604A802F05DF814
:102D9000002300934FF44073142209A9204602F047
:102DA000DFF8494949480CF051FF0EA947480CF09B
:102DB00056FF474945480CF049FF09A943480CF024
:102DC0004EFF42480CF052FF3D480BF087FF18B110
:102DD00098F90030002B40D030462946FFF714FB0D
:102DE00000201FB0BDE8F0833C4938480CF02EFFAE
:102DF00025F4807540E7204601F07AFF02283FF471
:102E00006BAF204601F074FF08283FF465AFE8057A
:102E100086D59DF81830002B82D0012306AA0EA972
:102E200027480CF0B8F9284928480CF00FFF0EA9E4
:102E300026480CF014FF264924480CF007FF06A989
:102E400068E7274996E70023B9F1000F00930CBF0C
:102E50004FF400734FF440739EE70EA9012309AAB3
:102E600017480CF098F94FF400713046FFF70CFB4F
:102E7000EA0540F18280204601F038FF013814282D
:102E800034D8DFE810F0D6003300330033003300CD
:102E9000D6003300330033003300330033003300F7
:102EA000DA00D4003300330033002F00D000D2000A
:102EB00042C03800010080003F7B0100247B0100FC
:102EC000E0030020B0030020DC7B01006803002049
:102ED000727A01009B8601002B7B0100CE7B0100F2
:102EE0004B7B01005B4906A810F0A1FF00230322E1
:102EF00040210EA807F0A0F833683F2219680EA8F9
:102F000010F0C1FF47B154490EA810F06AFF3F22EC
:102F100039460EA810F0B7FF4F490EA810F061FF18
:102F20004E490EA810F05DFF4D494E480CF08EFE44
:102F30000EA94C480CF093FE4B494A480CF086FE13
:102F400006A948480CF08BFE46480CF08FFE474817
:102F50000BF0C4FE00283FF43FAF98F90030002B7F
:102F60007FF43AAF0EA9012306AA40480CF013F9EA
:102F70004FF480713046FFF787FA6B0551D54FF457
:102F800080313046FFF728FA002858D0384906A883
:102F900010F04DFF0023032240210EA807F04CF84B
:102FA00033683F2219680EA810F06DFF47B12A4917
:102FB0000EA810F016FF3F2239460EA810F063FF4E
:102FC00025490EA810F00DFF2A490EA810F009FFA0
:102FD000234924480CF03AFE0EA922480CF03FFE8B
:102FE000214920480CF032FE06A91E480CF037FE9D
:102FF0001C480CF03BFE1D480BF070FE00283FF40F
:10300000EBAE98F90030002B7FF4E6AE0EA9012359
:1030100006AA16480CF0BFF84FF480613046FFF75F
:1030200033FA0120DDE614495DE714495BE71449F2
:1030300059E7337C052B7FF459AF124953E74FF41E
:1030400000313046FFF7C8F908B10F499FE70F4933
:103050009DE700BF6B7B01009B860100277B010081
:10306000DC7B010068030020727A0100E00300208D
:103070008C7B0100617B01005C7B01002F7B0100E8
:103080001B7B0100577B0100857B01007E7B0100DB
:10309000F0B5CB070C4644BF21F4805424F0010462
:1030A00014F4805785B005460CD004F4E06128463E
:1030B000FFF7AAF9144915480CF0C8FD4FF0FF308E
:1030C00005B0F0BD06F03EFF9528EED902F01CFEDB
:1030D0000028EAD002AE3A463946304601F0D8FA26
:1030E0004FF440722946304601F0C4FE4FF4E061CF
:1030F0002846FFF771F9009744EA000396E80600B6
:103100002846FFF783FDDBE7947B0100680300207E
:1031100010B54FF440710446FFF75EF9014670B1F7
:10312000074B93F90030062B09D12046FFF7B0FF7B
:1031300020464FF44071BDE81040FFF7A5B910BD1F
:10314000D803002043691BB11A681846D26B104798
:10315000007C70472DE9F04F91B00AAF09939DF8BC
:10316000683003939DF86C300493054687E80600A9
:1031700006F0E8FEB0F5966F04460EDAB549B6489B
:103180000CF064FD0A222146B3480CF0C8FDB24899
:103190000CF06CFD4FF0FF39A5E30DF053FB0790E9
:1031A000384601F059FE0290064602F0ADFD099B3B
:1031B00006901BB11A78002A40F002862B7E13B1CC
:1031C00005F118030993002E40F01286099B002B8D
:1031D00040F0F885AB6A0293002B00F00986384670
:1031E00001F03AFE002840F003869DF80820394699
:1031F0000EA801F035FE00F0FBBD2B68002BC9D0F6
:10320000029B042B07D1049B97E806002846FFF792
:10321000B5FB814667E3384601F068FD092800F2F6
:103220002382DFE810F00A002102210221026E0150
:10323000210221022102B001B00100220DF130096A
:103240001146484601F024FA384601F0B0FB064624
:10325000002800F05081029B0C2B1AD8DFE813F0F5
:103260000D00190069001900190019001900190052
:1032700019001900180104013401DDF82480B8F1A7
:10328000000F0AD0754976480CF0E0FC74480CF049
:10329000EDFC0024A2462646F7E0284600F0F2FFA7
:1032A0000028D4BF002101210A2204466C480CF0FA
:1032B00036FD6C496A480CF0D2FC384601F0B2FB8E
:1032C0000A22014666480CF008FD65480CF0CEFC69
:1032D000002C384640F36B8501F0A4FB70BB022242
:1032E00039460EA801F0B1FD40F201144FF001087B
:1032F00006E0012239460EA801F0A7FD40F20114B4
:103300004FF400722946484602F0EEFA484601F0B2
:10331000EFFC042814D1384601F0EAFC022814D14D
:10332000384601F0E5FC0CA902460EA801F0E3FCCA
:103330000BE0002426464FF0FF38E1E74446D5E78E
:10334000484601F0D5FC0528E5D02B7C072B08D199
:10335000384601F033FB20B102220CA90EA801F07F
:10336000CAFC2846FFF7EEFE00B200900DF1300ACD
:103370000DF128090EA899E80C00514601F07EFFD6
:10338000504601F001FF3EB1484601F0B1FC022871
:103390004FD1504602F0D4FA9AE8030089E80300BE
:1033A00044F490544FF0000A4FF0FF392B7C072B68
:1033B00040F05182039B73B36B681B7C03F00F03D7
:1033C000052B40F05A81069B002B00F053812846C4
:1033D00000F058FF0DF128090028049B099A68683D
:1033E0004946D4BF4FF0000B4FF0010B00F0CEFE6A
:1033F000029B012B4FFA8BF840F03F81484601F0C9
:10340000D6FA039038B1049B009399E806005B4616
:103410002846FFF733FB0AA801F068FC03380428AC
:1034200000F25181DFE810F02B014F01EE01730132
:103430005201484601F05CFC0128AAD0484601F040
:1034400057FC0A28A5D0484601F052FC0B28A3D10E
:103450009FE700BF017C010084030020417C010044
:1034600068030020147B010029464FF4007248468F
:1034700002F03AFA384601F0F3F9C1B2484601F0D9
:1034800097F998B9B246002634464FF0FF388BE7DB
:1034900029464FF40072484602F026FA384601F0F9
:1034A000D8F90146484601F069F9EAE799E80300CE
:1034B000022287E80300002639460EA801F0D0FC5E
:1034C0004FF49054B246E0E74FF400722946484664
:1034D00002F00AFA384601F0A2F90146484601F026
:1034E00078F999E803004FF0000A87E803004FF4E9
:1034F00090545646C9E7824604464FF0FF39C84605
:1035000054E7029B092B20D0284600F0BBFE002880
:103510000DDD022239460EA8012601F096FC40F28C
:1035200001144FF0FF394FF0000AB0463EE7012288
:1035300039460EA84FF0000A01F087FC40F2011452
:103540004FF0FF390126D04630E74FF4803128464E
:10355000FEF742FF06464FF4803128465EB1FEF783
:1035600093FF40F201444FF001094FF0000A564624
:103570004FF0FF381AE7FEF747FF40F201444FF0E3
:103580000109B246F3E797E803000DF1300888E837
:103590000300384601F00BFAE0B90524384601F083
:1035A000A5FB4FF4007209282946384608BF64423B
:1035B00002F09AF9002239460EA801F046FC029B5F
:1035C0000B2B49D8DFE803F021480D48484848480C
:1035D00048482343384601F0FDF904460028DCD072
:1035E000DCE700262846FFF7A7F9214602463846C1
:1035F00001F038F9044690BB98E8030087E803001F
:103600004FF0010A4FF0FF39B2E70126EAE7214601
:10361000384601F083F950B1022239460EA84FF026
:10362000000A01F01DFC4FF490545646EAE798E872
:10363000030087E80300AE49AE480CF007FBAD4835
:103640000CF014FB00244FF0010A2646DAE721466D
:10365000384601F088F9DEE70024A246F5E74FF48A
:1036600090544FF0000ACDE700244FF0FF39A246F6
:10367000264644E7069B0393CDE60023FBE7284656
:10368000FEF770FE0528804602D04FF003092AE1BC
:1036900099499A480CF0DAFA0A22414697480CF008
:1036A0003EFB96480CF0E2FA4FF4007229460AA855
:1036B00002F01AF901220AA90EA801F0C6FB44F48F
:1036C000807444F001044FF0000B47E02846FEF7F9
:1036D00049FE062880460DD1894988480CF0B6FA83
:1036E0000A22414685480CF01AFB84480CF0BEFAC9
:1036F0000222E0E7834981480CF0A8FA0A224146F9
:103700007E480CF00CFB7D480CF0B0FABDE74FF49E
:1037100080312846FEF760FE002871D1B8F1FF3FE6
:1037200008D1284600F0AEFD0028D4BF4FF00008B5
:103730004FF00108B8F1000F5DD14FF40072294637
:103740000AA802F0D1F801220AA90EA801F07DFB17
:1037500044F4807444F001044FF0060B0AA801F011
:103760001AF900286BD10AA844F0010401F01FF9EE
:10377000002867D044F40074039B13B124F4007450
:10378000A4B2224629460AA802F052F84FF00109D5
:10379000BAF1000F40F05C836869002840F0E481D2
:1037A0004FF400312846FEF717FE002800F0E581AF
:1037B000554950480CF04AFA4E480CF057FA630548
:1037C00000F1E88251494D480CF040FA0A2249467E
:1037D0004A480CF0A4FA4E4948480CF037FA0DF06C
:1037E00031F8079B0A22C11A44480CF0A4FA434856
:1037F0000CF03CFA77E0474940480CF027FA44E7E0
:103800004549F9E7B8F1FF3F08D1284600F03AFDF5
:103810000028D4BF4FF000084FF00108B8F1000FA6
:103820000BD002220AA90EA844F4807401F00DFB0B
:1038300044F001044FF0050B90E73849DCE744F40D
:10384000807490E74FF4007229460AA801F012FB39
:1038500000288FD190E7B8F1FF3F08D1284600F04B
:1038600011FD0028D4BF4FF000084FF00108B8F157
:10387000000F2B49214818BF01260CF0E7F90A2256
:1038800041461E480CF04BFA26491C480CF0DEF964
:103890000A22314619480CF042FA18480CF0E6F9B1
:1038A0000998002844D0FEF773FC08902846FEF7DC
:1038B00059FD0FFA80FB089BBBF1000F01D10FFAF5
:1038C00088FB002B5BD09B4530D017490B480CF090
:1038D000BDF90A22594609480CF021FA07480CF0B4
:1038E000C5F96FF00209484611B0BDE8F08F00BF7E
:1038F000567C010084030020627C010068030020E4
:10390000777C01008E7C0100427D01009E7D0100DC
:10391000A97D0100AC7C0100C67C0100DB7C0100BC
:10392000F87C0100067D01000D7D01000023099354
:10393000029B012B30D1039B1BB10AA801F037F881
:1039400003900AA801F0D2F9152800F2F880DFE808
:1039500010F0B700CA00A7002600B7009700740057
:103960005000B700B700F300F30004010401E100C8
:10397000E100F600F600F600E100E100E100686910
:103980000028D5D0049A0368CDE900620AAADC6A4F
:10399000099B06CAA0473CE400230393D1E72846CD
:1039A000FEF7E0FC052806467FF46FAE8D498E4891
:1039B0000CF04CF90A2231468B480CF0B0F98A48D9
:1039C0000CF054F94FF4007229460AA801F08CFF5C
:1039D0002B7C052B0CBF0E2201220AA90EA801F098
:1039E00034FA44F4807444F001044FF0000B0126D3
:1039F00068E02846FEF7B6FC0628064616D17B4945
:103A000079480CF023F931460A2277480CF087F9FF
:103A100075480CF02BF90AA90EA8022201F015FA3C
:103A20004FF400212846FEF72FFDDAE770496E4873
:103A30000CF00CF90A22314662E64FF48031284638
:103A4000FEF7CAFC00287FF4DBAEB8F1000F7FF46C
:103A5000D2AE4FF4007229460AA801F045FF0122B8
:103A60000AA90EA801F0F1F944F480744FF4002182
:103A70002846FEF7C9FC44F001044FF0060BB6E7F8
:103A8000B8F1000F3FF4D9AE02220AA90EA844F4FF
:103A9000807401F0DAF944F001044FF0050BA6E759
:103AA0000AA800F078FF064600285BD02846FEF7FB
:103AB00059FC05283FF4E9AD44F4807444F0010456
:103AC0004FF0000B039B002B3FF462AE049B00936E
:103AD0000AAA08F0010306CA284624F40074FEF777
:103AE000CDFFA4B254E60AA800F055FF00283FF429
:103AF0007CAFB8F1000F0DD03E493B480CF0A6F862
:103B000028460121FEF73CFC4FF488512846FFF778
:103B1000BFFABAE50AA800F03EFF064610B30AA8AD
:103B200000F045FF28B94FF4007229460AA801F0B9
:103B3000DBFE44F44074C1E744F4806455E70AA80E
:103B400000F024FF08B144F480740AA800F02FFFAD
:103B5000064638B144F40074B2E74FF0000B4FF45E
:103B6000806444E7B34642E703680AAA5B6B06CA6F
:103B7000984700287FF414AE1AE6D5F81480B8F1FF
:103B8000000F39D00AAF24B122462946384601F049
:103B90004FFE049A68690368CDE90062DE6A099BFA
:103BA00097E80600B047814668690368DB6B984771
:103BB000052808BF44F0010414F4806F18BF4FF0CB
:103BC0000109BBF1000F03D059462846FEF7D8FB88
:103BD000069B002B3FF4F6AD21462846FFF758FA26
:103BE000F0E500BF627C010068030020777C0100E3
:103BF0008E7C0100297D01002B7C052B75D0062BC6
:103C0000DFD10AA800F0C2FE00286ED04146284647
:103C1000FEF752FC074606B20AA801F067F8049BBB
:103C20008046002B47D024B1224629460AA801F03D
:103C3000FFFD002EC5D0BCBF7E4236B206F1FF3379
:103C40009BB2B4BF01270027192BBAD801213046F7
:103C50000CF0E6FFB8F1150F09D8012303FA08F8B4
:103C60007D4B18EA030F35D118F0A40F3AD17B49E8
:103C70007B480BF0EBFF0A22314679480CF04FF8F5
:103C8000784977480BF0E2FF0A22059974480CF056
:103C900046F873480BF0EAFF304606F015FC28B1F1
:103CA0002846FEF75BFE08B902F0C0FD44F48074BC
:103CB00044F0010468E0304606F006FC0028B2D06B
:103CC00069496A480BF0C2FF68480BF0CFFF6FF0FC
:103CD000040908E687F001030593194630460CF005
:103CE000C7FFC4E705973946F8E724B122462946BD
:103CF0000AA801F09DFD029B022B48D0032B09D09E
:103D0000012B7FF45EAF44F4807444F00104DDF8CD
:103D1000089056E72846FEF7A3FC030C064605D19B
:103D20002B6853491A6853480BF020FA384600F0C4
:103D300099FE0EF0B3FA504B00220EF007FB0EF086
:103D4000B5FD0FFA80F8082006F0A2FB68F30F0615
:103D5000074660F31F46494941480BF077FF0A22A6
:103D600041463F480BF0DBFF45493D480BF06EFFF5
:103D7000B9B20A223A480BF0D2FF39480BF076FF6D
:103D800031462846FEF784FC4FF0010919E744F458
:103D900000748DE7069B002B3FF414AD29464FF4C9
:103DA00080620AA801F044FD4FF4806115E700F03D
:103DB00039FE00287FF49DAA04468046FFF7A0BA8A
:103DC000029AAAB91B78002B3FF404AA09A8FEF7AF
:103DD00037FD0290384601F03FF828B99DF80820D9
:103DE00039460EA801F03CF8029B002B3FF4F2A9E3
:103DF00024491B480BF02AFF0A22214618480BF0E1
:103E00008EFF214916480BF021FF2B6814481968D2
:103E10000BF025FF1D4912480BF018FF09991048B7
:103E20000BF01DFF1A490E480BF010FF384601F049
:103E3000ABF9099B002B3FF4E0A91B78242B7FF4FE
:103E4000DCA9144906480BF001FF05480BF00EFFF2
:103E50006FF0030947E500BF42C03000817D0100DB
:103E600068030020F37A0100747D010084030020C0
:103E7000867D0100E003002000005940957D01008F
:103E8000997D0100157C0100207C0100277C010048
:103E9000147B01002D7C01002DE9F04F8FB080468E
:103EA000CDE90221002900F0688106F04BF8B0F559
:103EB000966F044610DAB249B2480BF0C7FE0A22E8
:103EC0002146B0480BF02BFFAE480BF0CFFE4FF071
:103ED000FF300FB0BDE8F08F029B0BB11B782BB900
:103EE00098F8183013B108F118030293029BE3B954
:103EF000D8F8286016BB402103980FF081FF0028F6
:103F000039D00446002304F8013B0398214606F00B
:103F1000D9FA039481460024039D2F5D6FB3384680
:103F200010F0CBFF28550134F6E71B78002BDFD0CB
:103F300002A8FEF785FC06460028D9D00D2EDAD15E
:103F400008AC00221146204600F0A2FB039A21464D
:103F50000AA800F06EFF324621460AA800F080FF52
:103F60000023019301230093029B94E8060040463E
:103F7000FFF7F0F8ADE78146CDE7284600F03AFBC1
:103F800004ACC2B205463946204600F081FB052E3E
:103F900024D0062E08BF17255FFA86FA0AAF5246CC
:103FA0002146384600F05CFF092D19DC082D80F20F
:103FB000D480AA1C03DB6B1C40F3DF80D5B103A8BF
:103FC00005F017FF024618B12146384600F0B1FE51
:103FD00001230093CDF804900023C6E71825DBE702
:103FE000172D00F08980182DE9D10022214638468E
:103FF00000F02BFF06AD03A9284605F01BFF524633
:104000002946384600F02CFF284600F071FE10F1DA
:10401000000A18BF4FF0010A4FF0000B039A0FFA85
:104020008BF35AB1BBF1030F07D003A805F0E1FEF3
:1040300047F82B000BF1010BF0E75B460B2E0DD080
:104040000C2E13D00A2E19D1284600F0EBFC81B2B9
:10405000204600F093FBCDF8049083E7284600F05B
:10406000E1FCC1B2204600F0A3FBF4E7284600F0D3
:10407000D9FC0146204600F0ACFBECE753449BB270
:10408000013B032B30D8DFE803F00207122095E84C
:10409000030084E80300DEE7284600F0C3FC9DF837
:1040A000283082B2214608A800F08CFED3E72846CB
:1040B00000F0B8FC9DF82C2000929DF8283082B2C8
:1040C000214608A800F067FEC5E7284600F0AAFCD4
:1040D0009DF82C200092214682B29DF8283008A835
:1040E00000F059FE0C99C5E7274926480BF0AEFDB4
:1040F00024480BF0BBFDAEE700222146384600F015
:10410000A4FE0025039A2BB242B1042D0AD003A8C5
:1041100005F06FFE47F825000135F3E7032B10D0BB
:10412000042B98D19DF8341001919DF83010009126
:104130009DF82C309DF82820214608A800F066FE46
:1041400089E79DF8301000919DF82C309DF82820CB
:10415000214608A800F04AFE7DE708AC03A92046E6
:1041600005F068FEEAB22146384600F06EFE52467F
:104170002146384600F074FE6DE70020A9E600BF36
:10418000B07D010084030020C87D01002DE9F04FBF
:104190000E468FB091469A46002856D0037C03F015
:1041A0000F03052B65D1344DC4682B78DFF8CCB0F4
:1041B000DFF8CC8001332B70002C57D0237C03F028
:1041C0000F03042B50D16269DBF8001040460AF05F
:1041D00034FA0746002847D0037C03F00F03052B71
:1041E00042D1014603A8FEF71FFB6EB103A8FEF7FC
:1041F0008FFA48B100230093CDF804A04B463168F4
:10420000726803A8FEF7A6FF0022394640460AF06E
:104210000AFAE8B1037C03F00F03022B18D14369BB
:10422000072B15D10122394640460AF0FCF95346C6
:104230004A463146FFF7AAFF9EB990B12B7803A8F2
:10424000013B2B70FEF784F801200FB0BDE8F08F22
:104250003EB903A8FEF75CFA18B103A800F012F803
:10426000EBE703A8FEF774F86468A5E72B78013B39
:104270002B700020E9E700BF65030020D403002075
:104280006C07002073B5002205461146684600F011
:10429000FFF92B68464819680BF0E1FC4549444892
:1042A0000BF0D4FC2846FEF733FA58B9424940488F
:1042B0000BF0CCFC3E480BF0D9FC4FF0FF3420460D
:1042C00002B070BD2846FEF74DF80646686958B141
:1042D00003681B6B984704B2002C05DB14BF012058
:1042E0000020FEF785FCEAE72B7C072B13D0701C1F
:1042F000152810D80126314C06FA00F0044004D1EC
:1043000010F0490F07D02046EBE72D4928480BF065
:104310009DFC3446D3E74FF400722946684600F00E
:10432000A9FD2B7C033B062B3AD8DFE803F03520B0
:104330003939043520006B681B7C03F00F03052B13
:1043400034D120491A480BF081FC002319461A4643
:104350006868FFF71BFF1C49044615480BF076FC04
:104360002046FEF745FC12480BF080FCA7E7002131
:10437000684600F04FFC044614490D480BF066FCFB
:1043800021460A220A480BF0CAFC09480BF06EFCD1
:10439000003418BF012492E7684600F043FBEAE7C7
:1043A0000B4903480BF052FC002488E70024E3E7A4
:1043B00068030020147B0100117E0100848030001E
:1043C000117B0100FD8101001A7E0100277E0100A2
:1043D0001D7E0100F0B54FF4006185B00546FDF784
:1043E000FBFF002847D0002202AC1146204600F017
:1043F0004FF94FF440722946204600F03BFD6B69AF
:10440000002B38D04FF400612846FEF73DF81B49D9
:104410001B480BF01BFC6869002301260268CDE9EC
:104420000063D76A94E80600B847431C044622D0CC
:104430002B68134819687CB90BF011FC114910481E
:104440000BF004FC10490E480BF000FC0C480BF07C
:104450000DFC204605B0F0BD0BF001FC09490848F1
:104460000BF0F4FB094906480BF0F0FB04480BF095
:10447000FDFB3446EDE70224EBE700BFA57B01001E
:1044800068030020CC7B0100E68701000681010063
:104490002DE9F04F044689B08946FFF79BFF0522BE
:1044A000216847480AF0BFF80646002872D0037C0E
:1044B00003934FEA131A45690CF0C4F9BAF1000FDF
:1044C00068D0A5EB000804AD52460B21284606AF84
:1044D00000F0DEF842462946384600F02AFCB9F1E1
:1044E000040F17D10023009395E806004FF4005302
:1044F0002046FEF78BFB0A224FF47A71314898FB75
:10450000F1F10BF0EAFB30492E480BF09FFB2D48F0
:104510000BF0ACFBB8F1000F3CDA2C4B984539DBC3
:1045200005F010FD4FF00008CDF8008083464FF4F1
:10453000005395E806002046FEF768FBBBF5966F32
:1045400010DA234923480BF081FB0A2259462148FF
:104550000BF0E5FB1F480BF089FB4FF0FF3009B073
:10456000BDE8F08F337C68F307133374524641463D
:10457000384600F08DF8039B03F00F03DA1F534217
:10458000534101930123009397E8060043462046D8
:10459000FEF7E0FDB9F1010F02D12046FEF7B8FDAC
:1045A000606908B90020DAE703689B69984700282A
:1045B000F8D0606903680FFA89F19B689847CEE7E5
:1045C0006C07002068030020D57D010002000080F8
:1045D000E47D01008403002007B5002300931A4600
:1045E000194603480BF0EAFA03B05DF804FB00BF7C
:1045F00030030020F8B50646F0B10378E3B12D2B67
:104600001ED0A3F13002092A1AD9252B1AD07B2BF0
:104610001AD0232B1BD00F4F012404EBC4053D44BB
:1046200028460FF028FC2946024630460FF03FFC92
:1046300020B10134192CF0D14FF0FF342046F8BDE1
:104640000024FBE70824F9E76FF00104F6E71724DC
:10465000F4E700BF447E0100F8B5064690B1037848
:1046600083B10A4F002404EBC4053D4428460FF0F3
:1046700002FC2946024630460FF019FC20B10134F5
:10468000172CF0D14FF0FF342046F8BD257F0100F4
:1046900010B500238370C370037143718371C371BC
:1046A00061F307134370027010BD10B50023072497
:1046B00003708370C37064F307134370416010BDCF
:1046C00093B2112B70B516469CBF134AD25C4B783F
:1046D00088BF002262F307134B7005460C460F4853
:1046E0000F490BF0B3FA0A2231460C480BF017FBC6
:1046F0000C490A480BF0AAFA617808480A2209090D
:104700000BF026FB05480BF0B1FA23682B606368B9
:104710006B60284670BD00BF327E01006803002038
:104720006A800100758001004B781B09013B082B52
:104730001AD8DFE803F0160E0E19191919050C0026
:104740000C4B4B600B6803604B68436070470A4B2F
:10475000F7E764238B71CB7923F00103CB7100233E
:104760004B71FF230B71EDE700230B714B718B71C4
:10477000CB71E7E70000A0410000964243781A0998
:1047800003D0022A05D000207047022262F30713EB
:10479000437040F26D139942A8BF1946C3798171E5
:1047A00023F00103C1F300211943C17101207047B7
:1047B00043781A0903D0022A05D00020704702224C
:1047C00062F3071343706429A8BF6421417101207B
:1047D000704713B50446084631B9E37960F34703DF
:1047E000E371012002B010BD642300934FF4FA720C
:1047F000002399210BF0B1FE63781A0908D0032A2F
:104800000BD820EAE0706428A8BF64200130E4E7F8
:10481000022262F307136370F3E70020E2E707B5B3
:10482000C27912F0FE0F11D043781B09013B022B15
:104830000CD850084FF4FA73009364229923002196
:1048400001380BF08AFE03B05DF804FB4FF0FF3037
:10485000F9E7C379827903F0010342EA0320704744
:104860004079704743781B09013B10B50A2B53D898
:10487000DFE803F00606525252482F2F2F10100087
:104880000279642391FBF3F1114481F30801017172
:10489000012010BD632944684FF064030FDC03FB63
:1048A00004112AB153439942A8BF194621EAE17184
:1048B00043784160062262F307134370E8E791FBF7
:1048C000F3F12144E2B19142A8BF114621EAE1711E
:1048D00016E0436807EE903AFDEEE77A642417EE9F
:1048E000903A91FBF4F1194422B19142A8BF1146CC
:1048F00021EAE17107EE901AF8EEE77A17EE901AC6
:104900004160C5E743681944002AF9D06423534342
:104910009942A8BF1946D9E70020BAE743781B0996
:10492000022B1ED1C279837902F0010243EA0223ED
:10493000642291FBF2F11944B1F5B77F0FDA40F22E
:104940006D1331EA210128BF1946C379817123F023
:104950000103C1F300211943C171012070470021F7
:10496000F3E70020704743781B09022B0CD14379F1
:10497000642291FBF2F1194421EAE1719142A8BF4E
:1049800011464171012070470020704700780030C7
:1049900018BF01207047437803F00F03012B04D8A0
:1049A0000078003018BF012070470020704743781E
:1049B00013F0F00F14BF012000207047407800F082
:1049C000E000202804D0A0F140035842584170472D
:1049D0000120704743781B09013B0A2B1ED8DFE8F2
:1049E00003F00A0A1D06061B0F0F0F060600436898
:1049F0006420584370470079642310FB03F070472C
:104A000043689FED077A07EE903A67EE877AFDEEEE
:104A1000E77A17EE900A70474068704700207047A9
:104A20000000C84243781B09013B0A2B18D8DFE875
:104A300003F00808170606120A0A0A06060040686C
:104A4000704700797047406807EE900AFDEEE77AFC
:104A500017EE900A70474068642390FBF3F07047AC
:104A60000020704743781B09013B0A2B1ED8DFE862
:104A700003F013131D06060E1919190606004368E4
:104A800007EE903AF8EEE77A17EE900A704743681F
:104A9000642293FBF2F3F3E7037907EE903AF8EE22
:104AA000677AF1E7436807EE903AEDE7DFED017AC8
:104AB000EAE700BF0000000043781B0907B50B2B95
:104AC00060D8DFE803F06216165F5F5F44245F5F23
:104AD0000606406849B1D0F1640056D46428A8BFE6
:104AE000642000B203B05DF804FB0028F6DA084643
:104AF000F8E7007931B1002100916423FF220BF027
:104B00002CFDEEE764230093FF220B46F7E7436892
:104B100007EE903A99B19FED1F7A77EE677AF5EE3E
:104B2000C07AF1EE10FA30D4F4EEC77AF1EE10FA52
:104B30002DDCFDEEE77A17EE903A18B2D2E7F5EEEB
:104B4000C07AF1EE10FAD2D49FED127AECE7436806
:104B500061B142F27372934217DC13F1630F16DBFB
:104B60006FF0630093FBF0F06430BAE713F1630F6A
:104B7000BDDB42F2737293424FF06400B2DC93FBF0
:104B8000F0F0AEE74FF0FF30ACE70020AAE764207A
:104B9000A8E700BF0000C84213B504460846637882
:104BA0001B09013B0A2B32D8DFE803F00F0F31312C
:104BB00031281A3131060600FF23009300236422B6
:104BC00019460BF0CAFC606007E0FF230093002346
:104BD000642219460BF0C1FC2071012002B010BD07
:104BE000FF2300930023642219460BF0B6FC07EE66
:104BF000900AF8EEE77A17EE900AE4E746F29C3363
:104C000000930023642219460BF0A7FC606000208B
:104C1000E4E7000043781B090B2B5FD8DFE803F0C3
:104C20006117175E5E5E461E5E5E0606406841B115
:104C3000002839DBFF28A8BFFF20C0F1FF0001B228
:104C40000AE0002808DBFF28A8BFFF20F7E700796B
:104C50000029F4D0C0F1FF01084670474368A9B1AC
:104C600007EE103AB5EEC07AF1EE10FA1CD4DFED83
:104C70001E7AB4EEE77AF1EE10FA32DC77EEC77AFC
:104C8000FDEEE77A17EE903A19B2E5E707EE903AB3
:104C9000F5EEC07AF1EE10FADED49FED137AF4EE61
:104CA000C77AF1EE10FAEBDDFF21D5E7406859B184
:104CB00010F1630FF8DBB0F5C84F12DA6FF0630143
:104CC00090FBF1F0FF30BAE710F1630FC4DBB0F5F1
:104CD000C84FE9DA642190FBF1F0B0E74FF0FF3103
:104CE000BAE70021B8E700BF00007F4300787047B3
:104CF0004078000970474B7810B562F307134B708A
:104D00000B6803604B68436010BD4B7810B51C09FD
:104D1000013C012C84BF012464F3071382F30802D1
:104D2000D2B288BF4B700B680A7103604B68436056
:104D300010BD4B784A6030B50A2565F307134B70F8
:104D40000B6803604B68436030BD4B784A6030B5F8
:104D5000072565F307134B700B6803604B684360CE
:104D600030BD4B7830B5062565F307134B700A2329
:104D70005A434A600B6803604B68436030BD4B7810
:104D80004A6030B5062565F307134B700B68036066
:104D90004B68436030BD70B54C788A71022666F36B
:104DA00007144C70C2F30024CA794B7122F001023F
:104DB0009DF810300B7122430B68CA7103604B6879
:104DC000436070BD70B54C788A71032666F3071492
:104DD0004C70C2F30024CA794B7122F001022243C5
:104DE0000B68CA7103604B68436070BD70B54D7845
:104DF0004B71042666F307159DF810304D700B714A
:104E00008A710B6803604B68436070BD70B54D7864
:104E10004B7105269DF810300B7166F307159DF850
:104E200014304D70CB718A710B6803604B6843601E
:104E300070BD4B784A6030B50C2565F307134B7095
:104E40000B6803604B68436030BD10B50A700B6897
:104E500003604B68436010BD407800F00F0070475E
:104E60004B7810B562F303034B700B6803604B681B
:104E7000436010BD2DE9F041044616460D4619B9B0
:104E800000273846BDE8F0810846FDF741FC07469B
:104E90000028F5D02846FDF783FBF305804603D5AF
:104EA0002846FDF75FFA207006F40076B8F1000F8F
:104EB00009D0637868F307136370002EE1D0AB6804
:104EC0005B696360DDE7002EDAD0AA68137C03F02B
:104ED0000F03022B03D0032B09D04746D1E7637899
:104EE000526962600A2161F307136370C9E753696D
:104EF0006278072161F307126270E2E710B50023C0
:104F00000446037043708370C370037143718371EF
:104F1000C3714FF40072FFF7ADFF204610BD70B5AE
:104F20000446C8B1037C03F00F03042B10D146697B
:104F30003046FFF791FB051E0EDB304609F072FC90
:104F4000237C6561022262F303032374284670BD4B
:104F5000022B01D14569F9E74FF0FF35F6E7000074
:104F60002DE9F0432DED028B85B004461546994698
:104F70009DF838800F46002948D0002A00F0E780CD
:104F800000230B70017871B319F4807F2BD0714B23
:104F900001EBC101194438460EF09BFF637813F012
:104FA000F00F07D019F4007F04D02A466A4938462A
:104FB0000EF069FF38460EF05EFF2D1A3E18013DD7
:104FC000637813F0F00F21D019F4007F1ED01B0975
:104FD000013B0B2B1AD8DFE803F0084071A6AC2583
:104FE0007B7B7B221FB43E46EAE72079B8F1000FB5
:104FF00006D0642300930023FF2219460BF0ADFA7C
:10500000564A0346294630460EF02AFE384605B079
:10501000BDEC028BBDE8F0836368514AF2E7636838
:10502000504AEFE7616800294FF064020EDA91FB05
:10503000F2F04B4202FB1011494293FBF2F34A4A51
:105040000091294630460EF00BFEDFE791FBF2F3AC
:1050500002FB13120092454AF3E72046FFF7DFFBFD
:10506000E279A37994F8059001B20029207902F041
:10507000010202DBB8F1000F14D043EA0224B8F1B8
:10508000000F06D0642300930023FF2219460BF083
:1050900064FACDE900902346354A294630460EF0A1
:1050A000DFFDB3E7CDE90101CDF8009043EA02232B
:1050B000304A294630460EF0D3FDA7E7E379A279BE
:1050C0006179009103F0010342EA03232A4AB8E719
:1050D000636808EE103AB5EEC08AF1EE10FA4CBFE4
:1050E000F1EE487AF0EE487AFDEEE78AB8EEE87A1B
:1050F00077EEC77A9FED217A67EE877A17EE900AEE
:105100000BF07CFE07EE900AB5EEC08AFDEEE77A62
:10511000F1EE10FACDED007A18EE903A01D5184A6A
:105120008FE7184A8DE72279A3790192627900927C
:10513000B2E7E279A3790292227901926279009230
:10514000B6E72A46616830460EF0C3FE5EE71746B2
:105150005CE700BF447E0100147B01008B800100EE
:105160008E800100928001009680010097800100EE
:10517000A3800100A0800100A680010000007A4405
:10518000AC800100AD80010030B58BB0134C002322
:105190002022009302A94FF440730546FFF7E0FE7A
:1051A00002A920460AF05BFD0D4920460AF04EFD9B
:1051B00069780A22090920460AF0CAFD09492046F1
:1051C0000AF044FD69780A2201F00F0120460AF036
:1051D000BFFD20460AF04AFD0BB030BD6803002039
:1051E000788001007D80010070B54B78B2EB131F11
:1051F00086B005460C46164606D123682B606368C8
:105200006B60284606B070BD184919480AF01EFDAB
:10521000617817480A2209090AF09AFD15491448CD
:105220000AF014FD0A22314611480AF091FD124994
:105230000F480AF00BFD0023CDE9043366F3071392
:1052400022788DF811304FF0FF338DF81020009345
:1052500002A86368226804A900F010F8029B23608A
:10526000039B63602046FFF78FFFC6E7B580010010
:1052700068030020727A0100147B01002DE9F04FD1
:105280008DB004AD85E80C00BDF85830112B98BFE7
:10529000B64A804628460C4694BF12F803904FF059
:1052A0000009FFF7BCFA011E02DB2046FFF791FA66
:1052B0009DF811306278C3F3030161F30302627059
:1052C0009DF810102170C2F303120B2A38D8DFE8C2
:1052D00012F0A0000C000C00C9002F010D01A80065
:1052E000CF00CF00CF00A800A8001B090C2B77D857
:1052F000DFE803F0265244180A0739557676303035
:105300006E009DF81720E2719DF81620A2719DF89D
:10531000152062719DF814202271627863F30712E0
:1053200062700DE0BDF81630C3F30802E379A27194
:1053300023F0010343EA1223E3719DF815306371F2
:10534000B9F1000F00F0FC804A46214606A8FFF79D
:105350004BFFF5E0059B002B36DBFF2BA8BFFF239F
:10536000DBB22371ECE7059B13F1630F2CDBB3F584
:10537000C84F2BDA642293FBF2F3F1E7BDF8163045
:10538000C3F30802E379A27123F0010343EA122375
:10539000E3719DF8153063719DF81430E1E7DDEDA0
:1053A000057AF5EEC07AF1EE10FA0DD49FED707A21
:1053B000F4EEC77AF1EE10FA08DCFCEEE77ACDEDF8
:1053C000027A9DF80830CCE70023CAE7FF23C8E73C
:1053D00063780C2262F307136370059B6360AFE789
:1053E000644965480AF032FC9DF8111062480A22AF
:1053F00009090AF0ADFC61495F480AF027FC6178B1
:105400005D480A2209090AF0A3FC5B480AF02EFC59
:1054100096E762781B0963F3071205986270606073
:105420008EE71B09032B04D00C2BD1D0059A6260A8
:1054300073E700212046FFF7EDFBBDF81630207121
:10544000C3F30802E379A27123F0010343EA1223B4
:10545000E3719DF8153063716378022262F30713DC
:1054600063706DE700212846FFF7D4FB2071F3E756
:105470001B090C2BB4D801A252F823F041530000B1
:10548000BB540000E954000033540000E95400000C
:10549000E9540000B1540000DD540000DD54000068
:1054A000DD540000C9540000D7540000D15300005F
:1054B000059B636006226378D0E79DF8143007EE01
:1054C000903AF8EE677A03E0DDED057AF8EEE77AD8
:1054D00017EE903A82E7DDED057AF2E7627863F342
:1054E00007126270059B79E7627894E701271B0930
:1054F0000C2B3FF675AF01A252F823F04153000088
:1055000055550000A95500005555000035550000BF
:10551000355500005555000055550000E153000079
:10552000E15300005555000055550000D1530000CF
:105530000027DCE7059A6260627863F30712627005
:105540002368C8F800306368C8F8043040460DB0DE
:10555000BDE8F08F013B0A2B00F2CD80DFE803F0BD
:10556000BACB10CBCBBFC4CBCBBDBD00327E0100CC
:1055700000007F43F47F010068030020727A01007D
:10558000FF23BDF816208DF81430642161F3080262
:10559000ADF8162000228DF815209DF8112002216B
:1055A00061F307128DF811200023FF259DF81500E7
:1055B0000095642219460AF0D0FF0028C0F29D80B1
:1055C00000239DF815000095642219460AF0C5FFD6
:1055D000A84208DC002300959DF8150064221946B6
:1055E0000AF0BBFF05469DF81400FAF747FF064690
:1055F000002F47D09DF817707F08013F3FB27B1CFA
:1056000040F088807F2D4FF0FF0778DC0023C5F144
:105610007F00194647F68162704300970AF09DFFAC
:105620004FF4FF73009300231946E0717F22284650
:105630000AF093FF0023194600903A4630460AF0DC
:105640008CFF00970646642328467F2200210AF03B
:1056500084FFBE420546A8BF3E466B496B480AF030
:10566000F5FA0A22294669480AF059FB6849674851
:105670000AF0ECFA0A22314664480AF050FB63480B
:105680000AF0F4FA00231A46194606A80AF056F959
:10569000BDF816004FF6FF7300930023194640F241
:1056A0006D12C0F308000AF058FFF2B2E9B280B2FE
:1056B0000AF05AF9030CA371030A6371207155496A
:1056C00052480AF0C3FA2046FFF75EFD06A80AF02A
:1056D000CAF835E69DF8143053E7059B51E7059B62
:1056E000642293FBF2F34CE7DDED057AFDEEE77AF9
:1056F00017EE903A45E7002343E7002573E764235C
:10570000284600973A4680210AF027FF00230546E5
:10571000E371A2E74FF01E0B64231A46CDF800B0E8
:10572000002138460AF019FF4FF0640A03905B46E7
:105730003846CDF800A0524600210AF00EFF7F2D1A
:1057400083464FF0FF0754DCC5F17F000023704310
:105750001946314A00970BFB00F00AF0FEFE4FF4A9
:10576000FF73E0710398009300231946E322281881
:105770000AF0F3FE00231946029000903A463046A4
:105780000AF0EBFE00230646009728467F221946C2
:105790000AF0E3FEBE420546A8BF3E461F491B482D
:1057A0000AF054FA0A22039918480AF096FA1C499A
:1057B00016480AF04BFA0A22594614480AF08DFAA4
:1057C000184912480AF042FA0A2229460F480AF0FC
:1057D000A6FA15490D480AF039FA0A2231460B4853
:1057E0000AF09DFA114909480AF030FA0A22029992
:1057F00042E75346284600973A4680210AF0ADFE1C
:1058000000230546E371C9E7068001006803002014
:105810001380010046800100646A3100218001008C
:10582000278001002D800100358001003D800100AE
:10583000F8B5054617460C4611B900263046F8BDA6
:105840000846FCF765FF06460028F6D079050CD51A
:105850002B780A3B032B08D8DFE803F01F02242A29
:105860004FF480312046FCF7CFFDFA0507D52978A3
:10587000A1F10A03032B02D92046FCF781FDBB05E9
:105880001BD56B7869681B09073B2046042B1FD882
:10589000DFE803F011111E1B1B004FF4803120467E
:1058A000FCF7F2FD4FF400312046FCF7EDFDDCE79C
:1058B0004FF40031D6E7FCF7A9FE094909480AF080
:1058C000C5F92846FFF760FCB8E7FCF783FEF4E76C
:1058D000FCF780FE697820460909FCF7B3FEECE787
:1058E000848001006803002073B504460D46FFF76D
:1058F000C1FA0646E8B9104910480AF0A7F9284647
:10590000FDF720FC214602B26846FEF7D9FE21468B
:105910006846FEF709FF29464FF400722046FFF75C
:1059200087FF2046FFF730FC4FF490512846FDF7E3
:10593000AFFB304602B070BD4D800100680300200F
:1059400043781B09013B012B37B5054620D80023BE
:10595000FF2400790094642219460AF0FEFD002815
:1059600014DB002328790094642219460AF0F5FD1F
:10597000A04207DC002300942879642219460AF02B
:10598000ECFDC4B22C71012003B030BD0024F9E756
:105990000020F9E707B5002300931A46194603488B
:1059A0000AF00CF903B05DF804FB00BF38030020D7
:1059B00002F06CBD02F02CBD07B5002300931A461F
:1059C000194603480AF0FAF803B05DF804FB00BF7B
:1059D00040030020024B0F221A70C820704700BFFE
:1059E000D803002008B5044904480AF02FF904F050
:1059F000A7FB4FF4FA7008BDFB850100B40300203B
:105A000038B5094D01244FF47A700AF04FFF214652
:105A100001340A222846E4B20AF09AF9142CF2D191
:105A20004FF4FA7038BD00BFB403002008B503F08E
:105A3000BDFFC82008BD10B5044604300AF097FD2C
:105A4000204610BD0128F8B507460C46174E184DE4
:105A500013DD48680CF0E3FFC1B216483170FBF764
:105A600026F9022F07D0A0680CF0D9FFC1B2114867
:105A70002970FBF72DF9C82401E04FF4C8740E49D2
:105A80000E480AF0E3F80A2231780C480AF060F96F
:105A90000B490A480AF0DAF80A22297807480AF07E
:105AA00057F906480AF0E2F82046F8BD0500002044
:105AB000060000203C04002090870100B403002071
:105AC000A487010030B587B00023044600931A462E
:105AD0000D4602A819460AF071F804A80AF066F803
:105AE000042C12DD04A9286904F034FA68B104A971
:105AF0002548FAF7C4FF04A9E86804F02BFA50B16E
:105B000004A92148FBF707F80BE002A91E48FAF7A1
:105B1000B6FF032CEFDC02A91B48FAF7FCFF022CAE
:105B20001CDD04A9A86804F015FAB8B104A9164848
:105B3000FAF7CBFF04A9686804F00CFAA0B104A935
:105B40001148FAF776FF114911480AF07FF8002151
:105B50000D48FBF77CF8C82007B030BD02A90A4801
:105B6000FAF7B3FF012CE5DC02A90748FAF761FF59
:105B7000012CE8D102A90448FAF75BFF0549044863
:105B80000AF064F8DFE700BF3C0400205D820100FA
:105B9000B40300204D82010008B548B149680548AA
:105BA000FAF7CCFD044905480AF050F8C82008BDB2
:105BB0000146F4E73C040020BF820100B40300204A
:105BC00008B548B149680548FAF7E3FD04490548B6
:105BD0000AF03CF8C82008BD0146F4E73C04002068
:105BE000E5850100B403002030B5144D144C85B098
:105BF000772201212846FBF795FA00230193114BE8
:105C00000093114902954FF0FF33204603930AF0A9
:105C10001DF80E4B0E4819686A4608F0D3FC28465A
:105C2000FBF72CFA0B4920460AF010F820460AF040
:105C30001DF80948FBF736F905B030BD54040020C3
:105C4000B4030020C4950100448501003004002005
:105C50006C0700205E8501003C040020012810B57F
:105C60000C4622DD124960680EF09DF818B901213A
:105C70001048FAF7D1FF104960680EF094F8014619
:105C800010B90C48FAF7C8FF0C490D4809F0DEFFBF
:105C90000848FAF7B8FF0A22014609480AF03FF817
:105CA000074809F0E3FFC82010BDFFF79DFFFAE7A2
:105CB000E28D01003C040020E58D01006E850100AD
:105CC000B403002010B50C48FBF7A6F818B10B4937
:105CD0000B4809F0BBFF0B4C722201212046FBF759
:105CE00021FA237D1BB1FF212046FBF7B9F90548B6
:105CF000FBF7C4F9C82010BD3C040020FA8801005D
:105D0000B403002054040020034B93F9000005382D
:105D100018BF0120704700BFD803002030B593B0F2
:105D200000230A460546402101A804F085F901A890
:105D30000EF0A1F801A90446024628460EF0B7F875
:105D400000280CBF2046002013B030BDF0B504463B
:105D50009DB00E4601B18AB96A496B4809F076FFD9
:105D60006A49694809F072FF2146674809F077FFE0
:105D70006749654809F06AFF634821E000258D54B2
:105D800004F0E0F85F4907465F4809F05FFF0A2228
:105D900039465D4809F0C3FF5E495B4809F056FF8C
:105DA0002146594809F05BFF5B49574809F04EFF0F
:105DB000B7F59D7F08DA5949594809F047FF584817
:105DC00009F054FF1DB0F0BD04215648564F03F0B2
:105DD0004BFF56494C4809F039FF31464A4809F013
:105DE0003EFF5249484809F031FF474809F03EFF5D
:105DF0003C2229460DA80C950DF097F897F9002044
:105E0000052A27D103212046FFF788FF05B26DBB85
:105E1000474DEB681B78DB07D4D501212046FFF7FF
:105E20007DFF00B20028CDD0242120460EF072F86C
:105E30000028C7D13F49344809F008FF21463248BD
:105E400009F00DFF304809F011FF2146284609F0FE
:105E50002EF9B7E701212046FFF760FF05B2C5B96B
:105E600002212046FFF75AFF05B2C5B12544324949
:105E700028460DF0D2FFA0B930460DF0FCFF0128F6
:105E80000FD921462A4809F012F9304608F0F2FCF1
:105E900098E73F2221460CA80EF01BF8E6E72749B9
:105EA00067E7204624210EF035F80446002889D102
:105EB000294601A8FCF7EEFC01A8FCF729FCE0B19B
:105EC0002246314601A8FDF7E7FF002815DD9DF8C1
:105ED000303093B197F90030052B0ED018490A489D
:105EE00009F0B4FE0CA9084809F0B9FE064809F00B
:105EF000BDFE0CA90E4809F0DAF801A8FCF728FA53
:105F000060E700BFE595010068030020F68101000D
:105F1000289B0100FF81010002820100058201002F
:105F20008403002034040020D8030020EC79010011
:105F3000E003002012820100708D01002A8201001E
:105F4000358201002DE9F04116491748174E184FC8
:105F5000154D09F07BFE0024A6F10F0816F8013F4D
:105F60000F2B03D83946284609F079FE052C4FF04F
:105F700010020DD03178284609F0AFFE0D492846B1
:105F800009F064FE0134E4B2062CE7D1BDE8F081EB
:105F900098F81510284609F0A0FE284609F066FE7C
:105FA000F0E700BF7F850100B40300204B04002010
:105FB000A8950100CC7B010010B58AB00DF11F033C
:105FC00004930DF12503039309AB0C4602930DF1E5
:105FD000230301930DF12203009308AA0DF121037D
:105FE0000E4960680DF070FE05280BDC0C490D4869
:105FF00009F02CFE61680B4809F031FE4FF4C870BF
:106000000AB010BD08A90848FAF74BFBFFF79AFF42
:106010000649074809F01AFEC820F1E70D8601007D
:1060200021860100840300203C0400203386010007
:10603000B403002008B508B9002008BD037C03F0B4
:106040000F03052BF8D1CAB20146064808F0EBFA57
:106050000028F1D0037C03F00F03042BECD140693E
:10606000EBE700BF6C070020F7B53C4C2678002E0C
:106070006CD13B4B93F90030012B67DD394B19682C
:10608000002963D0384A394808F0D7FA0546002875
:106090005CD00146354808F0BCFA07B2002F55D055
:1060A00031462846FFF7C6FF012F064650D0294645
:1060B00001222E4808F0B7FA4569684605F0DAF97A
:1060C00010222B49684603F06BFF2A492A4809F041
:1060D000BDFD3146284809F0C2FD2849264809F08F
:1060E000BEFD0A222946244809F019FE2349224808
:1060F00009F0B5FD1E49204809F0B1FD1E4809F020
:10610000B5FD40F202211E4805F04CFCAAB2314612
:106110001C481D4D09F098FC15491A4809F098FCD7
:106120001A4B186818B10021FFF784FF286029680E
:1061300089B1144809F094FC0021124809F098FC38
:10614000012313490C48237009F080FD03B0F0BD12
:1061500040F20225B1E70F49EBE700BF78040020C9
:10616000D803002030040020B18101006C0700201A
:1061700054030020B8810100B4030020CC7B01004F
:10618000C00400209C04002080030020DC030020C9
:10619000C7810100368E01002DE9F04FA7B0002322
:1061A00096488DF81330CDE90533CDE9073308F073
:1061B00095FD934F054610B105233B70F8E0914CD7
:1061C000216841B99049914809F040FD8F4809F094
:1061D0004DFD0F23F1E78E4808F01BFA0FFA80F807
:1061E000B8F1010FEEDD294620688A4EFFF722FF45
:1061F000002800F0E08030608749884809F026FDDB
:106200003168864809F02BFD844809F02FFD0121F3
:106210002068FFF70FFFB8F1020F824600F0CE8032
:10622000022221687A4808F0FEF9B8F1030FD0F88D
:10623000149000F0C58003212068FFF7FBFE05469F
:10624000102205A97648FAF753FA002840F0BB80DF
:10625000B8F1040F40F3B78004212068FFF7EAFE8D
:10626000704904466D4809F0F1FC6C4809F0FEFCE9
:106270001FFA89F25146614809F09CF80DF1240893
:1062800069495E4809F099F80DF1340B102267490D
:1062900040460DF01EFE002301222021584603F047
:1062A000CBFE634958460DF09CFD62495B4809F0FE
:1062B000CDFC5146594809F0D2FC5F49574809F0D6
:1062C000C5FC0A224946554809F029FD5B49534857
:1062D00009F0BCFC2946514809F0C1FC58494F4817
:1062E00009F0B4FC2B780BB91C461D46CDF80C8088
:1062F0004FF002094FF001082A46CDE90198CDF888
:1063000000B0234631683D484E4D08F0FDFD0028A1
:106310005BD04D4B4D49414800241C7009F096FC60
:1063200031683E4809F09BFC3C4809F09FFC484B13
:10633000032283F800804121234615A803F07CFE48
:10634000444915A80DF04DFD15A92C4809F000F899
:1063500023464A46412115A803F06EFE3E4915A882
:106360000DF03FFD15A93D4809F090FC15A9234803
:1063700008F0EEFF42462346412115A803F05CFEDB
:10638000354915A80DF02DFD15A9344809F07EFCFE
:1063900015A91A4808F0DCFF05233B700AF052FAF1
:1063A0002F4928601D4809F051FC1C4809F05EFC8B
:1063B00027B0BDE8F08F2B4B33601DE740F25B79CF
:1063C0000DF113053CE705AC52E727490F4809F0EA
:1063D0003DFC0A4808F0F3FF0A2201460B4809F089
:1063E0009EFC2249094809F031FC084809F03EFCAE
:1063F0000AF028FA0C232860DFE600BFE003002043
:10640000D8030020DC030020C78A01008403002099
:106410006C07002080030020FD8A0100B4030020E7
:106420003C0400200A8B01004D5D0000D58D010069
:10643000208E01002A8B0100CC7B01004A8B0100D9
:10644000008D01008804002020040020518B0100F1
:10645000660300205F8B0100707A01006803002052
:10646000658B0100368E0100828B01008E8B01004E
:1064700010B5114C1149204609F0E8FB104920469F
:1064800009F0EDFB4FF4FA700AF010FA0121152023
:106490000AF0C6FB002115200AF0EAFB4FF4FA705F
:1064A0000AF004FA152001210AF0E2FB4FF4FA7019
:1064B000BDE810400AF0FAB9B40300204D8D010088
:1064C0006D8D010070B592B002A809F06FFB04A8B1
:1064D00009F06CFB06A809F069FB08A809F066FB47
:1064E00071497248724E09F0B1FB704809F0BEFB69
:1064F00002A97048FAF7C9F9F8B96F496B486F4CAF
:1065000009F0A4FB4FF47A6242F6E0616C4804F0B3
:1065100051FE002840F091806A496B4809F096FBD3
:106520006A49694809F092FB237801332370F62306
:106530003370FFF79DFF12B070BD5E48FAF77FFB26
:1065400018B15E4B1B78022BD7D961495748614C73
:1065500010AD09F07BFB039B10942846119303F0C8
:1065600045FD04A95348FAF7FAF900285DD05A49C5
:106570004E4809F06BFB059B10942846119303F0DD
:1065800035FD06A94B48FAF71FFA002841D05349B8
:10659000464809F05BFB079B10942846119303F0D3
:1065A00025FD08A94348FAF7A5F910B34C493F481F
:1065B00009F04CFB099B11932846109403F016FD3B
:1065C000039B0095CDE90B34059B3D480A94CDE92A
:1065D0000D34079BCDE90F34099B11930CAA0EAB28
:1065E0000AA904F071FE314809F040FB0223337020
:1065F000A1E7039B32480C94CDE90D34059BCDE90E
:106600000F34079B11930EAA2B460CA904F08CFEA5
:10661000E9E7039B2A480E94CDE90F342A46059BEF
:1066200011930EA904F0A8FEDDE7039B2448109403
:106630002946119304F0BAFED5E72A491B4809F010
:1066400005FB10A804F016FF119B039310A8214B23
:10665000109303F0CBFC154809F008FB02A915487C
:10666000FAF7E7F9204B13485B68119304A90593E7
:10667000FAF72BFA10A804F041FF119B0D4807937D
:1066800006A9FAF748FA10A804F016FF119B09486A
:10669000099308A9FAF7F3F901210648FAF7D7FA9E
:1066A00000232370A2E700BF38880100B403002054
:1066B000D80300203C040020458801004803002046
:1066C0004C0400207988010084030020BB8801006D
:1066D0005188010090960100678801006D880100D3
:1066E00072880100EA8801005806002007B51049A9
:1066F000104809F0ABFA684604F0BCFE684603F0A7
:1067000075FC0D4B00930D4B68465B68019303F0DD
:106710006DFC684604F0F2FE684603F067FC6846CC
:1067200004F0CAFE684603F061FC03B05DF804FBA8
:1067300012880100B4030020909601005806002042
:1067400018B10349034809F081BA0349FAE700BFC9
:106750004B8D0100B40300202B9B010010B5264C8B
:106760002649204609F072FA2549204609F06EFABA
:10677000244B1868003018BF0120FFF7E1FF2249C1
:10678000204609F063FA214B1868003018BF012039
:10679000FFF7D6FF1E49204609F058FA1D4B18682E
:1067A000003018BF0120FFF7CBFF1B49204609F03E
:1067B0004DFA1A4B1868003018BF0120FFF7C0FFD0
:1067C0001749204609F042FA164B1878FFF7B8FF30
:1067D000204609F04BFA1449204609F037FA03F035
:1067E000B1FB0A220146204609F0A5FA2046BDE881
:1067F000104009F03BBA00BFB403002059870100E4
:1068000066870100D40300206E870100D0030020BA
:1068100077870100DC0300207E870100240400202C
:1068200087870100780400204F8101000020704715
:1068300010B5444C4449204609F008FA4349204623
:1068400009F004FA4249204609F000FA414920467D
:1068500009F0FCF9204609F009FA3F49204609F001
:10686000F5F93E49204609F0F1F93D49204609F085
:10687000EDF93C49204609F0E9F93B49204609F089
:10688000E5F93A49204609F0E1F93949204609F08D
:10689000DDF93849204609F0D9F93749204609F091
:1068A000D5F93649204609F0D1F93549204609F095
:1068B000CDF93449204609F0C9F93349204609F099
:1068C000C5F93249204609F0CAF93149204609F094
:1068D000BDF93049204609F0B9F92F49204609F0A1
:1068E000B5F92E49204609F0B1F92D49204609F0A5
:1068F000ADF92C49204609F0A9F92B49204609F0A9
:10690000A5F92A49204609F0A1F92949204609F0AC
:106910009DF92849204609F099F92749204609F0B0
:1069200095F92649204609F091F92549204609F0B4
:106930008DF92046234909F089F92046BDE8104029
:1069400009F094B9B40300200A8901002C890100E0
:106950003F8901004D8901005589010065890100C9
:10696000718901007E89010093890100A2890100DB
:10697000AA890100B5890100C2890100CC89010002
:10698000DB890100E3890100EF8901006D8D0100C1
:10699000058A0100248A0100398A0100468A010023
:1069A000548A0100608A0100688A0100738A01002C
:1069B000808A0100888A0100938A0100A28A01006E
:1069C000AB8A0100B98A010008B5FFF731FFFFF774
:1069D0008DFE0349034809F039F9C82008BD00BFFE
:1069E000D6820100B403002070B594B003F0AAFA77
:1069F000064609F027FF05462D4808F06FF90028E4
:106A000054D02C4B1C7864B2002C4FD12346012269
:106A1000402104A803F010FB274904A80DF0E1F978
:106A2000264904A80DF0DDF9254904A80DF0D9F98F
:106A30003146684603F07EFB01236A4604A91C48E0
:106A400008F0A9FB23460122402104A803F0F4FA30
:106A5000194904A80DF0C5F9184904A80DF0C1F9A9
:106A6000184904A80DF0BDF968464FF47A71B5FBDA
:106A7000F1F103F05FFB01236A4604A90C4808F01A
:106A80008AFB23460122402104A803F0D5FA0E49CF
:106A900004A80DF0A6F90F220C4968460DF019FA6A
:106AA00001236A4604A9024808F075FB14B070BDC2
:106AB000E0030020B0030020278E01009B86010028
:106AC000838D01003F8E0100208E01001A8E01008F
:106AD00010B50C4C2046F9F7B5FD78B90A490B48BA
:106AE00009F0B4F8DE232374AD236374BE23A374CA
:106AF000EF23E374FE232375FF236375BDE8104085
:106B0000FFF720BA3C040020BE850100B40300203A
:106B100008B5002007F06AFF1C491D4809F096F8E7
:106B20001C491D4807F0F0FE1C491D4807F0ECFE0B
:106B30001C491D4807F0E8FE1C491D4807F0E4FE0B
:106B40001C491D4807F0E0FE1C491D4807F0DCFE0B
:106B50001C491D4807F0D8FE1C491D4807F0D4FE0B
:106B60001C491D4807F0D0FE1C491D4807F0CCFE0B
:106B70001C491D4807F0C8FE1C491D4807F0C4FE0B
:106B80001C491D48BDE8084007F0BEBE84850100D1
:106B900068030020C9690000888501005D5C000071
:106BA0008D850100D559000092850100397B0000D8
:106BB000A08E0100B95F000097850100015A000016
:106BC0009B850100C55A0000A0850100995B00006B
:106BD000A6850100C15B0000A3850100C55C000023
:106BE000AA850100E5590000B0850100455A000062
:106BF000B48101002D5A0000B78501002DE9F04F46
:106C0000364D2B6885B00746002B63D0344C267870
:106C100076B2002E5ED12278DFF8CC90DFF8CC80FF
:106C2000013252B2227099F80020013252B289F832
:106C30000020D8F800A009F005FE334601460B22DB
:106C4000504603F08DFA4E4600283BD02B68DFF803
:106C5000A0A0DD68DFF89CB05DB32B7C03F00F03D0
:106C6000062B24D152462946584607F0E6FCA8B127
:106C7000037C03F00F03052B10D1D0F80C90B9F171
:106C8000000F14D049462A4601A8FAF7DFFA394620
:106C900001A8FBF7E3F9D9F80490F0E729460022B0
:106CA00001A8FAF7D3FA394601A8FBF7D7F96D68BE
:106CB000D2E7032F03D009F0C5FDC8F8000009484A
:106CC000FBF750FA3378013B5BB233702378013B1A
:106CD0005BB2237005B0BDE8F08F00BFD003002089
:106CE000CD0300202C030020650300208404002035
:106CF000C77A01006C0700200220FFF77FBF000069
:106D000010B5094C237801335BB2237009F0F0FD14
:106D10000320FFF773FF09F0EBFD07F055FE237822
:106D2000013B5BB2237010BDB00300202DE9FF4191
:106D30001E4F3B68002B35D01D4B1E7876B28EBBA4
:106D40001C4C1D4D2278013252B22270D5F80080C1
:106D500009F078FD3346014641F28832404603F09F
:106D6000FFF92E46D0B13B68DD68A5B12B7C03F05E
:106D70000F03062B08D12946002201A8FAF766FA6C
:106D8000012101A8FBF76AF909F0B2FD0220FFF723
:106D900035FF6D68E9E709F055FD30602378013B68
:106DA0005BB2237004B0BDE8F08100BFD0030020C7
:106DB000CD030020650300209004002030B5114B66
:106DC000196885B0D9B1104CCD682278013252B221
:106DD000227085B12B7C03F00F03062B07D1002214
:106DE000294601A8FAF732FA01A8FBF78FF909F052
:106DF0007FFD6D68EDE72378013B5BB2237005B042
:106E000030BD00BFD0030020650300202DE9F04F06
:106E1000934C23688FB0002B00F01C81914F3B787E
:106E2000002B40F017813B788F499048904D0133FB
:106E30005BB23B7008F00AFF8C4808F017FF8D4AE0
:106E400021688D4807F0F9FB8C4A286021688A4840
:106E500007F0F3FB8A4B8B4A18602168864807F0DD
:106E6000ECFB894B894A18602168834807F0E5FBF1
:106E7000874B1860FFF7F8F8864A21687E4807F0CC
:106E8000DCFB854BA946186070B1844C23785BB954
:106E900002F08EFD002814BF01230023237003D0CD
:106EA0007F49724808F0D2FE7E4A00231360D9F869
:106EB00000309246002B00F0AF80D3F80C80DFF852
:106EC00010B2794DD9F80030002B00F0C680B8F12F
:106ED000000F00F09E8098F8102002F00F02052AA3
:106EE000F2D14146644807F094FB0128EAD94146B3
:106EF00003A8FBF799FC03A8FBF70AFCA8B103A8B9
:106F0000FBF79CFA064680B9014603A8FBF7D4FAC2
:106F1000041E03A8BCBF64420126FBF723FA9DF8B8
:106F20001C20052A09D0062A44D009F0E1FC03A858
:106F3000D8F80480FBF70CFAC4E718B9022103A8BB
:106F4000FBF71EFA4FF4807103A8FBF75DFA059B6F
:106F500023B14FF4007103A8FBF756FA20B203F0F7
:106F6000B3FA064660B15149514808F06FFE0A2253
:106F700021464F4808F0D3FE4D4808F077FED4E78D
:106F80000121204609F04CFE3146204609F070FEF2
:106F90005946284608F05AFE21460A22284608F09B
:106FA000BEFE4449284608F051FE4349284608F0F1
:106FB0004DFEBAE701900121204609F031FE20B2D2
:106FC00003F082FA019B20B10021204609F050FE17
:106FD000ABE7D6B113F1FF3618BF01263146204684
:106FE00009F046FE3549284608F030FE0A222146BF
:106FF000284608F094FE3249284608F027FE0A2267
:107000003146284608F08BFECFE7013B5E425E41E9
:10701000E4E7DB68CAF8003023482A4C08F026FE73
:10702000FFF7CCFEFFF79AFB274B284801221A7086
:1070300004F0C4FA20B1254804F082FB0423237035
:1070400094F90030072B04BF042323703B78013BE5
:107050005BB23B700FB0BDE8F08FDB68FFDE00BFB6
:10706000300400206503002064810100B403002087
:10707000D4030020748101006C0700207B8B010089
:1070800098040020287A0100D00300207A810100B2
:10709000DC0300207F81010024040020280400205C
:1070A000828101002C0400206803002092810100ED
:1070B00084030020AA810100AF810100817D0100CD
:1070C000F37A0100D8030020640300209C03002011
:1070D000A28101002DE9F0433B4C23688DB0002BC9
:1070E0006ED03A4D2E6809F0ADFB002301464FF4F7
:1070F0007A72304603F034F8074610B109F0A2FB6B
:107100002860334DDFF8D4902B7801335BB22B70BD
:107110002368DE687BB2002B14BF4FF004084FF0E9
:1071200002082268F2B1EEB1337C03F00F03052BA5
:10713000F8D13146484607F06CFA0128F1D93146BA
:1071400001A8FBF771FB01A8FBF7E2FA18B1414671
:1071500001A8FDF79DF909F0CBFB01A87668FBF7C4
:10716000F7F8DEE72B78013B5BB22B70194B93F9F4
:107170000030052B24D01FB3174F00263D46396839
:10718000F1B1EEB90B7C03F00F03052B0CD101A874
:10719000FBF74AFB012101A8FDF77AF9061C01A8BB
:1071A00018BF0126FBF7D4F82B684BB109F0A0FB00
:1071B0002B685B682B60002BE1D12368DB682B60B8
:1071C0000DB0BDE8F08300BFD40300208C04002084
:1071D00065030020D80300202C0400206C07002049
:1071E000F8B580EAE074A4EBE074054620B20E46E0
:1071F00003F06AF9074668B11549164808F026FDFC
:107200000A222146134808F08AFD1248BDE8F840DA
:1072100008F02CBD0121204609F002FD022E09D103
:107220003946204609F024FD0B490C4808F00EFDB4
:107230000A48EBE736B9E943C90F204609F018FDC3
:107240000749F2E7E90F204609F012FD0549ECE78E
:10725000E081010084030020EE810100680300202A
:10726000258F0100308F01002DE9F04F2DED048BAB
:107270008A4B95B01C6809F0E5FA0023014647F2F5
:107280003052204602F06CFF002800F00081844B51
:107290001A68002A00F0FB808249D4680B78DFF876
:1072A00054929FED819A01335BB20B700025002C44
:1072B00000F0BF80237C03F00F03052B13D10022C5
:1072C0002146484607F0AFF94369052B0BD121460B
:1072D00009A8FBF7A9FA09A8FBF71AFA804620B912
:1072E00009A8FBF735F86468E1E709A907A8FDF7E5
:1072F00005FE09A8FBF7B4F90021064609A8FBF72B
:10730000DBF8054607A8FDF7ADFB08EE900A09A8D3
:10731000FBF728F833B207EE903AF8EEE77A8346A7
:1073200087EE898A09A8FCF7ADFF6049824660486C
:1073300008F08CFC022718EE900A0AF0AFFF0097C5
:1073400002460B46CDE90401594808F0BDFD5949F4
:10735000574808F07BFC18EE100A0AF09FFF0097D0
:1073600002460B46CDE90201514808F0ADFD5249F5
:107370004F4808F06BFC59460A224D4808F0CFFCF4
:107380005FEA164B50D0082003F082F84FF6FF73E7
:1073900081B240F62712584602F0E2FEC8B12168D9
:1073A000464808F05CFC4649444808F04FFC226817
:1073B0004449454807F0DAFEB1B209A8FBF768F97D
:1073C00039462846FFF70CFF09A8FAF7C1FF4546E2
:1073D00089E7DFED3E7AB4EEE78AF1EE10FA04DDDC
:1073E00022683B49384807F0C1FEBAF1000F01D1CD
:1073F0000121E6E70022374BDDE904010AF0EEFD4A
:10740000DDE902230BF032FA08B10021D9E7F4EEEE
:10741000C88AF1EE10FAEBD92F49254808F016FC7E
:10742000234808F023FCCFE72C49214808F00EFC44
:10743000CAE71C4C2378013B5BB2237009F002FAC7
:10744000164B1860FFF7D0FA35B32549184808F0F5
:10745000FDFB02F077FD0A220146154808F06BFC9F
:107460002049134808F0F2FB217811480A2249B25A
:1074700008F055FC1C490E4808F0E8FB1B4B0C4873
:1074800019680A2208F057FC094808F0EFFB15B00C
:10749000BDEC048BBDE8F08F1549D7E794040020BC
:1074A000D4030020650300200000C8420A810100C7
:1074B0006803002010810100A67C010084030020E5
:1074C0001681010026810100E0030020000018421F
:1074D000328101000000F03F3F8101001C8101006A
:1074E0004E810100548101005C8101007C04002078
:1074F000147B01006C0700202DE9F043644E3368D3
:107500008DB0002B00F0C280002832D101276149E4
:10751000614D624808F09AFB604808F0A7FB2B78A1
:107520005F4A01335BB22B7013689046002B61D029
:10753000DC68DFF8A091002C63D0237C03F00F03FC
:10754000052B14D12146484607F063F878B121682D
:1075500001A8FBF79FF901A8FBF7DAF810B101A821
:10756000FAF7F0FE09F0C4F901A8FAF7F1FE646831
:10757000E1E74C4949484C4CDFF8748108F066FB60
:10758000464808F073FB09F05DF927460546237865
:10759000EBB109F057F90023014642F21072284678
:1075A00002F0DEFD98B907F00FFA98F80030D3B971
:1075B0003E4B93F90030052B01D0FFF78BFDFFF711
:1075C00053FE0220FFF71AFB09F092F9DFE73B7840
:1075D000002B9BD03649374808F038FB354808F077
:1075E00045FB002793E7344B1B68002BE0D002F0EB
:1075F00015FBDDE73149294808F028FB274808F04A
:1076000035FB2F4B2F49254800241C6008F01EFB3A
:10761000224808F02BFB642009F048F92A4B2B493B
:107620001C702B4B1D481C7008F010FB02F08AFCEC
:107630000A220146194808F07EFB3168254806F009
:107640000AFC254B25491C60254B14481C60254B22
:1076500034601C60244BC8F800401C60164B1C6052
:1076600008F0F4FA02F06EFC0A2201460B4808F01A
:1076700062FB0A4808F0FAFA1C4B1C702B78013B9D
:107680005BB22B7038460DB0BDE8F0830127F9E7F7
:1076900030040020058D01008004002068030020D4
:1076A000D4030020CD8C010065030020D803002006
:1076B000E28C010084030020240400201B8D0100C3
:1076C0002C0400202B8D010078040020338D010054
:1076D000640300206C070020D00300202D7E0100F1
:1076E00098040020DC0300208003002066030020B3
:1076F00028040020F0B5454C267876B289B027469C
:10770000002E47D123784249424D434801335BB2B2
:10771000237008F09BFA404808F0A8FA7222012171
:107720002846F9F7FFFC2846F9F78AFC7B2846D162
:107730003A493B4808F08AFA394808F097FA394B39
:10774000049330464FF0FF33079305960695FFF7F5
:10775000D3FE04A93448354E06F092FE3060284628
:10776000F9F78CFC3568BDB93149324808F06EFA3A
:10777000304808F07BFA304901A808F03DFF01A924
:107780002E48F9F70BFB01A808F0F1FE2378013B26
:107790005BB22370002010E029491F4808F056FA18
:1077A0001D4808F063FA2378013B5BB22370FFF7B2
:1077B0002DFB2248F9F7B8FB012009B0F0BD28469F
:1077C000F9F722FC98B12B7D1BB1FF212846F9F770
:1077D00047FC194904A808F00FFF04A91748F9F756
:1077E000DDFA04A808F0C3FE1448F9F75BFB09486A
:1077F000F9F744FC1349084808F028FA064808F04D
:1078000035FA3B78013B5BB23B70C3E76503002070
:10781000B987010054040020B4030020D48701007C
:1078200068030020C49501006C070020300400208C
:10783000E287010084030020E69501003C0400205B
:10784000EE870100018801002DE9F041C0B0002160
:107850001C2214A813910BF068FB202213A99B484B
:10786000F8F7C2FF78B92022994913A80CF031FB30
:107870009849994808F0EAF913A9974808F0EFF9F0
:10788000954808F0F3F9914D6A7D2B7C04922A7D8E
:107890000392EA7C0292AA7C01926A7C00924021C7
:1078A0008E4A1BA80CF0DCF98D498B4808F0CEF904
:1078B00013A9894808F0D3F91BA9874808F0CFF924
:1078C000854808F0D3F94FF47A730022CDE90F23ED
:1078D000844A0E922BAC08228DF84820ADF84A302D
:1078E00013AA50230EA9204605F03CFF4FF47A63FB
:1078F0007D497E483B9308F0A9F902F023FB0A2258
:1079000001467A4808F017FA784808F0AFF920469F
:1079100005F057FF1BA9204606F07AF87449064681
:107920000AA808F069FE294607A8F9F7F3F9079AAB
:107930000A99204605F04AFF07A808F018FE0AA891
:1079400008F015FE204606F060F8002E40F0B780E3
:10795000204606F06BF8DFF8DC810646204606F08C
:10796000D7F9074600B3214607A806F0D5F84146E7
:107970000AA808F041FE0AA907A808F0E6FE074693
:107980000AA808F0F4FD07A808F0F1FD002FE5D0E3
:1079900021460AA806F0DAF80AA92846F9F7FEF9FE
:1079A0000AA808F0E4FDD9E752494B4808F04EF91F
:1079B0000A223146484808F0B2F9474808F056F91B
:1079C000C82E70D14C4B4D490A9348480C944FF047
:1079D000FF330D930B9708F039F902F0B3FA0A223E
:1079E00001464248464D08F0A6F9404808F03EF9E5
:1079F0000120FFF781FD43493C4808F027F93B4847
:107A000008F034F93D49394808F020F902F09AFAB3
:107A10000A220146354808F08EF9344808F026F964
:107A20000AA9394806F02CFD2860204605F0BEFE64
:107A30002C68C4B93549364808F008F9354907A813
:107A400008F0DAFD07A92148F9F7A8F907A808F016
:107A50008EFD2646304B2B933DA808F088FD30461E
:107A600040B0BDE8F0812D49204808F0EFF802F061
:107A700069FA0A2201461D4808F05DF91B4808F022
:107A8000F5F8FFF7C3F92649134808F0DFF8254B4E
:107A90001B78002BDED00D48F9F7B5F80028D9D0B7
:107AA000FEF7A2F8D6E7B6F5987F0CBF1E491F492E
:107AB000174808F0CBF8204605F078FECAE71C49C5
:107AC000134808F0C3F84FF0FF36C3E73C0400202A
:107AD000A88D01003C860100B40300205A860100F5
:107AE00089860100249401009D860100680300201E
:107AF000B3860100C6860100C49501000E8701000F
:107B000030040020D98601006C070020EF860100B8
:107B100084030020E69501003095010006870100EE
:107B200014870100640300201B8701002F870100D8
:107B300049870100C1860100012838B50C4630DDB7
:107B40004D682F4928460CF02EF928B901212D48FF
:107B5000F9F79AF8C82038BD2B4928460CF023F9CC
:107B600001460028F3D02949294808F06FF8254834
:107B7000F9F780F80A220146254808F0D0F8244891
:107B800008F074F861681F48F8F754FE61682048EF
:107B900008F065F81F491E4808F058F81C4808F01E
:107BA00065F81D4C94F90030012B1FDDFFF74CFEEA
:107BB000C82802D104232370CDE7431C10D11749F4
:107BC000174808F043F8164808F050F8154B1648C7
:107BD00000221A700323237003F0B2FDC920BAE714
:107BE000124B1B78002BE5D10F23E4E71049114815
:107BF00008F02CF80F4808F039F84FF4FA70AAE7AB
:107C0000E28D01003C040020E58D0100708201003E
:107C1000B403002090820100D80300209782010065
:107C200068030020660300209C03002064030020FA
:107C3000B2820100840300202DE9F3470024324D75
:107C400000942246214623463048314FDFF800A1F8
:107C500007F0B4FF28464FF47A762E4B6C60AE6086
:107C600040F8143B4FF0080807F0A0FF85F820808B
:107C70002946294D0122384607F0CEFE4FF0010972
:107C800000943B4629460722244802F037F83B4639
:107C90002946CDF800900322214802F02FF80094E5
:107CA0003B4606221F4F20482946204D02F026F869
:107CB0004FF48053C5E901462B611D491D4B2B60D4
:107CC000381D85F8204008F097FC3D601A4D1B498F
:107CD0005246384609F08CF8C5E90146184C194B54
:107CE00019482B60494685F810806E8201F0BAFF72
:107CF0002946204607F07EFB14495246204602B032
:107D0000BDE8F04709F074B8C00400204C0300201F
:107D10009C04002080940100D40700206803002008
:107D2000840300203C040020B403002054040020FD
:107D3000E6950100387A01009C030020375A0000C4
:107D4000E0030020249401003404002049EA0000EC
:107D5000000000202DE9F0470024C8B03C22214655
:107D600009A808940BF0E1F87C22214629A8289460
:107D70000BF0DBF823460122402108A802F05CF951
:107D8000AF49B04EB04F08A80CF02BF87F22AF4996
:107D900028A80CF09EF8012328AA08A9AC4807F0EF
:107DA000FAF923460122402108A802F045F9A94921
:107DB00008A80CF016F87F22A74928A80CF089F82B
:107DC000A64928A80CF00DF8012328AA08A9A04864
:107DD00007F0E1F923460122402108A802F02CF91E
:107DE0009F4908A80BF0FDFF7F229E4928A80CF0B0
:107DF00070F8012328AA08A9954807F0CCF9234672
:107E00000122402108A802F017F9974908A80BF0B1
:107E1000E8FF7F22954928A80CF05BF8012328AAE7
:107E200008A98B4807F0B7F933783D6801335BB296
:107E30003370002D00F03B818D4BDFF86092B3F87A
:107E40000080ADF800801E2221460DF102000BF0EB
:107E50006CF83E2221460DF16200ADF86080DFF83B
:107E600040A2DFF840820BF060F8ED683B68002B21
:107E700000F0AE80002D00F0AB802B7C03F00F03F0
:107E8000052B40F08E802946404606F0C2FB0028B4
:107E900000F0878028680BF0EEFF013404440022D4
:107EA0002946404606F0BFFB4369112B12D8DFE894
:107EB00003F07C87877C7C097C7C7C7C1111111110
:107EC000111111871F226B4968460CF002F800233C
:107ED0008DF8603000230122402108A802F0ACF8A0
:107EE0003F22296808A80BF0CEFF494608A80BF0EE
:107EF00078FF514608A80BF074FF01235E4A5448EE
:107F000008A907F0ADF900230122402108A802F0DA
:107F100093F83F22296808A80BF0B5FF494608A846
:107F20000BF05FFF554908A80BF05BFF0123544A93
:107F3000474808A907F094F900230122402108A826
:107F400002F07AF83F22296808A80BF09CFF4D49FF
:107F500008A80BF046FF514608A80BF042FF01238A
:107F60006A4608A93A4807F016F99DF86030C3B18F
:107F700000230122402108A802F05EF83F22296870
:107F800008A80BF080FF3F4908A80BF02AFF3B49E7
:107F900008A80BF026FF012318AA08A92C4807F00F
:107FA000FAF808F0A5FC6D6860E71F2236496846BC
:107FB0000BF08FFF35493F2218A80BF08AFF89E7A5
:107FC0001F22334968460BF084FF3F223149F3E713
:107FD00000230122402108A802F02EF82E49DFF8E4
:107FE000C4901B4D08A80BF0FCFE0123621E08A9DB
:107FF000174807F04AF93B68DC683B68002B53D010
:10800000002C51D0237C03F00F03052B14D1214603
:10801000484606F0FEFA78B1D4F8008040460BF0EE
:108020002AFF41460246284606F0FFFC63681BB162
:108030002C21284606F0ECFC08F05AFC6468DCE7CA
:10804000208E010065030020D40300201A8E010059
:10805000E0030020FA8D0100598E0100468E0100D8
:10806000278E0100928D01000C8E01008C8D010085
:10807000C1800100068E0100F58D01002E8E0100E9
:10808000B48D01006A820100ED8D0100A28D010016
:10809000008E0100E98D0100138E01006482010051
:1080A000798D01006C070020044806F0A6FD3378A6
:1080B000013B5BB2337048B0BDE8F087E0030020BD
:1080C00070B5A44C94F900300B3392B01A2B2BD816
:1080D000DFE813F0F300E3002A002A002A002A0058
:1080E0002A002A002A002A002A001B0047004A0012
:1080F00053009100AE00D3002A002A002A002A0073
:108100002A000301100125011F01934B93481B789E
:10811000002B14BF0921012101F0A5FD03F05CF93A
:10812000022801D0FEF7CEF994F90030012B40F37C
:1081300046818B4B1B78002B40F0368103F056F9BB
:10814000054603F049F9022800F03081013D042D75
:1081500000F23581DFE815F03701390147014901A7
:108160002A0102232370DFE77E4D2B781BB9FDF730
:108170007BFF01232B700323F4E7774D77482B789F
:10818000002B14BF0B21032101F06DFD764B1B78F2
:10819000002B40F02C817548F8F76CFDE8B1744B6A
:1081A0001B78C3B9FFF750FBC82801D10423D9E7D6
:1081B0002B783BB16F49704807F048FD6E4807F0D7
:1081C00055FDF3E701A803F055F9029B0BB10F230E
:1081D000C8E7F623C6E76949EDE72B784BB10423DE
:1081E00067496548237007F031FD634807F03EFD9D
:1081F0009AE70F23F4E7584B58481B78002B14BF1D
:108200000B21032101F02FFD5E4B196841B95E4936
:10821000594807F01BFD584807F028FD0723A1E740
:108220005A4806F0F6F90128F1D9FDF7B5FF7BE7CA
:10823000574B1D6808F006FB002301464FF4FA5225
:10824000284601F08DFF00283FF46EAF0023032283
:10825000412101A801F0F0FE4E4901A80BF0C1FD3B
:1082600001A94D4807F077F8FFF774FD06234B4945
:108270004148237007F0EAFC56E7374B37481B7834
:10828000002B14BF0A21022101F0EDFC424806F048
:1082900025FD00287FF448AF88E708F0D3FA3C4B6F
:1082A0001860F52323702C4B2C481B78002B14BF2F
:1082B0000921012101F0D7FC36E7354B1D6808F094
:1082C000C1FA0023014641F28832284601F048FFF6
:1082D00000283FF429AF002344E72F4806F0FEFCB6
:1082E00010B12D4806F0C7FC08F0ACFA284B186016
:1082F0000D2337E7264B1D6808F0A4FA002301463A
:1083000042F21072284601F02BFF00287FF44EAF96
:108310000AE708F097FA1E4B18600E2322E7FFF7D2
:10832000E9F9054600287FF441AF194B1E6808F0B3
:1083300089FA2B46014647F23052304601F010FFD1
:1083400000283FF4F1AE1649164807F07FFC01F013
:10835000F7FEE9E6D803002064030020340400207F
:1083600048030020CC030020650300203C040020CB
:1083700066030020A68B0100B4030020CD8B010012
:10838000DD8B0100DC030020178C01006C0700204E
:10839000880400205F8B0100E00300202A8C01008C
:1083A000418C0100840300200025CAE611491248CF
:1083B00007F04CFC104807F059FCF623237094F9A1
:1083C000000012B070BD0D49F1E70D490D4807F0EE
:1083D0003DFC01A803F04EF801A801F007FE094892
:1083E00007F044FCEBE70849E1E70849EEE7032022
:1083F000E7E700BF648C0100840300206D8C01005E
:10840000818C0100B40300209E8C0100B18C01001E
:1084100008B5184801F029FC08F06AFA06F0D4FA09
:10842000FFF74EFE022802DD134806F07FFD08F03C
:108430005FFA124B1B7823B1114B1B680BB101F093
:10844000EDFB104B1B6853B10F4B93F90030052B1C
:1084500001D0FEF73FFE08F04BFAFEF705FF08F0EB
:1084600047FA0220FEF7CAFB08F042FABDE80840CE
:10847000FEF75CBC34040020E00300202804002048
:1084800024040020D4030020D803002010B54FF4AA
:10849000E1311B4807F0F2FE1A48F8F7ABF8044642
:1084A00030BB1949164807F0E7FB21462046FDF787
:1084B00009FC1448F8F71DFC144B18701148F8F724
:1084C00020FC134B1870FEF723FBFEF7B1F9FEF703
:1084D000FFFA142008F0EAF90E490F4806F06DFF84
:1084E0004FF4FA7008F0E2F9BDE81040FFF702B966
:1084F0000A490B4807F0AAFB094807F0B7FBD8E781
:10850000D40700203C040020E18001000500002089
:10851000060000204D5D0000E0030020F680010011
:108520006803002007B5002300931A461946034844
:1085300007F044FB03B05DF804FB00BFE404002037
:1085400001207047032070477047000073B56E46E6
:108550000546304686E80600FCF77EFC04463046B9
:10856000FCF714FA10B1002C08BF01244FF480412D
:108570006868F9F749FF012C1BD0022C04D0FCB924
:108580001C491D4807F062FB3046FCF710FA70B337
:108590006868FAF765F818B90124204602B070BD82
:1085A00000206C6801F074FF01462046FAF770F86D
:1085B000F2E73046FCF79AFB01280AD0022808D0DF
:1085C0000E490D4807F042FB0B4807F04FFB002413
:1085D000E3E76868FAF744F80028DDD000206D680A
:1085E00001F056FF01462846FAF752F8D5E704464F
:1085F000D3E700BF638E0100680300207B8E01007B
:1086000010B5044608F0B6F9204610BD10B5044672
:108610001649174807F03AFB00216068FAF738F866
:1086200023682046DB690021984794F9080001F08F
:108630004BFF40B10F49104807F008FB0E4807F008
:1086400015FB002010BD94F9090001F03DFF002842
:10865000F0D1A17C94F9080008F00AFB94F9090014
:10866000A17C08F005FB0120ECE700BFA48E01000F
:1086700068030020B38E01008403002001292DE946
:10868000FF41044600F089804FF480414068F9F7CB
:10869000A3FE002800F081804FF400416068F9F7E4
:1086A0009BFE60B9764D95F90030002B75D04FF4E4
:1086B00000416068F9F7A8FE2B78013B2B7094F914
:1086C000080001F001FF002867D194F9090001F0CA
:1086D000FBFE0546002860D16068F9F7C1FF2A4615
:1086E0002946074602A8FBF7D3FF4FF400726168E2
:1086F00002A8FCF7BFFB294602A8FCF78BFA064646
:108700006068F9F72FFE022801D0052800D1002665
:1087100094F90A00A0F10E03DBB2072B00F29C8053
:108720004FF0FF0808F086F9E289218ACDF8008031
:10873000002307F012FF051EC0F28A80454500F3B2
:108740008980002F40F08B80751B15F10A0F55DAD8
:1087500094F90900A17C08F08BFA6068F9F780FFB2
:1087600030B9666801F094FE01463046F9F790FF93
:10877000A37C6842002B3CD000210091FF231922EA
:1087800007F0EBFEFF280146A8BFFF21462994F918
:108790000800B8BF462108F0F1F9002004B0BDE898
:1087A000F0813849384807F051FA374807F05EFA47
:1087B0003649354807F06AFAA17C94F9080008F0B8
:1087C00057FAA17C94F9090008F052FA0021606878
:1087D000F9F75EFF4FF480416068F9F755FE4FF4FA
:1087E00000416068F9F750FE254A13780133137091
:1087F000D3E7FF22009219461922C1E70A2DD7DDDF
:1088000094F90800A17C08F033FA6068F9F728FFB2
:1088100030B9666801F03CFE01463046F9F738FF92
:10882000A37C83B100210091FF233322284607F067
:1088300094FEFF280146A8BFFF214629B8BF462164
:1088400094F90900A7E7FF22009219463322EDE7C9
:10885000002576E7454674E77FB14FF0FF3507F016
:10886000F1FF00230146B4F90C20384601F078FCF2
:10887000002896D16B1C7FF467AFA6F17F0564E7F3
:1088800004000020878E010068030020968E0100FE
:10889000002110B5044681744068F9F70DFE43B21B
:1088A000002BBBBF4042207223720123B8BFA374C8
:1088B000237A6068013B182B84BF20232372012197
:1088C000F9F7FAFD43B2002BBBBF404260726372FE
:1088D0000123B8BFA374637A6068013B182B84BF7F
:1088E000212363720221F9F7E7FDC3B2192B8ABF76
:1088F0000023A072A37203216068F9F7DDFD80B246
:10890000431EB3F5806F26BF0023E381E08104217D
:108910006068F9F7D1FD80B2B0F5806F8ABF4FF47F
:1089200080632082238205216068F9F7C5FD00B2CB
:108930000028D6BF42F21073A081A38110BD0000B1
:1089400038B50446F7F755FD2046FFF7A1FF254946
:10895000254807F09BF994F9080001F0B5FD40B1F6
:108960002249234807F072F9214807F07FF90020D7
:1089700038BD94F9090001F0A7FD05460028EFD1A4
:10898000012194F9080008F04BF9012194F909003C
:1089900008F046F9A17C94F9080008F069F9A17C77
:1089A00094F9090008F064F9294694F90A0008F0DE
:1089B00037F929466068F9F76BFE4FF4804160682B
:1089C000F9F762FD4FF400416068F9F75DFD236837
:1089D0002046DB6902219847064B02221A700120CB
:1089E000C6E700BFC08E010068030020B38E0100FF
:1089F000840300200400002007B5002300931A46DA
:108A00001946034807F0DAF803B05DF804FB00BF2D
:108A1000EC040020012070470020704703207047BD
:108A2000704700002DE9F0410646F7F7E2FCB46814
:108A3000002C41D0E468254F254DDFF8A88064B3B1
:108A4000236843B31B7833B33A462146284605F0E2
:108A5000F4FD30B94FF0FF333A462146284605F081
:108A600034FE42462146284605F0E7FD30B94FF076
:108A7000FF3342462146284605F027FE154A214687
:108A8000284605F0DAFD30B94FF0FF33114A214690
:108A9000284605F01AFE6468D1E70F490F4807F031
:108AA000D5F80E4807F0E2F833683046DB6902215A
:108AB00098470120BDE8F0810949084807F0C6F849
:108AC000064807F0D3F82046F4E700BFC49201003F
:108AD0006C070020928E0100878F01006803002040
:108AE000968F0100838E010038B5084D0849044671
:108AF000284607F0ABF8284607F0B8F82368204668
:108B0000DB6900219847012038BD00BF68030020C1
:108B1000758F01002DE9F04F91B008AC0746204653
:108B200084E806000693FCF7E1F80B2800F02882A1
:108B30002046FCF7DBF80A2800F022822046FCF7EA
:108B40008BF983462046FBF721FF20B1BBF1000FD4
:108B500008BF4FF0010B2046FBF718FF90B12046ED
:108B6000FCF77AF907280DD12046FCF7BFF8112849
:108B70006AD012286AD0102804D1FF2221460EA8FC
:108B8000FCF7C3F8BB68002B00F0FA814FF0000837
:108B9000DC68CDF80C80C146C246CDF80880002CB8
:108BA00000F0DE80A24AA348214605F046FDA24A15
:108BB000214605469F4805F040FDA04A064621464D
:108BC0009C4805F03AFD0590002D00F08B80002EAA
:108BD00000F088802B7C03F00F03022B40F0828092
:108BE000337C03F00F03022B7CD1954A9148214638
:108BF00005F023FD43690493069B002B5DD01946C5
:108C000020680BF00AF9002857D108A8FBF7BEFE30
:108C100008BBBBF1070F6FD008AA10460792FBF7FD
:108C2000C6FE079A00283CD0104600210792FBF7A9
:108C3000F1FF6861FDF768F8079A002831D02368D2
:108C400000934FF4007328E0802297E70A21204622
:108C5000FBF7A2FF96E708A8FCF748F8706108A8A0
:108C6000FCF744F801283FD0022843D0FDF74CF828
:108C700058B17369012B08D16B69132B05DC1E22D7
:108C80006A6108A90EA8FCF740F8FDF73DF840B16D
:108C90002368009308AA4FF4407306CA7868F9F76E
:108CA000B5FF059B4BB10023CDE9003308AB0CCBDE
:108CB0004FF0FF31059801F06DFA7369022B0FD068
:108CC00001330DD06B69049A0299434502FB03F20C
:108CD0001144C4BF9846049B0291C4BF91460393BC
:108CE000049B9A4464685AE76A6908A90EA8FCF7CD
:108CF0000CF8BBE70022F8E708A8FBF758FE0028AD
:108D00008AD008A8FBF78EFE7369A8B1022B01D0A8
:108D100001330CD14B494C4806F0A1FF4A4806F0FC
:108D2000A5FF0122726108A90EA8FCF78EF808A819
:108D3000FBF778FE6861A8E7022B0ED001330CD058
:108D40004249414806F08BFF3F4806F08FFF022260
:108D5000726108A90EA8FCF778F800236B6194E70C
:108D6000BAF1000F00F00C8139493748029B93FBA0
:108D7000FAF506F06BFF0A225146334806F0CFFFA2
:108D80003449314806F062FFFF26029B2E4893FBD0
:108D9000F6F10A2206F0C3FF2F492B4806F056FFD2
:108DA0000A222946284806F0BAFF2C49264806F030
:108DB0004DFF99FBF6F10A22234806F0B0FF28493F
:108DC000214806F043FF0A2203991F4806F0A7FF37
:108DD00024491D4806F03AFF1B4806F047FF224A87
:108DE000B968144805F029FC0EAE82462246214699
:108DF0000AA8FBF74DFC2A460AA93046FBF785FF77
:108E00000DF13008002D14BF0122022231464046E8
:108E1000FCF71BF8CDE900444FF0FF3198E80C0057
:108E2000504601F0B7F90DBB012011B0BDE8F08F3D
:108E3000C49201006C070020838E0100188F01008E
:108E40001C8F01001E8F010068030020298F010084
:108E5000358F01003E8F0100498F0100508F0100C6
:108E60005E8F0100658F0100E6950100BB68002B55
:108E7000DAD0DD68434FDFF828B1002DD4D0424A64
:108E80002946384605F0D9FB5A46446929463846F2
:108E900005F0D3FB3D4A80462946384605F0CDFB18
:108EA0003B4A82462946384605F0C7FBB8F1000F19
:108EB00060D0BAF1000F5DD000285BD098F8102088
:108EC00002F00F02022A55D19AF8102002F00F0288
:108ED000022A4FD1027C02F00F02022A4AD1002C52
:108EE00048D04269022A47D0013245D0B9F1000F7B
:108EF00044D0DAF814302968264803FB04FA039BAF
:108F0000CAEB0A2292FBF4F45C4306F0A8FE94FB41
:108F1000F9F421491F4806F0A2FE0A22FF211D484C
:108F20009AFBF1F106F0FBFE1C491A4806F08EFE92
:108F30000A222146174806F0D0FE164806F096FE93
:108F4000D8F81430A34215D0002211460AA8FBF726
:108F50009FFB22460AA93046FBF7D7FE0023CDE946
:108F600000334FF0FF3196E80C00284601F012F96B
:108F7000C8F814406D6880E70024E1E74C46DFE75D
:108F8000002052E76C0700201C8F0100C4920100F2
:108F9000838E010068030020698F01006F8F01003C
:108FA000928E010010B5044607F0E4FC204610BD87
:108FB0000023836043683BB15B682BB11A7C02F0ED
:108FC0000F02062A08BF83607047000007B5002320
:108FD00000931A461946034806F0F0FD03B05DF809
:108FE00004FB00BFF404002043687BB1B0F90A2001
:108FF000042A05D0052A05D0032A05D1022070478E
:109000000120704711207047187C70471846704740
:109010007047000038B50446F7F7EBF928492948AE
:1090200006F014FE0A22B4F90810264806F077FE6E
:109030002549244806F00AFE636822481B6819681F
:1090400006F00DFE21491F4806F000FE1D4806F0FF
:109050000DFE606888B3B4F908307BBB23682046F6
:10906000DB6B98470128054605D002280AD001216C
:10907000B4F9080019E003212046F7F795FA2946CC
:1090800007F0CEFD00212046F7F78EFA012107F008
:10909000C7FD01212046F7F787FA012107F0C0FD3F
:1090A00002212046F7F780FA012107F0B9FD236875
:1090B0002046DB6902219847012038BD0020FCE7EB
:1090C000FC8F010068030020147B01008B910100DC
:1090D00010B504462449254806F0B8FD0A22B4F923
:1090E0000810224806F01BFE2149204806F0AEFD7C
:1090F00063681E481B68196806F0B1FD1D491B48CE
:1091000006F0A4FD194806F0B1FD23682046DB6B8C
:109110009847012805D002280AD00021B4F9080098
:1091200019E003212046F7F73FFA002107F078FD08
:1091300000212046F7F738FA002107F071FD0121E0
:109140002046F7F731FA002107F06AFD0221204698
:10915000F7F72AFA002107F063FD23682046DB6950
:1091600000219847012010BDFC8F010068030020FA
:10917000147B0100258D01002DE9F043044689B0E0
:1091800040689DF840309DF8445002AF87E80600E3
:10919000002800F09880B4F90820002A00F092809E
:1091A000002B00F093800021F9F786F923688146AF
:1091B000DB6B2046984706B2022E19D0032E19D039
:1091C000012E0CBF05210121002204A8FBF760FA43
:1091D0004FF0FF33009397E80C0004A906A8FCF7B2
:1091E0004DF8012E32D0022E27D1002D43D13DE083
:1091F0000421E9E71DB34FEAD9713846B4F90850A4
:10920000FBF708FD80460146284607F0B7FC3049C9
:10921000304806F01BFD0A22B4F908102D4806F06C
:109220007EFD2D492B4806F011FD0A2241462948B2
:1092300006F075FD274806F019FD012043E0B4F95A
:10924000080001F041F90028D5D0E0E703212046CD
:10925000F7F7AAF906462DB19DF81710304607F02A
:109260008DFCC2E701F030F90028F5D0B4F9080010
:1092700001F02AF928B99DF81610B4F9080007F092
:109280007DFC01212046F7F78FF9064685B19DF850
:109290001510304607F072FC20460221F7F784F9DA
:1092A000044655B19DF81410204607F067FCC4E74A
:1092B00001F00AF90028EAD0EEE701F005F90028EC
:1092C000F0D0BAE7104609B0BDE8F0831846FAE7D7
:1092D000817D010068030020F37A010010B5044687
:1092E00007F048FB204610BD07B5002300931A463F
:1092F0001946034806F062FC03B05DF804FB00BFAA
:10930000FC040020032070477047000038B5044675
:10931000F7F76FF82149224806F098FC0A22B4F9C1
:1093200008101F4806F0FBFC1E491D4806F08EFC85
:109330001B4806F09BFCB4F9080001F0C5F805468F
:1093400040B11949194806F081FC184806F08EFC16
:10935000002038BD0121B4F9080007F061FCB4F920
:109360000800A17A07F084FC606810B12946F9F77B
:109370008FF923680221DB69204698476068FAF775
:1093800081FF002807DD0020646801F081F80146B4
:109390002046F9F77DF90120DBE700BF8E90010040
:1093A000680300208B910100B38E0100840300202C
:1093B00038B50F4D0F490446284606F047FC0A22EF
:1093C000B4F90810284606F0AAFC0B49284606F016
:1093D0003DFC284606F04AFCB4F90800002107F0DD
:1093E0001FFC23682046DB6900219847012038BD17
:1093F000680300208E900100258D010010B5044601
:1094000007F0B8FA204610BD002110B5044681725D
:109410004068F0B1F9F750F803B2002BBBBF4042EF
:10942000208123810123B8BFA37223896068013B97
:10943000182B84BF202323810121F9F75DF808F060
:109440002DFF0022054B08F081FF09F057FA08B103
:10945000E06010BD41F28833E360FAE700408F40DE
:1094600030B5044687B000232F22CDE90023ADF8A4
:109470000830B0F90800A37A0D4671B383F00101FA
:1094800007F0F6FBE368B3F57A7F57D331493248EA
:1094900006F0DCFB0A22B4F908102F4806F03FFC66
:1094A0002E492D4806F0D2FB0A2229462A4806F00A
:1094B00036FC294806F0DAFB294968460AF091FC97
:1094C0006068F8F74FFF002D3ED0142807D015280C
:1094D00036D00F2836D1234902E01946D0E7224979
:1094E00003A80AF0A4FC21491B4806F0AFFB6368FF
:1094F0001968236809689D6A03AA6B462046A84735
:109500000A220146144806F00AFC1949124806F0DE
:109510009DFB636810481B68196806F0A0FB69464C
:109520000D4806F09CFB13490B4806F08FFB03A97E
:10953000094806F094FB084806F098FB07B030BDD8
:109540000D49CDE70D49CBE702280CBF0C490D4969
:10955000C6E700BF9A900100680300202D7E01003D
:109560006590010058900100739001009F900100E8
:10957000CC7B0100AB9001006C9001007B9001005E
:109580005C900100609001000129F7B5044644D0C9
:109590004368002B41D0002211466846FBF778F85B
:1095A0004FF4007261686846FBF764FC002168466E
:1095B000FBF730FB05466846FBF798FB6068F9F758
:1095C0004FF8064607F03EF9E268FF216A430023A0
:1095D000B2FBF1F20146304600F0C2FD0746E6B1AB
:1095E00007F030F900230146E268304600F0B8FD8C
:1095F000064620B30020666800F04AFF0146304668
:10960000F9F746F84DB1207A00F04CFFA37A834277
:1096100003D101212046FFF723FF002003B0F0BD56
:109620009FB131462046FFF71BFF6068FAF72AFE1C
:1096300001460028F1D16068F9F72AF8EDE7207AB1
:1096400000F030FFA37A8342EAD1002DE5D0207AE2
:1096500000F028FFA37A8342DFD1002FDDD1D8E7C5
:10966000F7B56E4686E806000446454945489DF82C
:1096700020501F4606F0EAFA3046FBF785FD37B169
:10968000414938460AF0C9FB08B9002051E0636837
:10969000002BFAD0B4F9080000F016FF0028F4D12E
:1096A0003046FBF773F9002845D13046FBF7D4FB71
:1096B000012840D010D302280DD004463349314848
:1096C00006F0C4FA0A2221462E4806F028FB2D484F
:1096D00006F0CCFAD9E7D5B100213046FBF79AFA6B
:1096E000054658B16068F8F7BBFF08BB646800F036
:1096F000CFFE01462046F8F7CBFF19E0014660682F
:10970000F8F7C6FF29462046FFF7AAFE10E060687A
:10971000F8F728FE15280BD8012303FA00F01C4B9C
:10972000184205D029463046FBF774FA0028D9D1F3
:10973000012003B0F0BD3046FBF7D8FA15280DD84C
:109740000125144F05FA00F00740CBD1430705D59A
:1097500039466068F8F79CFF3946D4E70E49094856
:1097600006F074FA3046FBF7C1FA0A2201460548B2
:1097700006F0EEFA034806F079FA01249EE700BFEE
:109780008390010068030020659001007A79010050
:109790000240380002C038006D79010007B500238F
:1097A00000931A461946034806F008FA03B05DF81C
:1097B00004FB00BF0405002090B1C3687BB11A7C94
:1097C00002F00F02042A01D1586948B9D86838B1AB
:1097D000037C03F00F03042B01D140697047002084
:1097E0007047000030B52DED028B054687B008EEBE
:1097F000101A002854D0334B1B68002B50D0FFF7B1
:10980000DBFF0446304806F031FA30492E4806F0B6
:109810001DFA18EE100A08F041FD022302460093DB
:1098200029480B4606F050FB2949274806F00EFA56
:109830002968254806F013FA2649234806F006FA57
:10984000DFED257AB4EE678AF1EE10FA2CD0DFED69
:10985000237AB4EE678AF1EE10FA25D0B5EE408A8D
:10986000F1EE10FA20D01CB12146174806F0F7F9A6
:10987000154806F0FBF904AC18EE101A02A8FAF726
:1098800014FF032202A92046FBF7EAFA0023CDE9E0
:1098900000334FF0FF3194E80C00284600F07AFCCA
:1098A00007B0BDEC028B30BD002CF9D00C49064846
:1098B00006F0CCF92146044806F0D1F9024806F03A
:1098C000D5F9EDE72404002068030020FC90010096
:1098D00001910100819201000000FEC20000AA4235
:1098E000049101002DE9F043284F386889B0002821
:1098F00046D0274E3368002B45D001F085F8254926
:109900002548DFF8A080DFF8A090234C06F09EF9F0
:10991000214806F0ABF901A9386801F0FDF90028EB
:109920002DDD03AA082101A800F004FA002303AAF0
:1099300031688DF81C30404604F07FFE49460546EC
:10994000204606F083F903A9204606F088F98DB178
:109950002846FFF731FF05460028DCD00F49204696
:1099600006F074F92946204606F079F9204606F0FB
:109970007DF9D0E70A49204606F068F9F6E70120AC
:1099800009B0BDE8F0831846FAE700BF18050020CB
:109990002404002039920100B40300202D7E010030
:1099A0004C9201006C070020FC900100FFF79ABF69
:1099B0002DE9F341484C2368002B40F08A80474949
:1099C000474806F043F9464806F050F945494448EF
:1099D00006F03CF900F0B6FA0A220146404806F0CB
:1099E000AAF93F4806F042F9142006F0C1FF0546E7
:1099F00000F0C4FF3C48256000F01AFE206800F02B
:109A0000D7FF00284ED03949394806F035F920688B
:109A100001F00AF9206800F0D7FF3649304806F017
:109A20002BF9206801F044F9002839D032492C483C
:109A300006F022F9314E3068002847D0304D2F68AB
:109A40007FB91C2006F094FF2168804601F0E8F9F8
:109A50004046C5F8008001F0C3FA3946286801F095
:109A6000FDFA3368DFF8AC80DC681D4F336883B3E0
:109A70007CB36946206800F095F950B341463846FA
:109A800006F0E4F82168384606F0E9F8384606F0B2
:109A9000EDF80C226946286801F05FFA6468E5E792
:109AA0001849C4E700F012FD206800F081FF054668
:109AB00038B115490E4806F0C9F80D4806F0D6F839
:109AC000B8E71249124806F0D7F8284602B0BDE8B8
:109AD000F0810120FAE700BF180500207091010015
:109AE000680300200E87010090050020919101007D
:109AF000B4030020A9910100C991010024040020B1
:109B000020050020D5910100E99101000692010095
:109B10008403002022920100034B0146186808B11B
:109B200000F03CBF704700BF1805002037B52F4C30
:109B3000206800F035FF042814D8DFE800F0150392
:109B4000031311002A492B4806F080F8294806F033
:109B50008DF8206801F0ACF841F2883003B030BDD8
:109B60002549F0E72549EEE7206800F021FF28B9F4
:109B70002349244806F080F800F0A8FC224D2B6809
:109B800013B1224B1B683BB921491A4806F05EF815
:109B9000184806F06BF8DFE71E4C22683AB91A7CC9
:109BA00002F00F02062A02D1DB6803B123601A48D3
:109BB000FFF7B2FF2368A3B16946186800F0F2F816
:109BC00078B19DF80030282B0BD16946286801F048
:109BD000D5FA01462068FFF705FE6946286801F0BE
:109BE00073FA23685B682360B6E700BF180500209E
:109BF0001591010084030020299101004291010088
:109C00004D910100B4030020200500202404002011
:109C10006291010014050020F96C000038B5094C70
:109C2000256806F00FFE0023014641F288322846DF
:109C300000F096FA20B1FFF779FF06F003FE2060EE
:109C400038BD00BF1C05002007B5002300931A464D
:109C50001946034805F0B2FF03B05DF804FB00BFEE
:109C60000C050020704770477047704707B5002308
:109C700000931A461946034805F0A0FF03B05DF8AB
:109C800004FB00BF24050020174B1B7870B5044669
:109C90000D469BB1154B027A1B789A420ED8144A96
:109CA0000A291368164616D1124A0021D154406978
:109CB00010B1217A05F048FF00233360E06840B11D
:109CC0000D4B227A1B789A4203D8036829461B68F9
:109CD0009847012070BD4E2BF0DC0D291FBF591C89
:109CE0001160044AD554E9E77804002006000020FA
:109CF00084050020340500200500002030B5002533
:109D000045604361034D9DF80C300560C1600272EF
:109D1000037430BD5C92010007B5002300931A461E
:109D20001946034805F04AFF03B05DF804FB00BF85
:109D30002C05002070B5D0B1CAB14D1E0C4E441E8A
:109D400013462844844203F102030CD014F8015F47
:109D50002D11755D03F8025C257805F00F05755D22
:109D600003F8015CEEE709B2002302F8113070BD80
:109D7000D2920100A0F16103052B02D85738C0B27E
:109D80007047A0F14103052B01D83738F7E7303889
:109D9000C0B2092805D919B101230B700020704702
:109DA0000846704737B500238DF80730F9B1E0B1A8
:109DB000851C4C1E00F1120215F8020C0DF1070172
:109DC000FFF7D8FF000104F8010F0DF1070115F8A6
:109DD000010CFFF7CFFF237802351843954220701E
:109DE000EAD19DF8070080F0010003B030BD0846BD
:109DF000FBE738B50546D8B10468ACB124789CB10E
:109E0000286803783BB12D2B05D0303B092B02D9B4
:109E100001302860F4E708F006FE2C21044628688B
:109E200009F0EEFF10B92860204638BD0130FAE78E
:109E30000446F9E72DE9F7430E46002206210746BE
:109E4000FAF726FC002E55D03368002B52D01B7831
:109E5000002B4FD0D6F8008098F800404CB32D2C42
:109E60006CD0303C092C03D908F101033360F1E7D1
:109E70004146002400220FFA82F9013211F809301C
:109E8000303B092BF7D92E21404609F0B9FF18B312
:109E9000002211B2431801325B78303B092BF8D90C
:109EA0004378A3F13002092A01D82F2B03D80022CE
:109EB00004E0A146E7E7392B88BF09220A2555436C
:109EC0008278A2F13003092B05D82F2A16D9392A16
:109ED00088BF09231D4499B9404608F0A4FD3946BE
:109EE00002466846FAF725FF2C21306809F088FF02
:109EF00010BB3060384603B0BDE8F0830023E9E7CB
:109F0000022940460EDCB9F1070F0BDC08F08BFD8F
:109F10006422424304B16D422A4439466846FAF746
:109F20002EFFE1E708F078FD08F008FD394602460B
:109F30006846FAF70AFFD7E70130DAE708F10101CE
:109F4000012497E708B500200AF0A2FFADEB00005E
:109F500008BD704730B5441E224612F8013F002B61
:109F6000FBD11A460A2514F8010F70B1032A14DC3C
:109F70002E2806D1FF2B10DC881801320371002334
:109F8000F1E7303805FB0303EDE7FF2B04DC032A80
:109F900002DC114401200B7130BD0020FCE7000001
:109FA0002DE9F3410024DFF840800C700D46174680
:109FB000061D0A2201A916F8010B08F04DFF3A46CA
:109FC00001A9284609F05FFF032C04D03A46414618
:109FD000284609F058FF0134A3B2042B1CB2E8D183
:109FE000284602B0BDE8F081038D01002DE9F04163
:109FF0000E4D0F4FDFF83C8006460024032C0ED098
:10A0000033190A221979284605F067FE4146284689
:10A01000013405F01BFE042CF0D1BDE8F081F1798C
:10A020000A22284605F059FE3946F0E7B40300201D
:10A03000147B0100038D01002DE9F047DFF8F0A04B
:10A04000DAF8005004460E4617469946002D49D0CE
:10A050002B7C03F00F03062B43D12C4A2C482946B6
:10A0600004F0EBFA022F804637D0032F37D1294A6C
:10A07000DAF80010264804F0E0FA0546B8F1000FBF
:10A0800030D098F8103003F00F03042B2AD1D8F801
:10A0900014103246204609F01CFF32461E49204665
:10A0A00009F0F1FE0DB32B7C03F00F03042B1CD140
:10A0B00069693246204609F0E6FE324616492046D6
:10A0C00009F0E1FEB9F1000F04D0324649462046BE
:10A0D00009F0D9FE2046BDE8F087104AC8E7002500
:10A0E000CCE7002532460E49D4E7022F0AD0032FD1
:10A0F00005D0012FE1D10B4B32461968DAE7324621
:10A100000949D7E732460949D4E700BFC8920100A0
:10A110006C070020928E01009B860100CD92010009
:10A12000EC92010080030020E6920100E39201001E
:10A13000980400200B460A220146184606F0D9BBB7
:10A1400010B5054C0549204605F089FD2046BDE8BF
:10A15000104005F08BBD00BF68030020AE920100E7
:10A1600010B54AB102441BB1B2FBF3F403FB142255
:10A170008A4208D288420AD9012010BD884294BF81
:10A1800000200120F9E78242F8D80020F5E782425A
:10A19000F5E700002DE9F04F99B00DF108090C46E4
:10A1A00089E80C00DDE922AB0646002800F0D780E4
:10A1B000037C03F00F03062B1CD8DFE813F0CB0061
:10A1C0001B001B001B00C70007001D009E4BC5683D
:10A1D0001A7801321A701E464DB1CDE900AB2846FF
:10A1E00099E80C002146FFF7D5FF6D68F4E7337856
:10A1F000013B337000200EE00146944A944804F07D
:10A200001CFA054650B10023CDE90033214699E8F8
:10A210000C00FFF7BFFF19B0BDE8F08F8D4A8C48E6
:10A22000314604F00AFA8C4A80463146884804F0E8
:10A2300004FA07461CB1012C6DD02C460CE0874A6D
:10A240008348314604F0F9F90546854A804831468D
:10A2500004F0F3F9044605B93546002C08BF34462E
:10A26000B8F1000F79D0002F08BF5F4635B12B7CC5
:10A2700003F00F03042B0CBF6D690025002C71D077
:10A28000237C03F00F03042B6CD16469B8F1000F39
:10A2900000F09380002D71D07249734805F0D6FC10
:10A2A000D8F81410704805F0DAFC70496E4805F0D3
:10A2B000CDFC29466C4805F0D2FC6B4805F0D6FC75
:10A2C0004846FAF761FF002F7CD198F8103003F070
:10A2D0000F03042B40F0B280D8F8141008A8F8F748
:10A2E000D9FA08A8F8F714FA88B1FFF72BFEB0F5F1
:10A2F000966F044650DA5E495E4805F0A7FC0A22D4
:10A3000021465C4805F00BFD5A4805F0AFFC08A853
:10A31000F8F71EF892E0584A4D48314604F08DF99E
:10A32000564A054631464A4804F087F90446002D4E
:10A3300040F08680494A4648314604F07EF9054699
:10A34000002C82D0002808BF354689E70024274624
:10A35000A04681E7002425462746D04683E75F468E
:10A36000D04605460023102200930DEB02014FF466
:10A3700040734846FAF7F4FD044687E740493A48F7
:10A3800005F064FCD8F81410374805F068FC37492C
:10A39000354805F05BFC93E72DB10022294608A85B
:10A3A000F9F77AFDB3E70123009301952B4699E86D
:10A3B000060008A8F8F7CEFEA9E7002F3ED0002C33
:10A3C0003CD001E0002C80D03B7C03F00F03042B39
:10A3D00030D12C49244805F039FC7969224805F030
:10A3E0003EFC2249204805F031FC21461E4805F07C
:10A3F00036FC1D4805F03AFC4022796908A809F0AE
:10A4000068FD214804F06AFCA0B1204B93F90030AC
:10A4100083B92F2108A809F0F3FC28B97B6903222E
:10A42000402108A8FFF708FE0123224608A9164884
:10A4300004F0B1FEB8F1000F7FF447AF0120EAE667
:10A4400000287FF40DAF00E765030020C77A010004
:10A450006C070020BE7A0100007B010064920100BD
:10A460006992010078920100680300207F92010048
:10A4700095920100840300206E9201007392010006
:10A48000849201008E920100E0030020B0030020BE
:10A4900010B5044606F0D6F9E040431E033388BFEA
:10A4A000012010BD054B1A68054B53F820100123FD
:10A4B0008B40134214BF0120002070470805005054
:10A4C00020960100012070470020704738B51D49D3
:10A4D0001D4805F0DBFB01211C4800F072F91B4808
:10A4E00000F0FCF80121172006F09AFB002116204D
:10A4F00006F096FB142400252946172006F0B8FB29
:10A500000A2006F0D3F9013C85F00105F4D1104C86
:10A510000E4800F08DF8206880B100F049FA68B16B
:10A52000206800F081FB206800F04EFA206800F0FF
:10A53000BFFB28B10749044805F09EFB012038BD48
:10A540000549F8E7BE92010068030020900500204D
:10A5500018050020C9910100D591010007B500231D
:10A5600000931A461946034805F028FB03B05DF82E
:10A5700004FB00BF880500202DE9F84380460D4606
:10A58000174601EB02090C464C45A4EB05060BD01F
:10A59000D8F8003014F8011B1B6840469847002883
:10A5A000F2D13046BDE8F8833E46FAE770472030E6
:10A5B00005F0B5BC203005F0A4BC203005F0B5BCDA
:10A5C00038B5437F0D460BB9002038BD00F1680453
:10A5D000204605F0B2FC0028F6D12046294605F0B9
:10A5E00081FC0120F1E700002DE9F0411E46002525
:10A5F0004FF47A73C0E901530C4B044640F8203BFA
:10A600008846174605F065FC04F1680005F061FC1A
:10A610009DF8183063769DF81C302676C4E90487CF
:10A62000A37665772046BDE8F08100BFFC9201006B
:10A63000817E284A0123C37670B552F82140417EBD
:10A6400052F821104FF0A04504F5E07401F5E071D7
:10A6500040F20C6645F8246045F8216001694FF02E
:10A66000CC74C1F8244501690624C1F80045847EF4
:10A67000016952F82440C1F80845447E016952F846
:10A680002420C1F80C2590F91820510902F01F026E
:10A6900093406031104A42F8213090F91830002B75
:10A6A000BDBF03F00F0302F6FC32D2189B18B5BFF2
:10A6B00040234022137683F8002390F918300122BA
:10A6C000590903F01F0302FA03F3034A42F8213049
:10A6D00070BD00BF2096010000E100E0C37E23B101
:10A6E00003690022C3F8002570474269C2F80035AB
:10A6F00070472DE9F041044688461F461546002A5A
:10A7000050D000F12006304605F0F7FB2369C3F86E
:10A710008885236901221A622369C3F83465236995
:10A72000C3F8385523691A602269D2F84C311BB935
:10A73000D2F82431002BF8D00023C2F84C31226922
:10A74000D2F85C311BB9D2F82431002BF8D00023A9
:10A75000C2F85C3122696FB9D2F8243153B90123B0
:10A76000D3612369D3F84821002AFBD00022C3F823
:10A77000482109E0012353612369D3F80421002A09
:10A78000FBD00022C3F804212369D3F8242112B19D
:10A790000022C3F824212369D3F83C052066C0B207
:10A7A000BDE8F0811046FBE70123FFF7A2BF10B51B
:10A7B000044680F8B010683005F09FFB01236377F2
:10A7C00010BDF8B500234377036990F8B020C3F8B3
:10A7D0008825036901261E62036900F168050446A5
:10A7E000C3F8445528460F4605F099FB2369C3F882
:10A7F000480523699E602369D3F850211AB9D3F81C
:10A800002421002AF8D00022C3F85021284605F060
:10A8100086FB236930B1D3F860211AB9D3F824211B
:10A82000002AF8D00022C3F8602123696FB9D3F859
:10A83000242152B90122DA612369D3F84821002A80
:10A84000FBD00022C3F8482109E001225A612369A4
:10A85000D3F80421002AFBD00022C3F80421236985
:10A86000D3F8240168B10022C3F824212369D3F866
:10A87000C404C3F8C404022803D004280CBF032076
:10A880000420F8BD0121FFF79CBF70B54369D3F8E0
:10A890006421044692B10022012500F12006C3F88C
:10A8A00064210577304605F028FB6369C3F83465F9
:10A8B00063694022C3F8382563691D636369D3F86F
:10A8C0006821DAB10025C3F8685104F16806012354
:10A8D00063772577304605F010FBD4F8B43003B128
:10A8E0009847636965773046C3F8446505F017FB00
:10A8F0006369C3F84805636901225A636369D3F841
:10A90000042162B10022C3F80421237F3BB16369B3
:10A91000D3F83C05D4F8B830206603B19847636992
:10A92000D3F8242152B10022C3F824216369D3F85B
:10A93000D024C3F8D024636901225A6170BD00009D
:10A940000148FFF7A2BF00BF9005002007B51623FE
:10A950001722CDE900324FF040220423114603486C
:10A96000FFF742FE03B05DF804FB00BF9005002036
:10A970000148FFF787BF00BF9005002010B54FF4D6
:10A98000C053038000230446837003610248FFF72D
:10A990004FFE204610BD00BF9005002001617047AA
:10A9A0008078704741780148FFF701BF900500208B
:10A9B00008B5FFF7F7FF0348FFF764FFB0FA80F030
:10A9C000400908BD90050020012303707047FF2354
:10A9D000C37200230373C370037143718371C37126
:10A9E000037243728372704710B5064A0144002314
:10A9F000884204D010F8014B6340D35CF8E7184656
:10AA000010BD00BF14930100FFF7E1BF38B5084C3B
:10AA10000D46FFF7C7FFE1212046FFF7D1FD29468C
:10AA20002046FFF7CDFDBDE83840FFF7A1BF00BFCE
:10AA30009005002010B5054C417801222046FFF713
:10AA4000B3FE2046FFF7B6FDC0B210BD9005002052
:10AA500010B5F0210446FFF7D9FF2046BDE81040AD
:10AA6000FFF7E8BF70B5054605F0ECFE002400F5E1
:10AA70007A7605F0E7FEB04246D22B6903B19847DB
:10AA80002846FFF7E5FFC30704463FD514200138E9
:10AA900000BF00BF00BF00BF00BF00BF00BF00BFBE
:10AAA00000BF00BF00BF00BF00BF00BF00BF00BFAE
:10AAB00000BF00BF00BF00BF00BF00BF00BF00BF9E
:10AAC00000BF00BF00BF00BF00BF00BF00BF00BF8E
:10AAD00000BF00BF00BF00BF00BF00BF00BF00BF7E
:10AAE00000BF00BF00BF00BF00BF00BF00BF00BF6E
:10AAF00000BF00BF00BF00BF00BF00BF00BF00BF5E
:10AB000000BF00BFC3D1B4E70123AB70204670BDC6
:10AB100010B5E1210446FFF779FF2046BDE810405B
:10AB2000FFF788BF10B50446FFF79CFF2046FFF7EC
:10AB300039FF96210648FFF743FDFFF719FF20462E
:10AB4000FFF790FF2046BDE81040FFF7E1BF00BFD0
:10AB500090050020FFF7E6BF10B5C3210446FFF7BC
:10AB600055FF2046BDE81040FFF764BF38B50446E6
:10AB70000D46FFF777FF2046FFF714FFD2210A4862
:10AB8000FFF71EFDE94345EA0111C9B20648FFF788
:10AB900017FDFFF7EDFE2046FFF74CFFA8421CBF54
:10ABA0000423A37038BD00BF9005002010B50446F3
:10ABB000FFF7D2FF40F00401C9B22046BDE81040C3
:10ABC000FFF7D4BF70B5164604460D46FFF74AFF9F
:10ABD00016B12046FFF7EAFF2046FFF7E3FEA52166
:10ABE0000548FFF7EDFC29460348FFF7E9FCBDE8FF
:10ABF0007040FFF7BDBE00BF9005002070B5002279
:10AC00000C4655210646FFF7DDFF651E073415F893
:10AC1000011F00223046FFF7D5FFA542F7D170BDD6
:10AC2000FFF7ECBFFFF7CEBF10B50446FFF7BAFE43
:10AC300020460022F021FFF7C5FFBDE81040FFF7D6
:10AC400097BE000070B5164605460C46FFF70AFF92
:10AC500016B12846FFF7AAFF2846FFF7A3FE872173
:10AC60000648FFF7ADFC002C0CBF214680210348AD
:10AC7000FFF7A6FCBDE87040FFF77ABE9005002004
:10AC800010B5002204460121FFF7DCFF2046FFF744
:10AC9000E9FEC0F3401010BDFFF7F2BF10B5044647
:10ACA000FFF75AFF20460021BDE81040FFF75EBFC6
:10ACB00038B50446FFF7D6FEC30729D42046FFF770
:10ACC000EDFF2046FFF7CEFE2046FFF76BFEB421D6
:10ACD0001048FFF775FCFFF74BFE2046FFF7C2FE5A
:10ACE00010F00403054602D00223A37002E0A2780C
:10ACF000022AFAD0237843B12046FFF72DFF40F017
:10AD00000101C9B22046FFF731FFC5F3400038BD4D
:10AD10000020FCE7900500202DE9F74F057B044655
:10AD20000F46002D6BD1FFF7C3FF002869D02046E6
:10AD3000FFF798FE2A46F0212046FFF743FFDFF891
:10AD4000C8804FF0FF394FF0010A94F90B30EEB292
:10AD50004FEAD60B9D4206F007060AFA06F623DAFA
:10AD600004EB0B03DB78334020460193FFF77AFEB8
:10AD70002046FFF717FE78214046FFF721FC019B94
:10AD8000002B0CBF194680214046FFF719FCFFF746
:10AD9000EFFD2046FFF766FE820600F0400307D570
:10ADA0005BB16FF0010027E00CBF01230023DBE75C
:10ADB0001BB9030658BF4FFA85F904EB0B030106D4
:10ADC00093F9032076B205F101054CBF3243B2433B
:10ADD000402DDA70B9D1B9F1FF3F04BF01232373CD
:10ADE00084F80B90E31C013F0B3413F8012B07F898
:10ADF000012FA342F9D1012003B0BDE8F08F00205C
:10AE0000FAE74FF0FF30F7E79005002008B5FFF7AD
:10AE100083FF20EAE070C0B208BDFFF749BF70476A
:10AE2000054A8261002202710270092242700122E9
:10AE300081608270C27070471FAE000010B50C4672
:10AE400020460721FFF7D0FDE3791B1A58425841ED
:10AE500010BD70B5044680680E461546FFF7DDFF4D
:10AE6000B8B13146A068FFF7DBFE0022BE21A06822
:10AE7000FFF7D8FE6E1E0835A068FFF76BFE06F8D8
:10AE8000010FAE42F8D1A068FFF7C7FF431E58423A
:10AE9000584170BD10B51446FFF7DBFF38B10821EB
:10AEA0002046FFF7A1FD237A1B1A5842584110BDD6
:10AEB00070B504460D4680681646FFF7AEFF29467A
:10AEC000A068FFF7ADFE00224E21A068FFF7AAFEA2
:10AED0000022B178A068FFF7A5FE0022F178A068F3
:10AEE000FFF7A0FE2B78102B04D000223179A06848
:10AEF000FFF798FEA068FFF790FF2946A068FFF7CC
:10AF00008FFE2278A0684821FFF78CFE142005F000
:10AF1000CDFC237813B10A2005F0C8FCA068BDE879
:10AF20007040FFF77ABF38B504460D468068FFF7DA
:10AF300074FF2946A068FFF773FE0022B421A068C1
:10AF4000FFF770FEA068FFF7A7FE0546A068FFF7B1
:10AF500064FFB5FA85F0400938BDF0B585B01446F8
:10AF600001AA07460E46FFF795FF054690B13378D4
:10AF7000102B0FD00B2C10D00C2C03D00A2C0ED180
:10AF80003F2300E07F2301AA314638468DF8083080
:10AF9000FFF78EFF284605B0F0BD5F23F3E71F23C0
:10AFA000F1E71FB50B78102B10D001AAFFF772FF45
:10AFB00078B19DF808303F2B0ED003D81F2B0DD051
:10AFC000002006E05F2B03D07F2BF9D10C2000E09E
:10AFD0000B2005B05DF804FB0A20FAE70920F8E72A
:10AFE000F0B587B0044605F02DFC00F51C55A068AF
:10AFF000FFF70AFD002310352371012601A9A0687F
:10B00000FFF704FF40B305F01DFCA84224D201A9BC
:10B010002046FFF713FF0028F0D023782BB901A9B1
:10B020002046FFF780FF00B1267003AA01A9204641
:10B03000FFF70FFF01A920466778FFF7B2FF8742AD
:10B0400005D960782379607001332371D6E701A9AF
:10B050002046FFF7A6FFF5E707B0F0BD8170704707
:10B060001FB501AAFFF7F5FE9DF80400003018BFD8
:10B07000012005B05DF804FB0939C9B20229F8B511
:10B0800098BF104B0546164694BF33F9114040F265
:10B09000EE248AB1C3787BB103786BB905F0D2FB9B
:10B0A000074631462846FFF7DBFF20B905F0CAFB0B
:10B0B000001BB842F5D3F8BD2046BDE8F84005F0C6
:10B0C000F5BB00BF14940100F8B504460F46FFF726
:10B0D00068FF064610B900252846F8BDA068FFF7AE
:10B0E0009CFE0028F7D03946A068FFF799FD22782A
:10B0F000A0684421FFF796FDA5782DB13A46314668
:10B100002046FFF7B9FFE7E70125E5E71078537818
:10B11000C00040EAC3200B78102B00B20BD1D179CC
:10B120009379C000CB1ADB0120F07F0093FBF1F391
:10B13000103B184400B2704730B585B001AA0446F0
:10B140000D46FFF7A7FE30B101AA29462046FFF7BA
:10B15000DDFF05B030BD0148FBE700BF80E4FFFF25
:10B1600010F5DC5FCABF07EE900ADFED037AFAEE56
:10B17000EC7A17EE900A70470000FEC208B5FFF7A0
:10B18000DBFFBDE80840FFF7EBBF014604220120CA
:10B1900001F0AABA01460422052001F0A5BA014631
:10B1A0000622092001F0A0BA014604220F2001F076
:10B1B0009BBA00002DE9F04F3D4E3E4C336813F032
:10B1C000010387B082468B4615460ED1E3644FF4E7
:10B1D0007A732365384BA36404F15C0004F0E6FC49
:10B1E000082384F8683001233360344E346001F062
:10B1F0004DFC0027002859D04FF000494FF00208BD
:10B20000CDF80C9005978DF8108003AC94E80E00F3
:10B210002B4805F0B7FD5046FFF7C1FF3B463A46C5
:10B2200039460097204604F0C9FC04A8FFF7BCFF8C
:10B23000234805F0B3FD2B465A465146306801F0CD
:10B240008FFF012805462DD1CDF80C9005978DF87C
:10B25000108094E80E001A4805F094FD31682046ED
:10B2600001F0E5FC04A8FFF79FFF3168204601F0DC
:10B27000ECFC04A8FFF789FF3168204601F0DEFCF2
:10B2800004A8FFF787FF0E4805F088FD31682046C7
:10B2900001F0E2FC0B4B049A5A6005F0EDFA80B223
:10B2A00000F08EFD284607B0BDE8F08F0546F9E7AF
:10B2B0004C060020640600208094010060060020F7
:10B2C0004C08002058060020F0B585B007460E4611
:10B2D00014461D4601F0DAFB00B34FF00043019322
:10B2E0000023039302238DF8083004AB13E90E000A
:10B2F0000B4805F047FD3846FFF751FF301DFFF7BB
:10B3000053FF281DFFF741FF0A980430FFF742FF63
:10B31000034805F043FD034B62685A6005B0F0BD79
:10B320004C08002058060020F0B58DB01D460023C3
:10B330000F460093FF230446164619461A4602A8F4
:10B3400004F03CFC0B4B7A680493CDE9052372684A
:10B35000CDE907236A68CDE90923039B0B930AAB68
:10B36000009306AA08AB04A92046FFF7ADFF0DB075
:10B37000F0BD00BF9096010000B50B4B49685268C4
:10B3800089B0CDE90231CDE9052304930123019170
:10B390008DF80730019B079304AA06AB02A9FFF7BB
:10B3A000C3FF09B05DF804FB909601007FB5094B1F
:10B3B0004A680493CDE90232012301928DF80730E7
:10B3C000019B059304AA02A9FFF7D6FF07B05DF819
:10B3D00004FB00BF9096010008B501F0BDFB0128F9
:10B3E00003D002280CBF0220002008BD7FB51E4EEE
:10B3F0003068002836D001F0CBFE0228044601D088
:10B4000004282CD14FF0004301930023039302231F
:10B4100001AD8DF8083095E80E00144805F0B2FC37
:10B420003168284601F003FC02A8FFF7BDFE316831
:10B43000284601F00AFC02A8FFF7A7FE316828465B
:10B4400001F0FCFB02A8FFF7A5FE084805F0A6FCEA
:10B450003168284601F000FC054B029A5A602046EC
:10B4600004B070BD0446FAE7600600204C080020D6
:10B470005806002030B585B0044604F097FB4FF025
:10B4800000430193002303930A4D02238DF80830F3
:10B4900004AB13E90E00284605F074FC0422A11841
:10B4A0000F2001F0D9F9284605F078FC204605B0B8
:10B4B00030BD00BF4C08002030B585B0044604F014
:10B4C00075FB4FF000430193002303930A4D0223C1
:10B4D0008DF8083004AB13E90E00284605F052FC45
:10B4E0000422A118052001F0B7F9284605F056FC02
:10B4F000204605B030BD00BF4C08002030B585B0F7
:10B50000044604F053FB4FF00043019300230393E0
:10B510000A4D02238DF8083004AB13E90E002846CB
:10B5200005F030FC0422A118012001F095F928460D
:10B5300005F034FC204605B030BD00BF4C080020AB
:10B5400007B5002300931A461946044804F036FB59
:10B55000034803B05DF804EB04F028BB500600205C
:10B5600058060020007C07288CBF0020012070476F
:10B5700081F0010070470846704708B50368DB6B2F
:10B58000984780F00100C0B208BD4182704713B5F2
:10B5900002AB026803F8011D546819460122A04756
:10B5A00002B010BD037C087C984204D107288CBFF0
:10B5B00000200120704700207047000010B50446AD
:10B5C000007C072816D800F0A1FD182806D80A4BE1
:10B5D00023FA00F0C04300F0010010BD1C2807D181
:10B5E000236820469B689847003018BF0120F4E785
:10B5F0000120F2E70020F0E701001001F0B591B062
:10B60000044604A80F46164604F0D0FA00224FF470
:10B610007A73CDE908230CA8184B079304F0C6FAF7
:10B62000082368468DF83C3004F0C0FA207C0728D7
:10B6300007D800F06BFD10B1207C00F0CBFD082393
:10B6400023740F4B0F4D5B68039302A904A8029566
:10B6500001F0DDFD41F288336A46394604A801F065
:10B660005FFF40B12368019A9B69039202953246BD
:10B6700002A92046984711B0F0BD00BF8094010098
:10B68000580600209096010008B5007C072802D8D3
:10B6900000F02EFF08BD0020FCE710B50446207C1A
:10B6A00007280BD800F032FD172801D01C2805D13F
:10B6B000207C00F01DFFB0F5006FF0D310BD38B551
:10B6C0000546007C0728144605D892B200F092FE89
:10B6D00010B901236B600024204638BD08B5007CFA
:10B6E000072802D800F02EFE08BD0020FCE7007CF1
:10B6F000072802D812B200F08BBD0020704707B5B2
:10B7000001220DF10701007C00F082FD0028CCBF72
:10B710009DF807004FF0FF3003B05DF804FB10B553
:10B72000037C072B044602D94FF0FF3010BD03689D
:10B730009B6898470028F7D0207C00F02FFEF5E7A3
:10B7400038B50446007C07280AD800F043FD05F010
:10B7500079F80546207C00F0D9FC10B90823237441
:10B7600038BDFBF7CDFA012005F0A0F805F06AF826
:10B77000638A401B9842EDD3207C00F0E5FCEDE7A6
:10B780007FB50446007C07280D46164607D800F012
:10B79000BDFC10B1207C00F01DFD082323740021A6
:10B7A000684604F017FA6A68019B9A4202D10020A9
:10B7B00004B070BD4FF0FF3102A804F00BFA6A68C4
:10B7C000039B9A42F3D00021212000F003FB0728BD
:10B7D0002074ECD8291D324600F0D4FC05F032F874
:10B7E0000546207C00F092FC172815D01C2813D0A9
:10B7F0000028DCD005F026F8638A401B984205D863
:10B80000FBF77EFA012005F051F8EAE7207C00F012
:10B810009BFC08232374CAE70120C9E710B414462F
:10B82000064A127801EB022101EB00201A4621465C
:10B8300080B25DF8044B01F00FB800BF3007002064
:10B840007FB5037C072B05464FF000041BD84FF053
:10B85000004302260394019301AC8DF8086094E83C
:10B860000E000A4805F08EFA334622460421287C51
:10B87000FFF7D4FF9DF804309DF80540034844EAE3
:10B88000032405F08BFA204604B070BD4C0800205C
:10B890007FB50B7C072B05460E4605D9002104F029
:10B8A00099F9284604B070BD4FF00043019300237E
:10B8B0000393022301AC8DF8083094E80E00084889
:10B8C00005F060FA042322460C21307CFFF7A6FF26
:10B8D000034805F063FA2146284604F081F9E0E7C1
:10B8E0004C0800207FB5037C072B05464FF0000471
:10B8F0001BD84FF0004302260394019301AC8DF84E
:10B90000086094E80E000A4805F03CFA33462246E7
:10B910001021287CFFF782FF9DF804309DF8054038
:10B92000034844EA032405F039FA204604B070BD08
:10B930004C08002007B5002300931A461946034817
:10B9400004F03CF903B05DF804FB00BFD006002012
:10B9500003681B6B18470000024A02608A69426054
:10B96000704700BF90960100808B7047008A704737
:10B97000408C704713B502AB026803F8011D546890
:10B9800019460122A04702B010BD704710B5044609
:10B9900090F82000072804D800F0D6FB082384F88C
:10B9A000203010BD38B5044690F8200007280D4619
:10B9B00001D800F0C9FB2946022000F00BFA072845
:10B9C00084F820004FF000009EBF60842582012093
:10B9D00038BD0000F0B591B0044604A80F461646E5
:10B9E00004F0E4F800224FF47A73CDE908230CA8A0
:10B9F000134B079304F0DAF8082368468DF83C30BF
:10BA000004F0D4F80F4B104D5B68039302A904A80F
:10BA1000029501F0FCFB41F288336A46394604A8DE
:10BA200001F07EFD012808D12368019A1B6A039268
:10BA30000295324602A92046984711B0F0BD00BFDA
:10BA400080940100580600209096010008B500235C
:10BA5000C383043190F8200000F09CFD08BD08B5B8
:10BA600090F8200000F0C4FD08BD10B593B2044664
:10BA70000A46C18B90F8200000F060FDE38B034480
:10BA8000E38310BD13B5438C04461BB94FF0FF3060
:10BA900002B010BD01220DF1070190F8200000F066
:10BAA000B7FB0028F2DD638C9DF80700013B63843F
:10BAB000EEE710B5438C044613B94FF0FF3010BDCC
:10BAC000934294BF1AB212B290F8200000F0A0FB8B
:10BAD0000028F2DD638C1B1A6384F0E708B590F848
:10BAE0002030072B05D8428C1AB1184600F056FCBE
:10BAF00008BD4FF0FF30FBE773B5044690F8200017
:10BB000007280E46154601D800F01EFB094B00938E
:10BB10002A46736801936946822000F017FA0728C5
:10BB200084F820004FF000009EBF60840120258231
:10BB300002B070BD9096010013B50446628C2AB124
:10BB4000236800211B6B20469847F7E794F82000F4
:10BB500000F0F8FBD8B10822694694F8200000F004
:10BB600057FB002813DD694604F1140004F040F887
:10BB70009DF804209DF805309DF8070003EB022393
:10BB8000A3839DF8063000EB032080B2608402B0EE
:10BB900010BD000007B5002300931A46194603485C
:10BBA00004F00CF803B05DF804FB00BFD8060020D9
:10BBB00007B5084B1B7801EB032101EB00200122A4
:10BBC0000DF1070180B200F047FE9DF8070003B0B9
:10BBD0005DF804FB3007002007B5084B1B7801EB2C
:10BBE000032101EB002002A980B201F8012D0122FE
:10BBF00000F07AFDC0B203B05DF804FB300700200E
:10BC000010B41446064A127801EB022101EB002021
:10BC10001A46214680B25DF8044B00F065BD00BFB6
:10BC2000300700202DE9F7430C4617461E4601AAAF
:10BC3000022324210546FFF7F1FD9DF804209DF81D
:10BC4000053043EA0223224A1C441378332B0CBFED
:10BC500005F1080005F11000A4B2C002C4F30A09FE
:10BC600080B24844372B904680B22DD009EB0603B2
:10BC7000B3F5006F28DDC9F500691FFA89F94A4656
:10BC8000394600F031FD98F80030332B0CBF05F138
:10BC9000080005F11000C002A6EB090280B292B2C2
:10BCA00007EB09013444A4B200F01EFD23128DF805
:10BCB000043001AA0223242128468DF80540FFF70D
:10BCC0009FFF03B0BDE8F08332463946EAE700BF84
:10BCD0003107002008B50321FFF76AFF08BD07B54B
:10BCE0000B128DF804308DF80510022301AA0421EF
:10BCF000FFF786FF03B05DF804FB08B50A4604238E
:10BD00000C21FFF77DFF08BD07B50B128DF804303D
:10BD10008DF80510022301AA1021FFF771FF03B06F
:10BD20005DF804FB07B5022301AA2021FFF776FD89
:10BD30009DF804009DF8053043EA002003B05DF84B
:10BD400004FB000038B50546FFF7ECFF0446284623
:10BD5000FFF7E8FF8442034604D1034B03EBC5031E
:10BD60009C8038BD1C46F2E7E806002007B5022398
:10BD700001AA2621FFF752FD9DF804009DF8053029
:10BD800043EA002003B05DF804FB07B5022301AAD3
:10BD90002821FFF743FD9DF804009DF8053043EA94
:10BDA000002003B05DF804FB044B1B78332B0CBF61
:10BDB0000C301830C00280B2704700BF310700203D
:10BDC000034B1A88C0F30D0050401880704700BF25
:10BDD000080000202DE9F043574B1B7885B08146C1
:10BDE0000F468BB3332B4FF0004301934FF0000508
:10BDF0004FF0020303958DF8083001AE96E80E006F
:10BE00004E4814BF4FF008084FF0040804F0BAFF82
:10BE1000ECB22046FFF75EFF7055D8B10135EBB2AA
:10BE20009845F5D800234FF03451F25C1D2ADCB25E
:10BE300003D821FA02F2D20708D40133DAB242451C
:10BE4000F3D33E4804F0AAFF082465E01021204601
:10BE500000F0C6FE3A4B002123F81410FA200138F6
:10BE600000BF00BF00BF00BF00BF00BF00BF00BFDA
:10BE700000BF00BF00BF00BF00BF00BF00BF00BFCA
:10BE800000BF00BF00BF00BF00BF00BF00BF00BFBA
:10BE900000BF00BF00BF00BF00BF00BF00BF00BFAA
:10BEA00000BF00BF00BF00BF00BF00BF00BF00BF9A
:10BEB00000BF00BF00BF00BF00BF00BF00BF00BF8A
:10BEC00000BF00BF00BF00BF00BF00BF00BF00BF7A
:10BED00000BF00BFC3D14A462046FFF77DFEFF22C8
:10BEE00002212046FFF778FED7B139462046154D8E
:10BEF000FFF7F5FE00260121204600F071FE25F82F
:10BF000034602046FFF741FF05EBC40358809E7163
:10BF10009E800A4804F042FF204605B0BDE8F08349
:10BF2000094B1A88013292B2B2F5404F38BF4FF434
:10BF300040421A801988D9E7310700204C080020B8
:10BF40004C070020E8060020080000202DE9F047FB
:10BF5000694B1B7886B082460E461746A3B3332B37
:10BF60004FF0004303934FF000054FF00203059597
:10BF70008DF810300DF10C0898E80E005F4814BFE2
:10BF80004FF008094FF0040904F0FCFEECB2204623
:10BF9000FFF7A0FE08F80500E0B10135EBB29945C6
:10BFA000F4D800234FF0345118F803201D2ADCB2D6
:10BFB00003D821FA02F2D20708D40133DAB24A4593
:10BFC000F2D34E4804F0EAFE082485E01021204612
:10BFD00000F006FE4A4B002123F81410FA20013825
:10BFE00000BF00BF00BF00BF00BF00BF00BF00BF59
:10BFF00000BF00BF00BF00BF00BF00BF00BF00BF49
:10C0000000BF00BF00BF00BF00BF00BF00BF00BF38
:10C0100000BF00BF00BF00BF00BF00BF00BF00BF28
:10C0200000BF00BF00BF00BF00BF00BF00BF00BF18
:10C0300000BF00BF00BF00BF00BF00BF00BF00BF08
:10C0400000BF00BF00BF00BF00BF00BF00BF00BFF8
:10C0500000BF00BFC3D152462046FFF7BDFDFF22FF
:10C0600002212046FFF7B8FD002F39D0394620467F
:10C07000FFF735FE5E238DF80630737903F07F03FA
:10C080008DF80730B3798DF808300125F3798DF8F4
:10C090000930311D2046ADF80450FFF72EFE394619
:10C0A0002046FFF731FE0623194601AA2046FFF776
:10C0B000A7FD2946134D0026204600F091FD25F8E6
:10C0C00034602046FFF761FE05EBC40358809E7183
:10C0D0009E800A4804F062FE204606B0BDE8F08764
:10C0E000094B1A88013292B2B2F5404F38BF4FF473
:10C0F00040421A801988BAE7310700204C08002016
:10C100004C070020E80600200800002030B585B06C
:10C110004FF000430193002303930A4C02238DF850
:10C12000083004AB13E90E000546204604F02AFE51
:10C130002846FFF7CFFD0546204604F02FFE28468F
:10C1400005B030BD4C08002030B585B04FF000433D
:10C150000193002303930A4C02238DF8083004ABAB
:10C1600013E90E000546204604F00CFE2846102177
:10C1700000F036FD204605B0BDE8304004F00EBEAC
:10C180004C080020F0B585B04FF000430193002328
:10C1900003930F4D02238DF8083004AB04460F467D
:10C1A0001646284613E90E0004F0ECFD39462046F9
:10C1B000FFF7A3FD31462046FFF7A6FD20460421E8
:10C1C00000F00EFD284605B0BDE8F04004F0E6BDE5
:10C1D0004C08002030B585B04FF000430193002398
:10C1E00003930A4C02238DF8083004AB13E90E00C8
:10C1F0000546204604F0C6FD2846082100F0F0FC64
:10C20000204605B0BDE8304004F0C8BD4C08002011
:10C210002DE9F04F85B04FF000430193464E0023C7
:10C220000393022336F830408DF8083001AB1746EF
:10C230000546894641480ECB04F0A4FDA7420EDD19
:10C240002846FFF793FD04462846FFF78FFDA042DE
:10C25000F9D106EBC5039B79E41A26F835408CB971
:10C260002846FFF737FD142805D020B1B0F11C0493
:10C2700018BF4FF0FF34314804F090FD204605B060
:10C28000BDE8F08F4FEAC50BBC4206EB0B03A8BF1D
:10C290003C46B3F80280A7B2B9F1000F21D028467E
:10C2A000FFF782FD264A1278C8F30A0A5044372A5B
:10C2B00080B23DD01AFA84F2B2F5006F38DDCAF5CB
:10C2C00000631FFA83FA5246494600F0C5FA284631
:10C2D000FFF76AFDA7EB0A02D14492B2494600F08B
:10C2E000BBFA06EB0B0236F835309179B844DB1B0C
:10C2F0000F44BFB21FFA88F89BB2F92FA2F8028050
:10C3000026F8353000D8ABB95E440023B3714FEA4C
:10C3100028238DF8043001AA0223282128468DF80D
:10C320000580FFF76DFC4021284600F059FCA2E78C
:10C330003A46D3E797719EE7E80600204C080020B4
:10C34000310700207FB5134D064635F83000F8B9A7
:10C350004FF000430193022303908DF8083004ABA3
:10C360000D4813E90E0004F00DFD3046FFF7FEFC0A
:10C3700004463046FFF7FAFCA042F9D1064804F023
:10C380000DFD05EBC6039879201A80B225F836001A
:10C3900004B070BDE80600204C0800207FB54FF0C7
:10C3A0000043019300230393104D02238DF80830BE
:10C3B00001AC94E80E000646284604F0E3FC304643
:10C3C000FFF7F2FC0A4B03EBC60301225B88C3F3C1
:10C3D0000A031844214680B200F03EFA284604F0D1
:10C3E000DDFC9DF8040004B070BD00BF4C080020C7
:10C3F000E80600202DE9F04FB2F5006F87B028BFA6
:10C400004FF40062DFF8E49005468A46164603AC16
:10C4100002234FF000474FF000080397CDF8148037
:10C420008DF8103094E80E00484604F0ABFC284626
:10C43000FFF788FC83462846FFF74CFC01904846EE
:10C4400004F0ACFC019B172B01D01C2B32D104F063
:10C450004FFAB345DCD303974FF000080227CDF81D
:10C4600014808DF8107094E80E00204804F08AFCC7
:10C470004146334652462846FFF7D4FB2021284642
:10C4800000F0AEFBDFF864804FF0004B022128463D
:10C49000FFF78EFB10F0100A1FD12846FFF71AFC99
:10C4A000814648B9114804F079FC4E46304607B041
:10C4B000BDE8F08F4646CEE7404604F06FFC04F03E
:10C4C00017FACDF80CB0CDF814A08DF8107094E8E0
:10C4D0000E00404604F056FCD8E710220221284600
:10C4E000FFF77AFB014804F059FCDFE74C08002015
:10C4F00030B585B04FF0004301930023039302232E
:10C500008DF8083004AB054613E90E000A4804F024
:10C5100039FC2846FFF716FC04462846FFF7DAFBED
:10C520000546054804F03AFC172D02D01C2D18BF13
:10C530000024204605B030BD4C0800202DE9FF4105
:10C540001C464FF00043019300230393104D022338
:10C550008DF8083004AB06460F469046284613E98E
:10C560000E0004F00FFC3046FFF7ECFB844228BFBE
:10C570000446A4B22346424639463046FFF752FBF2
:10C58000284604F00BFC204604B0BDE8F08100BF53
:10C590004C0800207FB50B7806460D4614462BB993
:10C5A0004B781BB98B780BB9C878D0B1DCB14FF0A0
:10C5B000004301930023039302238DF8083004AB5A
:10C5C00013E90E00094804F0DDFB29463046FFF769
:10C5D00094FB21463046FFF797FB044804F0DEFB4E
:10C5E000012004B070BD2046FBE700BF4C080020CE
:10C5F0002DE9FF4700234FF000480227CDF80480C3
:10C6000003938DF8087001AC94E80E0005461F48AE
:10C61000DFF8789004F0B6FB2021284600F0E0FA1D
:10C6200002212846FFF7C4FA10F0100623D1022198
:10C630002846FFF7BDFA10F0080A0BD01822022195
:10C640002846FFF7C9FA114804F0A8FB304604B0A9
:10C65000BDE8F087484604F0A1FB04F049F9CDF8A5
:10C660000480CDF80CA08DF8087094E80E004846C0
:10C6700004F088FBD4E7102202212846FFF7ACFA29
:10C68000024804F08BFB0120E1E700BF4C080020CA
:10C6900007B5002300931A461946034803F08EFAA3
:10C6A00003B05DF804FB00BFE006002070B505464E
:10C6B0000C468E18B44206D02178284604F06FFB51
:10C6C00004F8010BF6E770BD024B0021187804F066
:10C6D000CFBA00BF0A000020024B0121187804F0F5
:10C6E000C7BA00BF0A0000202DE9F3414F4B1B7869
:10C6F000332B04460D4616461FD100EB02084C4F63
:10C700004D1E1FFA88F8A0457AD0FFF7DDFFF02113
:10C71000384604F044FB210A384604F040FBE1B2FD
:10C72000384604F03CFB013415F8011F3846A4B22A
:10C7300004F035FBFFF7D0FFE5E7342BC7B21DD17E
:10C74000FFF7C2FF330A241263F07F030422694615
:10C7500037488DF800408DF801708DF802308DF863
:10C760000360FFF7A3FF013D314CAF19AF4245D045
:10C7700015F8011F204604F012FBF7E7FFF7A4FFAE
:10C78000FF2C08D800238DF800308DF801700423A9
:10C790008DF802300DE0230419D4E41024F01F04B6
:10C7A000002344F00C048DF800308DF801708DF8F2
:10C7B0000240052E28D82A46531BDBB2B34218DAB2
:10C7C00002A8034412F8011B03F8051CF4E744F324
:10C7D000871323F01F03B4F5404F4FEA14228DF85E
:10C7E00000208DF8017034BF43F0140343F01C03A4
:10C7F000CEE7F21C69460E48FFF758FFFFF76CFFC3
:10C80000304602B0BDE8F081032269460848084F6F
:10C81000FFF74CFF731E6C1E15FA83F514F8011F09
:10C82000384604F0BCFAA542F8D1E7E7310700200A
:10C830004C08002007B502AB012203F8011D194680
:10C84000FFF752FFC0B203B05DF804FB08B5014624
:10C850000020FFF7EFFF08BD2DE9F3413E4B1B78A9
:10C86000332B04460E46154620D100EB02083B4F01
:10C870004E1E1FFA88F8A0453AD0FFF725FF0F217A
:10C88000384604F08CFA210A384604F088FAE1B2FE
:10C89000384604F084FA0021384604F080FA013466
:10C8A00006F8010FA4B2FFF717FFE4E7342BC7B275
:10C8B00022D1FFF709FF2412C5F3062304228DF8C5
:10C8C00004408DF805708DF806308DF807500DEB9B
:10C8D00002012248FFF7EAFE2A460021304606F010
:10C8E00024FB2A4631461D48FFF7E0FEFFF7F4FE21
:10C8F000284602B0BDE8F081FFF7E6FEFF2C07D81E
:10C9000000238DF804308DF805708DF806300DE0A9
:10C9100023040ED4E41024F01F04002344F0080480
:10C920008DF804308DF805708DF80640032201A9BA
:10C93000CFE744F3871323F01F03B4F5404F4FEACA
:10C9400014228DF804208DF8057034BF43F01003D5
:10C9500043F01803D9E700BF310700204C0800203E
:10C9600007B501220DF10701FFF776FF9DF80700DB
:10C9700003B05DF804FB08B50020FFF7F1FF08BD28
:10C9800010B58020FFF762FF1424FFF7F4FF40B1D9
:10C99000013C0120A4B203F089FF002CF5D1204610
:10C9A00010BD0120FCE7000008B50F4B33221A70C0
:10C9B000FFF7E6FF08B9002008BD1020FFF746FF8B
:10C9C000FFF7D9FF1028F6D11220FFF73FFFFFF73E
:10C9D000D2FF1228EFD10020FFF738FFFFF7CBFF7F
:10C9E000B0FA80F04009E7E73107002008B5124BA4
:10C9F00034221A70FFF7C4FF08B9002008BD0820D0
:10CA0000FFF724FFFFF7B7FF0828F6D11020FFF744
:10CA10001DFFFFF7B0FF1028EFD10020FFF716FF32
:10CA2000FFF7A9FF0028E8D11F20FFF799FFC31ED9
:10CA300058425841E2E700BF3107002008B5124BC9
:10CA400037221A70FFF79CFF08B9002008BD0820A4
:10CA5000FFF7FCFEFFF78FFF0828F6D11020FFF745
:10CA6000F5FEFFF788FF1028EFD10020FFF7EEFE5C
:10CA7000FFF781FF0028E8D13920FFF771FF031F7E
:10CA800058425841E2E700BF310700207FB52D4EE4
:10CA90003478002C53D14FF40C7003F007FF2A4870
:10CAA00004F05AF9294B0121187804F0B9F8FFF77E
:10CAB00013FE4FF00043019302238DF808300394D6
:10CAC00004AB13E90E00204804F05CF9FFF78EFF79
:10CAD000B0B11F4B40221A70E5B202221E21284637
:10CAE000FFF77AF8013402221F212846FFF774F875
:10CAF000082CF1D11448012404F050F934701BE0E3
:10CB0000FFF79CFF18B1124B10221A70F2E7FFF7E3
:10CB10004BFF044658B10E4B042255211B201A70BE
:10CB2000FFF788FE55211A20FFF784FEE2E7094B44
:10CB30001870054804F032F9204604B070BD012495
:10CB4000FAE700BF320700204C0800200A0000204E
:10CB500030070020310700201FB5FFF797FF38B1DD
:10CB60001D4B1B78342B4FF0000003D0372B1BD00C
:10CB700004B010BD4FF000430193022303908DF8E1
:10CB8000083004AB13E90E00144804F0FBF835201C
:10CB9000FFF7E6FE0446114804F000F914F0200FF8
:10CBA00014BF01200220E3E74FF00043019302236A
:10CBB00003908DF8083004AB13E90E00074804F029
:10CBC000E1F82E20FFF7CCFE0446044804F0E6F816
:10CBD00014F0010FE4E700BF310700204C080020EB
:10CBE00038B50A4601210446FEF7F6FF054D24023A
:10CBF000287804EB0020013080B2FFF7B1FE002856
:10CC0000F6D138BD3007002007B5002300931A463F
:10CC10001946034802F0D2FF03B05DF804FB00BFE1
:10CC20002807002014220021103006F07EB910B52C
:10CC30001031044602F0D4FF204610BD10B5143167
:10CC4000044602F0CDFF204610BD10B51831044651
:10CC500002F0C6FF204610BD10B52031044602F098
:10CC6000BFFF204610BD30204B1C0870110902F098
:10CC70000F02092A94BF3032373203F801290A46DD
:10CC80000029F3D17047000007B5002300931A462E
:10CC90001946034802F092FF03B05DF804FB00BFA1
:10CCA000340700202DE9F0418EB004468846164630
:10CCB0000021202206A806F038F9FF231A4619465B
:10CCC000009302A802F07AFF04F14805554B049343
:10CCD0004322039B059304A92846FEF7B7FE0130C3
:10CCE00000F09D80504B069363688DF821601BBA5D
:10CCF0000793330A8DF820301C22802306A926468C
:10CD00002846ADF82230FEF7B0FE1A2200210DF1C0
:10CD10001E0006F00AF956F8080F0690B388ADF821
:10CD20001C30102206A92846FEF79FFE2022002173
:10CD300006A806F0FAF80627202206A92846FEF7DC
:10CD400094FE013FF8D1394B069340F23513ADF80C
:10CD50001C303D238DF81F3007238DF82030012330
:10CD60008DF821303368CDF82230B388ADF8263005
:10CD70002F498DF81E8040F60C430DF12A00ADF8C6
:10CD8000283007F054F8E27A0CA92046FFF76BFF31
:10CD9000227B0DF132012046FFF765FF627B0DA972
:10CDA0002046FFF760FF1E2206A92846FEF75DFE1B
:10CDB000B8F1030F24D140F23243ADF81830237C90
:10CDC0008DF81A30637C8DF81B30A37C8DF81C30F5
:10CDD000E37C8DF81D3040F23643ADF81E30237FE2
:10CDE0008DF82030637F8DF82130A37F8DF82230BD
:10CDF0000C22E37F8DF8233006A92846FEF735FE86
:10CE00000C4A0D4B06A9CDE906232846FF2309222B
:10CE10008DF82030FEF729FE2846FEF720FE0EB0E2
:10CE2000BDE8F08190960100010106006382536322
:10CE3000C894010037060103060F3A3B2DE9F04381
:10CE400091B005468846164603F0FCFC05F14804FF
:10CE500007462046FEF770FE00280BDC03F0F2FCCC
:10CE6000C01B404500F2D280F9F74AFF012003F0D1
:10CE70001DFDEEE7242207A92046FEF71AFE9DF8C5
:10CE80001C30022B40F0BD80B5F86430432B40F0DD
:10CE9000B880089F3FBA3760062205F108010EA846
:10CEA00006F010F8064628B92B689F4202D36B683B
:10CEB0009F4207D92046FEF768FD0026304611B094
:10CEC000BDE8F0830B9B2B610146CC222046FEF788
:10CED000F0FD05F124072046FEF74AFD002840F347
:10CEE00091802046FEF7CEFD33287DD015DC012849
:10CEF00044D006DC0028EED02046FEF7C3FDC2B2C7
:10CF000053E0032844D00628F6D12046FEF7BAFDA8
:10CF10000422804605F1200141E03A284AD020DC75
:10CF2000352823D03628E7D12046FEF7ABFD05F1A2
:10CF30001C084146814601A802F052FE002103A8C8
:10CF400002F048FE029A049B9A4230D0414605A85E
:10CF500002F046FE2A6E069B9A4228D05FFA89F2BA
:10CF600023E03B2833D0FF28B5D0C5E72046FEF7A5
:10CF700089FD2046FEF786FDC6B2ACE72046FEF7E7
:10CF800081FD042205F114012046FEF792FDA2E77F
:10CF90002046FEF777FD0422804605F11801204661
:10CFA000FEF787FD5FFA88F2043A0021ECE70422DD
:10CFB0004146E9E72046FEF765FD042205F1280118
:10CFC0002046FEF776FDAB6A1BBAAB6283E72046CC
:10CFD000FEF758FD042205F12C012046FEF769FDFD
:10CFE000EB6A1BBAEB6276E72046FEF74BFD0422A4
:10CFF00039462046FEF75DFD6B6A1BBA6B622B63F8
:10D0000069E700262046FEF7C0FC57E7FF2655E7F4
:10D010002DE9F34704464FF4FA61012003F093FA37
:10D020002746606047F8480B3846FEF7AFFC4421BE
:10D030003846FEF7B7FC002800F0908003F002FCB1
:10D040004FF00009804600254FF0030A94F8443061
:10D05000032B1CD043BB63680133636003F0F2FB16
:10D060004FF47A72A0EB08000121B0FBF2F22046E7
:10D0700092B2FFF717FE012384F84430002DE5D16A
:10D0800003F0E0FBA36BA0EB08009842DBD9384625
:10D09000FEF77CFC63680133636003F0D3FB20641C
:10D0A000284602B0BDE8F087042B11D16368013334
:10D0B000636003F0C7FB4FF47A72A0EB0800032112
:10D0C000B0FBF2F2204692B2FFF7ECFD0223D3E769
:10D0D000012B19D101AAE16B2046FFF7AFFE022810
:10D0E000064638D1019B636003F0ACFB4FF47A72C3
:10D0F000A0EB08000321B0FBF2F2204692B2FFF74A
:10D10000D1FD84F84460B9E7022BB7D101AAE16BE5
:10D110002046FFF793FE0528064617D1636A84F878
:10D1200044A013B94FF461736362A36A13B9636ACD
:10D130005B08A362E36A1BB9636AA3EBD303E362F0
:10D14000A36A2363E36A636301257FE7062802D1AC
:10D1500084F8449092E7FF2EFAD08FE705469FE7C8
:10D16000F8B500250F460446C0E90955C562C0E977
:10D170000E2385608581FFF755FD3B68A360BB8862
:10D18000A38184F844502046BDE8F840FFF740BF33
:10D1900010B5044603F056FB236CC31AB3F57A7F2F
:10D1A00014D34FF47A71B3FBF1F201FB1233C01ABE
:10D1B000236B206451008B4234BF00239B1A2363EE
:10D1C000636B99428CBF00239B1A6363206BE0B9A9
:10D1D00094F84430032B06D1042384F844302046CD
:10D1E000FFF716FF0130636B73B994F84430032BDB
:10D1F00000D04BB9002384F844302046FFF712FDDD
:10D200002046FFF705FF033010BD0020EBE74B6819
:10D21000436000230381704770B500240139234621
:10D2200011F8010FB8B1A0F13005EEB2092E08D8FF
:10D2300003EB830305EB43039BB2FF2BF0D90020E4
:10D240000DE02E28FBD1032CF9D0601C144423716F
:10D25000C4B20023E4E7032C01D1D371012070BDD7
:10D2600007B5002300931A461946034802F0A6FCAE
:10D2700003B05DF804FB00BF3C0700202DE9F74335
:10D2800005460E4603F0DEFA05F10C04288105F18F
:10D290000801022202AD2046FEF7E7FB012325F834
:10D2A000023D022229462046FEF7DFFB4FF4807341
:10D2B000022229462046ADF80630FEF7D6FB0023B1
:10D2C000022229462046ADF80630FEF7CEFB0222A8
:10D2D00029462046FEF7C9FB022229462046FEF7D2
:10D2E000C4FB37463378E3B13E46B04618F8013BFD
:10D2F0000BB12E2B13D1A6EB0709B9F1000F0CDDF2
:10D3000001220DF1050120468DF80590FEF7ADFBD9
:10D310004A4639462046FEF7A8FB4746E2E746461E
:10D32000E3E702A9012201F8033D2046FEF79DFB39
:10D330004FF48076294602222046ADF80660FEF7BB
:10D3400094FB022229462046ADF80660FEF78DFBCD
:10D35000012003B0BDE8F0832DE9F04387B0064615
:10D360000F46904603F06EFA06F10C04054620467F
:10D37000FEF7E2FB002808DC03F064FA401BB84229
:10D3800000F2C480F9F7BCFCF1E7726A73689A4254
:10D3900040F0BF80338D352B40F0BB802046FEF738
:10D3A000E7FA0B2840F3B8800C220DEB020120466F
:10D3B000FEF77FFBBDF80E203189130A43EA0223F2
:10D3C000BDF80C201BB29DB29142ADF8065001D1C0
:10D3D000002B07DB2046FEF7D8FA4FF6FC7007B0AB
:10D3E000BDE8F08340F20F231D4005D02046FEF734
:10D3F000CCFA4FF6FB70F2E7BDF812301F0A47EA8D
:10D400000327BFB22FB92046FEF7BFFA4FF6FA70D6
:10D41000E5E7BDF810305BBAAAB29BB29A4216DAC1
:10D4200001220DF10A012046FEF743FB9DF80A2078
:10D430001AB100212046FEF73CFB9DF80A10002996
:10D44000EED104222046FEF734FB0135E1E7002649
:10D45000B14601220DF105012046FEF72AFB9DF899
:10D46000052012F0C00134D112B12046FEF721FB95
:10D470009DF80550002DECD1022202A92046FEF7AE
:10D4800018FB02220DF10A012046FEF712FB0422CE
:10D4900029462046FEF70DFB02220DF1060120462B
:10D4A000FEF707FBBDF80830BDF80620B3F5807F16
:10D4B00052BA92B21CD1BDF80A0040BA85B2012D11
:10D4C00016D1042A0DD02046FEF75FFA4FF6F7700A
:10D4D00085E7012200212046FEF7EBFA8DF8059042
:10D4E000C6E708F104012046FEF7E3FA284676E78E
:10D4F000013600212046B6B2FEF7DBFAB742A8D1CA
:10D500002046FEF742FA4FF6F67068E74FF6FF70D6
:10D5100065E74FF6FE7062E74FF6FD705FE70000CB
:10D520002DE9F34705468A4691469846FFF774FE73
:10D530000446B8BB1E4B6A685B689A4234D003F05D
:10D5400081F905F10C0600F00F0101F5806130460C
:10D55000FEF728FA0128074620D1164B0093352202
:10D560006B68019369463046FEF770FA98B15146F0
:10D570002846FFF783FE70B13046FEF770FA50B1CF
:10D580004A4641462846FFF7E7FE0446F9F7B8FB4E
:10D59000384603F08BF93046FEF7F8F9204602B022
:10D5A000BDE8F0870124F9E76FF00104F6E700BF5A
:10D5B0003C0700209096010007B5002300931A460F
:10D5C0001946034802F0FAFA03B05DF804FB00BF05
:10D5D00044070020006903681B6918470069036855
:10D5E0005B69184713B5006949680368034C0191EA
:10D5F0009B6900946946984702B010BD909601005F
:10D6000000690368DB691847006903689B6A18476B
:10D610000069003018BF01207047006C704701643A
:10D62000704710B590F83830044633B92069036864
:10D63000DB689847002808DA10BD03689B689847A4
:10D640000028F3D14FF0FF30F6E794F82220A2F142
:10D650000803022BF0D8A36A002BC2BFE36A013390
:10D66000E3620A2AE8D1E36B013BE363002BE3D1D9
:10D67000092384F82230DFE710B504460069036807
:10D680001B6A984794F82230083B022B07D8A36AFC
:10D69000002B04DD0028A2BFE36A1B18E36210BD63
:10D6A00073B590F82230092B04460ED1002620696C
:10D6B00003689B68984740B120690368DB68984716
:10D6C000C5B20A2D1CD184F8225094F822300A2BBE
:10D6D00004D1E36B13B9092384F8223094F8223083
:10D6E000092B22D0206903689B68984794F8223060
:10D6F0000A2B03D1E36B9842A8BF184602B070BD55
:10D700000D2DD4D0284605F086FB0028CFD0E06B45
:10D71000ADF8046010228DF804500021050101A825
:10D7200007F014FB2844E063C1E70020E6E70000AF
:10D7300000234FF0FF32C0E90A23084A80F8223064
:10D7400012680263064A4362126880F83830C36385
:10D7500047F2305342630364704700BF100000205B
:10D760001400002038B504461D4600204FF47A739B
:10D77000C4E901030B4B2360C4E9041204F118004F
:10D7800002F014FA0123258484F8443084F84530EB
:10D79000054904F1480002F02FFF2046FFF7C8FFBB
:10D7A00038BD00BF30950100E695010010B5044674
:10D7B000006903685B6A98472046BDE81040FFF7A0
:10D7C000B7BF012380F822307047000038B5044607
:10D7D0000069154602F043FA0449206902F03FFA55
:10D7E00029462069BDE8384002F050BAE9790100C5
:10D7F00038B504460D460069114602F030FA1D495D
:10D80000206902F02CFA2946206902F028FA1A4908
:10D81000206902F03BFA94F84530F3B16369B3B183
:10D820001649206902F01BFAD4E9040102F017FA44
:10D83000238C502B08D01249206902F010FA0A22DA
:10D84000218C206902F06BFA206902F00FFA0D4B6F
:10D850000D491A682046FFF7B9FF94F8443023B108
:10D860000A4A0B492046FFF7B1FF012384F8223012
:10D87000002038BD147B0100F5940100FF940100E5
:10D88000CC7B01000C0000200695010011950100E1
:10D890001795010038B504460069154602F0DFF916
:10D8A0000549206902F0DBF9294620690A22BDE812
:10D8B000384002F036BA00BFE979010010B50446DD
:10D8C000006902F0D3F9022384F8223010BD70B54C
:10D8D00090F82230012B04460D46164601D8FFF77A
:10D8E000EDFF20690368324629465B68BDE8704059
:10D8F000184770B590F82230012B04460D4601D828
:10D90000FFF7DCFF2069036829461B68BDE870400B
:10D91000184710B50446206903689B68984720B1F2
:10D9200020690368DB689847F5E710BD2DE9F347E8
:10D93000994690F82230083B022B04460E46924648
:10D94000DDE90A7804D8FFF7E4FF2046FFF7F0FE90
:10D9500094F82250012D45D894F844305BB1D4E9B5
:10D960000401228C0368B9B921490091E169019150
:10D970009B69694611E0206903689B6A9847002803
:10D98000EDD0314652462046FFF732FF064650B1F1
:10D99000304602B0BDE8F087DB6998470028F0DC2C
:10D9A0004FF0FF36F4E7B9F1000F04D04A461149B1
:10D9B0002046FFF70BFF002F17DD3A460E492046A1
:10D9C000FFF768FFB8F1000F0FD001252046FFF7E1
:10D9D00075FF002DDCD023683A465B68414620463F
:10D9E0009847D5E76FF00106D2E7002DD0D1EDE7DB
:10D9F00090960100CF940100DC94010090F8223051
:10DA0000012B01D8FFF75ABF7047FFF7F7BF00009F
:10DA100007B500234FF0FF32CDE90023024AFFF79C
:10DA200085FF03B05DF804FB229501002DE9F04766
:10DA300090F82230012B044651D9DFF8D880002518
:10DA4000032700236362022384F8223002F0FAFEE7
:10DA5000464682464FF00A090A2D46D002F0F2FEF1
:10DA6000236CA0EB0A00984245D2236820469B68AD
:10DA7000984748B323682046DB689847431C05460F
:10DA8000ECD094F82230022B05D0032B0FD002F0FB
:10DA9000D9FE8246E0E733782A2B01D083421AD19F
:10DAA0007278731C0AB984F822701E46EFE7A0F161
:10DAB0003002092A95BF636A042309FB032384F813
:10DAC000223098BF6362E2E74FF47A7002F0EEFE14
:10DAD000C2E70A2D06D16FF00300BDE8F0876FF0B2
:10DAE0000100FAE76FF00200F7E7636AC72B02DC78
:10DAF000652B18BF002594F82230042BE9D1606A09
:10DB0000C72801DC65289CD10A2D18BF6FF00200E0
:10DB1000E3E700BFEB94010038B501F14805044686
:10DB20003A21284602F048FE421C034605D1064928
:10DB3000204602F061FD204638BD002229462046DD
:10DB400002F058FEF7E700BFE6950100F8B501F1D5
:10DB5000480605460F4630463A2102F02DFE441C89
:10DB6000013005D10C49284602F046FD2846F8BD93
:10DB70003B6DA34209DD2146304602F001FE0078EC
:10DB800005F040F908B10134F2E73B6D2246314619
:10DB9000284602F02FFEE9E7E695010010B503687C
:10DBA0000446DB68984794F82230A3F10802022A61
:10DBB000C0B232D9052B31D0072B39D0042B54D128
:10DBC000226B137883420BD1531C2363537823B900
:10DBD000C4E90A33052284F822200A281DD136E040
:10DBE000636B197881420BD15A1C62635B78002BFE
:10DBF000F3D1012384F83830062384F82230ECE78F
:10DC00001B4909688A42F7D11A4A12689342F3D134
:10DC10000D28F1D1072384F8223010BDA0F1300285
:10DC2000092AE9D8A36A0A2101FB0323A362D4E7E6
:10DC30000A28F2D194F838309BB1092384F82230B5
:10DC40000023E36394F82230083B022BE5D9042338
:10DC500084F82230064B1B682363064B1B68636302
:10DC6000DBE7082384F82230ECE70A28D5D1E9E77E
:10DC7000100000201400002038B5044602F0E2FD38
:10DC8000054694F82230083B022B13D902F0DAFD46
:10DC9000236C401B98420DD2236820469B6898470E
:10DCA00018B12046FFF77AFFE8E74FF47A7002F0E8
:10DCB000FDFDE6E794F82230083B022B94BF0020DC
:10DCC0006FF0020038BD10B590F82230083B022BEF
:10DCD000044601D9FFF7D0FFA06A10BD38B590F80F
:10DCE0002230083B022B054601D9002038BDFFF742
:10DCF000EAFF0130F9D02846EC6AFFF7E4FF8442DE
:10DD0000B4BF00200120F1E7FFF7E8BFFFF7E6BF4F
:10DD100038B500F1480504460E49284602F0C9FC12
:10DD200094F82230083B022B09D92046FFF736FF32
:10DD30000D2801D00A2807D1236D002BF0D0206DCB
:10DD4000003018BF012038BDC1B2284602F0D2FC15
:10DD5000E6E700BFE695010007B5002300931A46E9
:10DD60001946034801F02AFF03B05DF804FB00BF29
:10DD70005C07002080687047C1607047036810B579
:10DD80009B690C469847036821461B68BDE8104014
:10DD900018472DE9F84380460D46174601EB020966
:10DDA0000C46A145A4EB050609D0D8F80030404642
:10DDB000DB689847431C03D004F8010BF1E73E46AB
:10DDC0003046BDE8F883C368013310B5044612D16C
:10DDD000236820469B69984703689B68984758B119
:10DDE00023682046DB6898472028F1DD2368C1B20C
:10DDF0005B6920469847012010BD70B50446C06895
:10DE0000431C18D102F01EFD00F5FA752368204668
:10DE10009B69984703689B68984718B902F012FD00
:10DE20008542F3D8236820469B6998470368BDE87C
:10DE30007040DB6818474FF0FF33E36070BD10B5EA
:10DE4000182005F01DF8044618B11822002105F02D
:10DE50006CF8204610BD70B506460C46D4B1237C44
:10DE600065681B0704D4E16811B13046FFF7F3FF82
:10DE7000237C03F00F03042B03D1606908B100F089
:10DE8000D1FC206808B100F0CDFC204605F000F878
:10DE90002C46E3E770BD00002DE9F04F036885B024
:10DEA000DB6805460E469847421C044604D14FF0F5
:10DEB000FF3005B0BDE8F08F2D282FD12B68284604
:10DEC000DB689847431C0446F1D04FF0FF330093C2
:10DED000A4F13003092B4FF000070DD84FF00A08CA
:10DEE0002B682846DB689847A0F13003303C092BAB
:10DEF00008FB07470446F3D92E2C11D024F0200349
:10DF0000452B0DD0009B7B437361022333742B6838
:10DF100028465B69E1B298470020CAE70123D6E7AB
:10DF2000384604F0A9F92E2C8046894639D12B6851
:10DF3000DFF814B1DB6828469847002704464FF005
:10DF4000000A52465B464046494604F0FFF98046C7
:10DF50008946A4F1300004F08FF942464B4604F0A4
:10DF60003FF82B688046DB68284689469847A0F131
:10DF70003003092B07F1FF370446E2D924F02003D0
:10DF8000452B2AD12B682846DB6898472B28044666
:10DF900009D12B682846DB68984704464FF0010AF0
:10DFA0000AE00027EAE72D28F8D12B682846DB682D
:10DFB00098474FF0FF0A04464FF0000B0A22A4F1E5
:10DFC0003003092B0DD802FB0B3B2B680392DB6857
:10DFD00028469847039A0446F1E74FF0010A4FF0AC
:10DFE000000B009804F048F942464B4604F0AEF9A5
:10DFF000CDE90001584604F03FF980465046894675
:10E0000004F02AF902460B464046494604F09EF9C0
:10E0100080463846894604F02FF902460B464046B2
:10E02000494603F0DDFF02460B460020064902F098
:10E03000F7FE0B460246DDE9000104F087F904F023
:10E040007DFC0323706161E70000244019B10A22BE
:10E05000496901F042BE0846704700000000000018
:10E06000F8B506462DED028BD1B391ED058A18EE79
:10E07000100A04F013F9B5EEC08AF1EE10FA044666
:10E080000D4606D51A49304601F0E9FD05F1004379
:10E090001D462946204604F031FC0A220146074667
:10E0A000304601F048FE1349304601F0D8FD3846AD
:10E0B00004F0D2F802460B462046294603F08EFFB4
:10E0C00009A3D3E9002303F08BFF00220A4B04F0DD
:10E0D0003DF904F013FC0A220146304601F03AFEF5
:10E0E000BDEC028B0020F8BD9A9999999999A93FA6
:10E0F0002B9B0100038D010000002440F8B503684C
:10E10000DB6806460F469847222803D04FF0FF34BD
:10E110002046F8BD04233B7400F0F4FA05460028BD
:10E12000F4D033683046DB689847431C044611D06E
:10E13000222C36D01F2C34DD5C2C04D02946E0B2D2
:10E1400000F0F6FAEDE733683046DB689847421C8A
:10E15000044603D1284600F0F7FAD9E7622817D021
:10E1600007DC2F2803D05C2801D02228D9D12946EA
:10E17000E6E76E280FD004DC6628D2D129460C20B1
:10E18000DEE772280AD07428CBD129460920D7E7C8
:10E1900029460820D4E729460A20D1E729460D2040
:10E1A000CEE7284600F012FB00247861B0E70000BB
:10E1B00038B50D461D49044601F051FD7DB3013DC2
:10E1C00015F8011F59B31F2907D9222905D05C2949
:10E1D00003D0204601F047FDF2E75C21204601F024
:10E1E00042FD29780C2914D007D8092915D00A290D
:10E1F00011D00829E4D16221EBE72229E9D003D824
:10E200000D29DDD17221E4E72F29E2D05C29E0D08D
:10E21000D6E76621DDE76E21DBE77421D9E722210D
:10E22000204601F020FD002038BD00BFEC79010040
:10E230004969FFF7BDBF38B50368DB6804469847F6
:10E240004FF48075411C0FD020280EDC013D6A1C64
:10E25000236803D0DB6820469847F3E72368C1B200
:10E260005B6920469847002038BD002DF6D14FF05D
:10E27000FF30F9E703682DE9F047DB68044688467C
:10E28000914698477B2803D04FF0FF30BDE8F087D8
:10E29000062388F810302046FFF7CDFF236820467C
:10E2A000DB6898477D2843D02368C1B25B6920466C
:10E2B0009847FF264FF0000AFFF7C1FD05460028EA
:10E2C000E2D096B3C8F80C002046FFF7B4FF294609
:10E2D0002046FFF713FF0130D6D02046FFF7ABFFF3
:10E2E0006B692B602368C5F814A0DB68204698474B
:10E2F0003A28C9D12046FFF79EFF4A4629462046C4
:10E3000000F018F80130BFD02046FFF794FF2368D3
:10E310002046DB6898472C282F464FF00006CBD0CC
:10E320007D3818BF4FF0FF30B0E778608760CBE7EB
:10E330000020ABE7F7B504460E461746FFF77BFF14
:10E34000013002D14FF0FF3011E023682046DB6836
:10E350009847431C0546F5D02368C1B25B69204647
:10E360009847222D05D131462046FFF7C7FE03B05E
:10E37000F0BD2D2D03D0A5F13003092B04D8314673
:10E380002046FFF789FDF2E75B2D05D13A4631467D
:10E39000204600F078F8EAE77B2D05D13A46314671
:10E3A0002046FFF767FFE2E76E2D15D102AD00238F
:10E3B00045F8083D236804221B69294620469847F2
:10E3C00004280246BED11D49284605F070FD0028EC
:10E3D000B8D100233374CAE7662D16D10023009309
:10E3E0008DF80430236805221B696946204698474A
:10E3F0000528A7D105221249684605F058FD0028D6
:10E40000A0D1012333743075B1E7742D9AD102ADD8
:10E41000002345F8083D236804221B69294620464D
:10E420009847042802468DD10649284605F03FFD4D
:10E43000002887D101233374337598E7AA9501002A
:10E44000AF950100B5950100F8B5064617460D4693
:10E4500011B900242046F8BDFFF7F1FC044600285E
:10E46000F7D02846FFF7E7FE3A4621462846FFF751
:10E4700061FF0130EED121463046FFF7ECFCE8E7C2
:10E480000022FFF7E1BF2DE9F8430368DB6804468B
:10E490008846914698475B2803D04FF0FF30BDE88F
:10E4A000F883052388F810302046FFF7C4FE236860
:10E4B0002046DB6898475D282AD02368C1B25B6993
:10E4C00020469847FF26FFF7BAFC05460028E4D00F
:10E4D000DEB1C8F80C002046FFF7ADFE4A462946DB
:10E4E0002046FFF727FF06460028D6D12046FFF733
:10E4F000A2FE23682046DB6898472C282F46E2D0EE
:10E500005D3818BF4FF0FF30C9E778608760E2E7F9
:10E510000020C4E738B5054651B3CC687B2101F033
:10E52000A2FB013002D14FF0FF3038BDB4B12168F9
:10E530002846FFF73DFE0130F5D03A21284601F08C
:10E5400092FB0130EFD02146284600F013F801304D
:10E55000E9D0646814B12C212846E0E77D212846E3
:10E5600001F081FB01304FF0FF3018BF0020DCE7E5
:10E570000846DAE7E9B10B7C03F00F03062B18D845
:10E58000DFE803F004070D0F111315000A4901F02D
:10E5900066BB0B7D0BB10949F9E70949F7E7FFF7BE
:10E5A00055BDFFF75DBDFFF743BE00F00EB8FFF7A6
:10E5B000B1BF0020704700BFAA950100B5950100CA
:10E5C000AF9501001046FFF7D5BF38B50546F1B14C
:10E5D000CC685B2101F047FB013002D14FF0FF30E6
:10E5E00038BD54B121462846FFF7C4FF0130F5D0AD
:10E5F000646814B12C212846ECE75D21284601F01F
:10E6000032FB01304FF0FF3018BF0020E8E708462A
:10E61000E6E731B1CB680022D0B2013213B15B68BA
:10E62000FAE70846704731B1C96821B11AB1013A19
:10E63000D2B24968F9E70846704738B515460C4626
:10E6400041B1CC6834B12946206805F0ACFB08B173
:10E650006468F7E7204638BD51B14AB1CB6813B9B9
:10E66000CA6070470B4659680029FBD15A60936015
:10E670007047F8B505460E4617461C4673B1186834
:10E6800008B100F0CFF8384600F076F82246206056
:10E6900031462846BDE8F840FFF7DEBFF8BD08B5B3
:10E6A000FFF7CDFB18B1037C6FF303030374037C06
:10E6B0006FF30713037408BD10B50C46FFF7BFFBDB
:10E6C00010B102230374446110BD70B50D461946A4
:10E6D00004461646FFF7F0FF324603462946204619
:10E6E000BDE87040FFF7C5BF07B5002300931A4689
:10E6F0001946034801F062FA03B05DF804FB00BF5D
:10E700006407002038B50C2004F0BAFB044650B171
:10E71000064820604FF480752A46002104F005FC6D
:10E7200000236560A360204638BD00BF7808002044
:10E73000D1E90132013B9A4204D20B6898548B68AC
:10E7400001338B600020704708B104F0A1BB704713
:10E7500038B5054658B1074C216819B1284605F06F
:10E760005CFB10B1A468002CF6D1204638BD0446ED
:10E77000FBE700BF70070020F8B50746FFF7E8FF8A
:10E7800020B10379013303710068F8BD0E4D2B6889
:10E7900043B9384605F054FB012328602B71F4E798
:10E7A0003546F4E7AE68002EFAD10C2004F068FB81
:10E7B00004460028E9D0A860384605F041FB012353
:10E7C00020602371A660E0E770070020826838B5FA
:10E7D000044622B10368134413F8013C1BB12146DF
:10E7E0000020FFF7A5FF0548FFF7C6FF054610B15B
:10E7F000204604F04DFB284638BD00BF78080020B5
:10E8000010B5074CA06800B910BD0268836822B932
:10E81000A36004F03DFBA368204604461846F2E7D7
:10E820007007002038B5FFF793FF054660B1047903
:10E83000013CE4B204713CB9006804F029FB2C608F
:10E84000BDE83840FFF7DCBF38BD000008B5064B17
:10E850001B7843B9054801F009FA05490348BDE8AA
:10E86000084001F0F3B908BDC1070020D40700201B
:10E87000E0950100F0B504789FB005464CB31C4B01
:10E880001C4F1B68986804F0ABF92846194906F03C
:10E890007BF91EAD012445F8780D3946002006F0BD
:10E8A00073F91E2C264645F8240002D001340028B6
:10E8B000F3D1114B009F1C6884B12168384605F0E4
:10E8C000ACFA48B963682946304698470446FFF7D2
:10E8D000BDFF20461FB0F0BDA468EDE7074B1B78D5
:10E8E000002BF6D10649074801F0C6F9EFE700BF53
:10E8F00038000020147B0100BC070020C107002065
:10E90000E7950100D4070020F8B505460C200F4616
:10E9100004F0B6FA0C4B04461860284605F0ABFA32
:10E92000013004F0ADFA2946064605F080FA284683
:10E9300005F0A1FA00233354044B1A68A260C4E91D
:10E9400000671C60F8BD00BFBC0700207C070020EA
:10E95000184B1B7870B5FBB91748184D01F0D4FC63
:10E96000C4B20A2C0CD00D2C0AD0082C15D121468B
:10E97000114801F078F92B7873B1013B2B700BE053
:10E980002B780F4E0F490C480024F45401F067F91E
:10E990003046FFF76FFF2C7070BD2146064801F02E
:10E9A00062F92B783A2B9FBF5A1C2A70044AD45420
:10E9B000F2E700BFC1070020D4070020C0070020F5
:10E9C00080070020E4950100064B1B7810B53BB989
:10E9D000054C204601F092FC10B1FFF7B9FFF8E7B3
:10E9E00010BD00BFC1070020D4070020054A002346
:10E9F0001370054A0146136010B1044801F03EBC93
:10EA0000704700BFC00700207C070020D40700200B
:10EA100070B504460D4601F015FFA061A0680368BB
:10EA200029461B68BDE87040184770B504460D467E
:10EA3000164601F007FFA061A06803683246294628
:10EA40005B68BDE87040184710B50446C06804F024
:10EA50001FFA204610BD2DE9F04105460E4601F093
:10EA6000F1FE4FF47A778046A86803689B68984760
:10EA7000044658B901F03CFF01F0E4FEAB8AA0EB7C
:10EA800008007B439842EFD3204605E0A86803685E
:10EA9000DB68984730700120BDE8F08138B51488F4
:10EAA00021441546FFF7D7FF08B101342C8038BD4B
:10EAB0002DE9F74F02AD002625F8026D8A462A4659
:10EAC000C1680446FFF7EAFF18B9002003B0BDE8AB
:10EAD000F08FE3680DF1080993F8008009F8036DE1
:10EAE0000127BDF80630052B07D14FF0FF33A06892
:10EAF000E36303685B6A9847E7E749462046FFF708
:10EB0000AAFF0028E1D0BDF80630E268591CADF834
:10EB100006109DF80510D1549DF8053003F07F02D2
:10EB200007FB02661A064FEAC717DAD49DF80630CB
:10EB300008F0F008013BB8F1300F8AF800301DD121
:10EB40002A46E1682046FFF7A9FF0028BDD02A46E3
:10EB5000E1682046FFF7A2FF0028B6D0E2689AF8E5
:10EB60000030134459789D78137805EB01259B07F5
:10EB7000ADB201D50235ADB2022701E000273D4616
:10EB8000BDF806B0A7EB0B0707EB0B0296422AD99C
:10EB900049462046FFF75FFF002896D0A06B88B15A
:10EBA000B8F1300F0ED19AF80020C2F1FF2202F521
:10EBB0007F02FE325A44AA4204D902689DF8051029
:10EBC00012689047BDF80620218A914208D9E16871
:10EBD0009DF805008854BDF806200132ADF80620E6
:10EBE0000BF1010BD0E7A26B22B9218A594538BF3E
:10EBF000ADF80620BDF8060068E70120704773B540
:10EC00000025DC1103F07F06A3B20CB146F08006AC
:10EC10000DF1080C681C6544C0B205F8046C05468B
:10EC2000002CEED1C0F10405515501ADA04205DD27
:10EC3000231A1344615D59710134F7E7013002B0C2
:10EC400070BDF8B5064617461C46FFF7D8FFB368F7
:10EC5000C0B21A680444C0F105015568394422461F
:10EC60001846A847054601F0EDFDB061A8B2031BA8
:10EC700058425841F8BD10B5C368E0221A70C36805
:10EC800000225A7004468068E168036802225B68CB
:10EC90009847A0684FF0FF33E36303685B699847C8
:10ECA000A06803685B6A984701F0CCFDC4E90600E0
:10ECB00010BD023330B598B20C46631A14F8015BEC
:10ECC0009BB21DB1431C155498B2F6E7C11A0A4411
:10ECD000191202F8021C02F8013C30BD38B5054695
:10ECE000806808B9002038BD03689B6A9847EC6BC0
:10ECF00068B9002CF6D1A8686FF00203EB630368D3
:10ED00005B699847A86803685B6A9847EAE7B4FAC2
:10ED100084F04009E7E700002DE9FF470C9D9DF8CE
:10ED200040A00446894617461E46FFF7D7FF804697
:10ED3000002840F0DF80A06803689B6A984700289D
:10ED400040D00123E3826E4B029345F25443ADF869
:10ED50000C3004238DF80E30052302A91944E26813
:10ED600011F8051CD15401330C2BF6D1002D3DD0E8
:10ED70009DF838309DF834205B0143F0040343EAEA
:10ED8000C203DBB2BAF1000F01D043F002031FB19E
:10ED9000002E2DD143F08003E2681373638AE2688A
:10EDA0001B125373E368628A9A73218A484605F0FE
:10EDB000A5F8238A113098421DD9A06803685B6AC0
:10EDC000984797E0A068216B0368A28E39B1DB6990
:10EDD00098470128B5D06FF00103E3638AE0494901
:10EDE0009B690291E16A039102A9F1E72B46C9E709
:10EDF00043F0C003D0E749460F23E2682046FFF7FF
:10EE000058FF814605B3218A284605F077F809F1B5
:10EE100002031844238A9842CFD84B462946E26819
:10EE20002046FFF746FF218A05460F9805F066F851
:10EE3000238A023028449842BFD82B46E2680F99B3
:10EE40002046FFF736FF814617B3218A384605F082
:10EE500055F809F102031844238A9842ADD84B466D
:10EE6000E26839462046FFF724FF814686B1218AB1
:10EE7000304605F043F809F102031844238A98420A
:10EE80009BD84B46E26831462046FFF712FF814689
:10EE9000A9F105039BB2E26810212046FFF7D1FEDD
:10EEA00001F0D0FCC4E906004FF47A75A06803684D
:10EEB0009B68984758B901F0C5FCE369C01AA38A5A
:10EEC0006B439842F2D36FF00303E36375E70DF1F0
:10EED00007012046FFF7ECFD04287FF46EAFE368DE
:10EEE000DD785DB901F0AEFC4FF00108E06184F817
:10EEF0002050E563404604B0BDE8F087E5635CE779
:10EF000000044D519096010010B586B00124049480
:10EF10000B9C03949DF8284002949DF82440019492
:10EF2000089C0094FFF7F8FE06B010BD2DE9F347EA
:10EF30000446FFF7D3FE8046D0B101F083FC628A1D
:10EF40004FF47A735343E269821A9A42074603D810
:10EF5000A269821A93421FD294F8203063B16FF0F5
:10EF60000303A068E36303685B6A98474FF00008F7
:10EF7000404602B0BDE8F087E268C0211170E26847
:10EF80005370A068E168036802225B689847C4E98F
:10EF90000677012384F82030A06803689B689847AF
:10EFA0000028E5D00DF107012046FFF781FD83B26F
:10EFB0000646002B73D0E368E7611A7802F0F0028E
:10EFC000302A57D1626A002AD2D09DF807209918BA
:10EFD000901C49781D5C05EB0125ADB2D11C19448C
:10EFE0002A46184403F088FFE3689DF807202B4465
:10EFF000134400229A70E1689DF807C091F80090D0
:10F0000009F00609B2B20CF10200B9F1020F08448E
:10F01000666A0CF10303A2EB0C0225D12B440CF120
:10F02000050C11F803E00B44521B93F801A0654452
:10F03000053A29440AEB0E2AB047E36840221A70C9
:10F04000E36883F80190E3681FFA8AFA4FEA2A22FC
:10F050009A70E36883F803A0A068E168036804225B
:10F060005B689847A76183E72B44033A521B194416
:10F07000B0477DE7C02A0BD1D0221A70E368002286
:10F080005A70A068E168036802225B6898476FE7DE
:10F09000D02A7FF46DAF002384F8203068E7204643
:10F0A000FFF71CFE002808BF4FF0000860E770B5AE
:10F0B00090B005460E46FFF711FEE0B1304604F071
:10F0C000DAFE3123C4B28DF80030A31C8DF8013074
:10F0D0003B220023314601A88DF802308DF8034011
:10F0E00004F0F7FE2B68221D5B68694628469847A6
:10F0F000003018BF012010B070BD2DE9F047044664
:10F10000884617461D469DF82060FFF7E7FD50B37F
:10F11000B4F810904046494604F0F0FEEB1D184448
:10F12000814520D341460523E2682046FFF7C1FD13
:10F1300000211FFA81FC4318AC459BB2E26801F143
:10F14000010104D217F80CC002F803C0F1E7002E49
:10F15000A3F1050320469BB214BF31213021BDE845
:10F16000F047FFF76EBD0020BDE8F08773B5054698
:10F170000E4614466AB1018A104604F0BFFE0346EB
:10F1800000220092314622462846FFF7B6FF02B021
:10F1900070BD1346F4E7F7B505460E461F46144604
:10F1A00062B1018A104604F0A9FE03460097224688
:10F1B00031462846FFF7A1FF03B0F0BD1046F4E743
:10F1C0002DE9F0470446884692461E46FFF786FD25
:10F1D000002843D0218A404604F090FE9DF820305C
:10F1E000002BE3680CBF3022312287B21A70B21CA8
:10F1F0003A44012002F07F01E568D20918BF41F0CE
:10F200008001431C29545FFA80F9D2B941469BB270
:10F21000E2682046FFF74DFDA368E1681A68D2F85E
:10F22000048002461846C04755468046B244AA4567
:10F2300009D0A06815F8011B03681B689847804433
:10F24000F5E71846D6E701F0FDFAA06109F10300E1
:10F2500038443044A0EB080358425841BDE8F087D9
:10F26000F7B505460E461F46144662B1018A1046A0
:10F2700004F044FE03460097224631462846FFF735
:10F280009FFF03B0F0BD1046F4E7F8B505460E4603
:10F2900014461F46FFF722FD28B331460523EA68CE
:10F2A0002846FFF706FD631F002F03440CBF3021E3
:10F2B000312106469BB2EA682846FFF7A0FC0146CA
:10F2C000A868EC680368053E0E44C1F105015B685F
:10F2D000214432469847044601F0B4FAA861A0B22E
:10F2E000831B58425841F8BD70B50D460446018A4B
:10F2F0002846164604F002FE45B3012E26D8238A7E
:10F300000930834222D32046FFF7E8FCF0B1E38ABC
:10F3100001339BB2C3B1E382E38AE2681B125371EB
:10F32000E368E28A9A71E268294607232046FFF7DC
:10F33000C0FCE3681E54031FE26820469BB2822192
:10F34000BDE87040FFF77DBC0123E4E7002070BDFD
:10F350000022FFF7C9BF70B50D460446018A284652
:10F3600004F0CCFD25B3238A0930834220D3204604
:10F37000FFF7B4FCE0B1E38A01339BB2B3B1E3829F
:10F38000E38AE2681B125371E368E28A9A71E268C9
:10F39000294607232046FFF78CFC431FE2682046DE
:10F3A0009BB2A221BDE87040FFF74BBC0123E6E70A
:10F3B000002070BD01638286704741627047C06B58
:10F3C000704738B504460D4609B9002038BD038A98
:10F3D0004BB9084603F054FDE060E0682582003038
:10F3E00018BF0120F2E7C06804F022FC0028F3D126
:10F3F000EBE7000070B50C4B00250446456040F873
:10F40000283B0E4600F0D2FB4FF0FF33E363A660CB
:10F41000A56325824FF480712046FFF7D2FF0F23AA
:10F420006382A382204670BD0096010007B50023C9
:10F4300000931A461946034800F0C0FB03B05DF87C
:10F4400004FB00BFC40700208271054A41711268A5
:10F450000449B2FBF1F14FF47A724A43C26070473B
:10F460001800002040420F0038B504460D46407990
:10F47000022101F0D5FB01F0E5F9A0F5FA60A060EA
:10F48000657438BD70B505460E460024687901F0F4
:10F4900001FCB042A3B206D1EA689A4204F1010429
:10F4A000F4D84FF0FF33184670BD30B50D46D1B0DB
:10F4B000044601F0C7F93DB9A368C31AB3F5FA6F62
:10F4C00002D2207C51B030BD00250221A060256011
:10F4D0006079257101F0A4FB012001F0E7F9012119
:10F4E000607901F09DFB2946607901F0C1FBA379A9
:10F4F000153B012B00F28C8040F24C40013800BFDC
:10F5000000BF00BF00BF00BF00BF00BF00BF00BF03
:10F5100000BF00BF00BF00BF00BF00BF00BF00BFF3
:10F5200000BF00BF00BF00BF00BF00BF00BF00BFE3
:10F5300000BF00BF00BF00BF00BF00BF00BF00BFD3
:10F5400000BF00BF00BF00BF00BF00BF00BF00BFC3
:10F5500000BF00BF00BF00BF00BF00BF00BF00BFB3
:10F5600000BF00BF00BF00BF00BF00BF00BF00BFA3
:10F5700000BFC3D16079022101F052FB607C0028FA
:10F580003BD0013800BF00BF00BF00BF00BF00BFBD
:10F5900000BF00BF00BF00BF00BF00BF00BF00BF73
:10F5A00000BF00BF00BF00BF00BF00BF00BF00BF63
:10F5B00000BF00BF00BF00BF00BF00BF00BF00BF53
:10F5C00000BF00BF00BF00BF00BF00BF00BF00BF43
:10F5D00000BF00BF00BF00BF00BF00BF00BF00BF33
:10F5E00000BF00BF00BF00BF00BF00BF00BF00BF23
:10F5F00000BF00BF00BF00BFC3D172B600212046CC
:10F60000FFF740FF013007D10020207462B659E7B0
:10F61000142001F04BF9ADE701212046FFF732FF3E
:10F620000130F1D0002500212046FFF72BFF0121FA
:10F630004DF805002046FFF725FF0DEB05030835C3
:10F64000B5F5A07F5860EED162B600225DF8325069
:10F650000DEBC203691C586801D0431C02D1002085
:10F6600020742FE7D1108542635C4FEA4303DBB27D
:10F6700002F1010238BF43F00103282A6354E5D1A7
:10F680006178237822790B44A1780B44E1780B440C
:10F69000DBB29A42E3D10120E2E700000000000063
:10F6A0002DE9F8430D462DED028B11460446FFF778
:10F6B000FCFE00287ED0A3790B3B0B2B7AD8DFE829
:10F6C00003F0063F79797979797979796565A37855
:10F6D000E07808EE103A0106B8EE488A48BFFFEE1F
:10F6E000007A00F00F0048BF37EEC88A02F0C4FD70
:10F6F00031A3D3E9002302F029FE064618EE100AD2
:10F700000F4602F0CBFD0B4602463946304602F06A
:10F7100067FC03F013F903466DB102F0BFFD2AA3A5
:10F72000D3E9002302F012FE254B002202F058FC20
:10F7300003F004F90346BDEC028B1846BDE8F883DC
:10F74000E078A67800F00F0002F096FD1AA3D3E946
:10F75000002302F0FBFD07EE906AF8EE677A804620
:10F7600017EE900A894602F099FD02460B46404684
:10F77000494602F035FC03F0E1F83206034648BF83
:10F7800080F00043002DD6D01846C6E7A678E3786F
:10F79000300200F4FE40184307EE900AF8EEE77AD4
:10F7A00017EE900A02F07AFD03A3D3E9002302F0DA
:10F7B000CDFDE0E7034BBEE79A9999999999B93F36
:10F7C000000040400000C07FCDCCCCCCCCCCFC3F76
:10F7D000D0B50446FFF769FE90B3A3790B3B0B2B22
:10F7E0002ED8DFE803F006062D2D2D2D2D2D2D2DE5
:10F7F0001C1C607802F040FD14A3D3E9002302F042
:10F80000A5FD064620780F4602F036FD02460B465F
:10F810003046394602F0E4FB03F090F8D0BD208872
:10F8200040BA80B207EE900AF8EEE77A17EE900A37
:10F8300002F034FD05A3D3E9002302F087FDEBE7D6
:10F840000148EBE7AFF300800000C07F9A999999D7
:10F850009999B93F00B55DF804FB0020704700B5E9
:10F8600001205DF804FB10B50446C06803F010FBEE
:10F87000B4F90600002802DB002101F0D1F920468E
:10F8800010BD70B50546C0680E4603F001FBEC7C68
:10F890002A7C94420CBF0324042414FB06F4A4B273
:10F8A000AC80204603F0ECFAE86028B12246002143
:10F8B00003F03BFB6E8070BDA8806880FBE7F0B46E
:10F8C000FF29C1F38107C1F38112C1F30115477408
:10F8D00001F003078CBF002101210170C168C47CC5
:10F8E000067CC2740574877461B1A41B6142A2EBEB
:10F8F000050561416A426A41914203D04188F0BCEA
:10F90000FFF7BFBFF0BC704738B5437804460D46DB
:10F9100033B1B0F90600002802DB002101F080F9C4
:10F920006378E5804BB12846012101F079F928463A
:10F930000021BDE8384001F09BB938BD70B50E46D6
:10F940000021044641700172C160416119461546AB
:10F95000FFF7B5FF31462046FFF793FF20462946C3
:10F96000FFF7D2FF204670BD70B540F2FA5404FB99
:10F9700000F303F500431B14B3F5FF7F98B222DABE
:10F98000FE2BD8B242DDC0F1FE00C5B20023FF203D
:10F990004E1CC943C9B27043013201EB20205043D1
:10F9A00000F47F4406FB03F006FB05F301EB202087
:10F9B00001EB232150434A43120244EA102002F48F
:10F9C0007F02104370BDB3F57F7F0DDAB0F53F7F46
:10F9D000DBB28BBFC3F1FC030233D8B2DBB294BFFE
:10F9E000FF20FF230025D3E7A04211D040F2FA44C4
:10F9F000A042DBB204D80433DDB20020FF23C7E706
:10FA0000C3F1FA03DBB20020FF25C1E70023FBE7C7
:10FA100000231846F8E7000070B504460830154684
:10FA20000E4600F0C3F8FF23064A84F82230002374
:10FA3000266025712361A382C4E90622238420461F
:10FA400070BD00BF2B9B01000161828270470000E6
:10FA5000024B002908BF1946816170472B9B0100AA
:10FA6000024B002908BF1946C16170472B9B01005A
:10FA70000184704773B50D4601690446164639B9CD
:10FA80002B4BC2685B689A4202D1002002B070BD65
:10FA9000A28A002AF9D094F8223005F00700034129
:10FAA000DB0738D515F47E7F08BF238C206804BFA0
:10FAB00003F47E731D43036800292ED05B6A9847C8
:10FAC0000128E2D13C21206800F0CDF80A22294625
:10FAD000206800F024F9237933BB1649206800F030
:10FAE000B5F8A169206800F0BAF82021206800F07C
:10FAF000BAF8E169206800F0B2F82379B3B90E4989
:10FB0000206800F0A3F83146206800F0A8F82068CB
:10FB100003689B6A98470120B8E708490091E168AB
:10FB200001911B6A6946CAE70549D7E70549E7E736
:10FB3000CC070020089601000E9601009096010067
:10FB4000737A01001996010008B5FFF793FF08BD0D
:10FB500007B5002300931A461946034800F02EF813
:10FB600003B05DF804FB00BFCC0700202DE9F8438B
:10FB700006460D46071D00F10709002417F8011B72
:10FB80000A22284600F0E4F82E218046284600F09C
:10FB90006AF84F4540440444F0D10A22F1792846DE
:10FBA00000F0D6F82044BDE8F8830000024A026065
:10FBB00000224260704700BF9096010030B583710B
:10FBC000034D9DF80C30056001714271C37130BD69
:10FBD00090960100014AC0E900217047909601000B
:10FBE000024A02600A684260704700BF90960100B6
:10FBF0000B6843607047416070472DE9F04106464D
:10FC00000D4601EB02080C464445A4EB050707D05E
:10FC1000336814F8011B1B68304698470028F3D15D
:10FC20003846BDE8F08170B5044608460D4604F03C
:10FC300022F923680246294620465B68BDE87040E9
:10FC4000184709B1FFF7EFBF0846704708B5FFF73F
:10FC5000F8FF08BD03688A685B680968184708B53B
:10FC6000FFF7EFFF08BD03681B6818470149FFF75E
:10FC7000DABF00BFE495010038B50546FFF7E1FFA4
:10FC800004462846FFF7F2FF204438BD38B5054644
:10FC9000FFF7D7FF04462846FFF7E8FF204438BDAA
:10FCA00070B58AB00D460AA9002301F8043D012A67
:10FCB00098BF0A22B5FBF2F402FB1456F3B2092EE8
:10FCC00094BF30333733DBB2254601F8013D002CB9
:10FCD000F0D1FFF7B6FF0AB070BD2DE9F04107463D
:10FCE0000E4615462AB90368C9B21B68BDE8F04143
:10FCF00018470A2A05D1002905DBBDE8F041FFF7C6
:10FD0000CFBFD2B2F9E72D21FFF7ADFF2A46044657
:10FD100071423846FFF7C4FF2044BDE8F081FFF789
:10FD2000DCBF38B50546FFF7D8FF04462846FFF785
:10FD30009DFF204438BD10B42AB903685DF8044B18
:10FD40001B68C9B21847D2B25DF8044BFFF7A8BFD1
:10FD5000FFF7F1BFFFF7EFBF2DE9F84F1946064651
:10FD6000104614461D469DF8287002F089FD28B102
:10FD70004C493046BDE8F84FFFF755BF25F0004924
:10FD80004FF0FF32484B2046494602F079FD48B912
:10FD90004FF0FF32444B2046494602F053FD08B96C
:10FDA0004249E6E74FF06042414B2046294602F0C7
:10FDB0005DFD08B13F49DCE74FF060423E4B204615
:10FDC000294602F035FD0028F4D100220023204608
:10FDD000294602F02DFDD0B12D213046FFF743FF1B
:10FDE00005F1004382461D463449DFF8D8904FF0B4
:10FDF000000B00204FF000085FFA8BF39F4208D9F8
:10FE000042464B4602F0CCFB0BF1010BF4E7824675
:10FE1000EAE722462B4602F0E3F80D46044602F0DC
:10FE20006DFD0A22014680463046FFF739FF8244C5
:10FE3000A7B3404602F010FA02460B462046294678
:10FE400002F0CCF804460D4630461D49DFF87490A8
:10FE5000FFF7E9FE4FF000088244013FFFB2FF2F99
:10FE60001CD04B4642462046294602F06FFA0D460A
:10FE7000044602F01BFD0A22014683463046FFF786
:10FE80002CFF8244584602F0F7F902460B46204602
:10FE9000294602F0A3F804460D46DEE75046BDE8C9
:10FEA000F88F00BF94960100FFFFEF7F9896010046
:10FEB000FFFFEF419C960100FFFFEFC10000E03F14
:10FEC000038D0100000024409DF800100091FFF711
:10FED00043BF08B54022002103F027F80022C0E903
:10FEE000102208BD026C10B5531C446C03F03F0394
:10FEF0009C421CBF8154036410BD0023C0E9103331
:10FF00007047D0E9102393421FBFC25C013303F056
:10FF10003F03436414BF10464FF0FF307047D0E9F1
:10FF20001030181A48BF40307047D0E91023934270
:10FF300014BFC05C4FF0FF307047036C406C01335E
:10FF400003F03F031B1A5842584170470649074ABD
:10FF5000074B9B1A03DD043BC858D050FBDC00F074
:10FF600037F8F0F76DF900003C9B0100000000201D
:10FF7000A0020020FEE7FEE7FEE7FEE7FEE7FEE761
:10FF8000FEE7FEE7FEE7FEE7044B1868421C04BFED
:10FF9000034B1878831F58425841704730010010B6
:10FFA000E00F00F0074B1B78062B09D1064B1B68AE
:10FFB000C3F30313033B032B02D8044AD05C7047FE
:10FFC00000207047E00F00F0E80F00F0A496010059
:10FFD00008B5FFF7D9FF28B1654B664A1B68C3F324
:10FFE00004231360FFF7DEFF10B1634B634A1A600E
:10FFF000FFF7CAFF28B1624B624A1B68C3F3423362
:020000021000EC
:100000001360FFF7CFFF20B15F4AD36823F08073FE
:10001000D360FFF7B9FF40B14FF080430022C3F82F
:100020000C21C3F81021C3F83825FFF7BBFF10B12E
:10003000564B03221A60FFF7B5FF40B1544B05221F
:100040001A6001229A6700229A603F225A60514B3F
:100050001A68511C0BBF504B504B1A781B6802BFDB
:1000600008331B68C3F30313062A4DD1033B032B4C
:1000700003D84B4AD35C002B46D04FF08052494BFB
:10008000D2F80414C3F82015D2F80814C3F82415C4
:10009000D2F80C14C3F82815D2F81014C3F82C1594
:1000A000D2F81414C3F83015D2F81814C3F8341564
:1000B000D2F81C14C3F84015D2F82014C3F8441524
:1000C000D2F82414C3F84815D2F82814C3F84C15F4
:1000D000D2F82C14C3F85015D2F83014C3F85415C4
:1000E000D2F83414C3F86015D2F83814C3F8641584
:1000F000D2F83C14C3F86815D2F84014C3F86C1554
:10010000D2F84424C3F87025FFF73EFF28B1264BF0
:10011000264A1B6803F04F031360FFF735FF48B111
:100120004FF08043D3F80024D20744BF6FF00102A0
:10013000C3F80024174B1B68062B09D1174B1B680B
:10014000033B022B81BF1A4A136843F48063136098
:10015000184AD2F8883043F47003C2F88830BFF3ED
:100160004F8FBFF36F8F144B144A1A6008BD00BF46
:10017000240300104035014074C007400DF0ADBAB3
:10018000440200103C050040F0ED00E0A0050040F6
:100190001056004030010010E00F00F03401001054
:1001A000A096010000C0004058020010E40E00407C
:1001B0003C17004000ED00E0180000200090D00344
:1001C00010B5044600F03EFBE06023682046DB6883
:1001D0009847002808DA00F035FBE368C01AA368E6
:1001E0009842F2D34FF0FF3010BD2DE9F041804628
:1001F0000D468F180C46BC42A4EB050607D04046BE
:10020000FFF7DEFF002802DB04F8010BF3E73046BE
:10021000BDE8F0812DE9F8438046894616461C4624
:100220007BB1D7181546BD42A5EB060409D0404660
:10023000FFF7C6FF002804DB814502D005F8010B5B
:10024000F1E72046BDE8F88370B50D46094904463C
:10025000164600F0D1F92846FFF7B2FF002806DB6A
:10026000864204D0C1B2204600F044FAF3E72046AB
:1002700070BD00BFE695010001207047036813229E
:10028000DB69184770470369C3F81C150369D3F885
:100290001C21002AFBD00022C3F81C21012070473A
:1002A00010B490F95C30144C59090122203103F04C
:1002B0001F0302FA03F344F8213003695DF8044B8D
:1002C0000421C3F8081303695A600369DA600369FB
:1002D0000022C3F8002502694FF0FF33C2F80C3545
:1002E0000269C2F814350269C2F80835026914308F
:1002F000C2F81035FFF701BE00E100E01430FFF74F
:100300000EBE1430FFF711BE1430FFF7FABD000027
:10031000036990F85E2010B5C3F80C25036990F8C6
:100320005D20C3F8142590F861200369012A01BFFC
:1003300090F85F40C3F81045036990F8604006BF2D
:10034000C3F8084503690022B1F5966FC3F86C2520
:1003500069D9B1F5166F69D9B1F5965F69D9B1F56B
:10036000165F68D9B1F5615F67D9B1F5964F66D967
:10037000B1F5E14F65D9B1F5164F64D9B1F5614FCB
:1003800064D9B1F5963F64D9B1F5E13F63D9B1F5D0
:10039000613F63D9364B994263D9B1F5E12F63D9F7
:1003A000B1F5612F94BF4FF070634FF08053026935
:1003B000C2F8243503690422C3F80025016900232B
:1003C000C1F808310169C1F81C31016901230B60D2
:1003D00001698B600169C1F8042390F95C2051091F
:1003E00002F01F0293406031224A42F8213090F916
:1003F0005C30002BBDBF03F00F0302F6FC32D218B5
:100400009B18B5BF60236022137683F8002390F910
:100410005C300122590903F01F0302FA03F3154A65
:1004200042F8213010BD4FF49E23C0E74FF41D2346
:10043000BDE7114BBBE7114BB9E7114BB7E7114BC8
:10044000B5E7114BB3E74FF41D03B0E74FF46B036F
:10045000ADE70E4BABE74FF0EB73A8E74FF06C73D3
:10046000A5E74FF08063A2E74FF0E8639FE700BF86
:1004700090D0030000E100E000B01300005027001E
:1004800000F03A0000A04E0000C0750000903A0154
:100490002DE9F0411E4600254FF47A73C0E901535F
:1004A0000D4B044640F8143B17468846FFF711FDF4
:1004B0000A4AC4F8108084F85C7052F8263084F838
:1004C0005D309DF8183052F8233084F85E3084F89F
:1004D00061502046BDE8F081B096010020960100F1
:1004E00010B50369D3F8082104464AB1D3F81815AA
:1004F0001430C9B2FFF7F6FC23690022C3F80821C3
:1005000010BD00000148FFF7EBBF00BFD40700207B
:1005100007B5192300930222182303490348FFF764
:10052000B7FF03B05DF804FB00200040D4070020B3
:1005300010B5044628B103F047FB90FBF4F303FB2E
:100540001404204610BD884210B5044603DA081A88
:10055000FFF7EEFF0444204610BD10B5029C401A80
:10056000E41A6043521A90FBF2F0184410BD10B523
:100570000446006802F08CFC204610BD10B504460D
:10058000006808B102F084FC00232360C4E9013351
:1005900010BD38B504460D460068013103F048FB34
:1005A00010B1C4E90005012038BD036810B5044648
:1005B00023B143688B4201D3012010BD2046FFF7D1
:1005C000E8FF0028F9D0A368002BF5D1226813704A
:1005D000F2E770B50E46114604461546FFF7E5FFF3
:1005E00020B92046FFF7CAFF204670BDA5603146FE
:1005F000206803F01CFCF7E738B500230446C0E987
:10060000003383600D4639B1084603F034FC2946B7
:1006100002462046FFF7DDFF204638BD38B50546C7
:1006200008460C4603F027FC214602462846BDE852
:100630003840FFF7CEBF38B5054600680C4668B1B4
:100640006A688B689A4207D3096803F0F0FBA368D5
:10065000AB600023A36038BD02F01AFC23682B6056
:1006600063686B60A368AB600023C4E90033F1E703
:10067000884210B50B46044604D0096821B19A6837
:10068000FFF7A7FF204610BDFFF778FFFAE710B588
:1006900000230446C0E900338360FFF7E9FF2046EA
:1006A00010BD884210B5044601D0FFF7C4FF2046B4
:1006B00010BD10B5044619B1FFF7B0FF204610BDBC
:1006C000FFF75CFFFAE770B505460E4609B9002052
:1006D00070BD6AB1846814442146FFF766FF0028A4
:1006E000F5D02868AB683146184403F0A0FBAC6035
:1006F0000120EDE707B500238DF80410012201A9C0
:100700008DF80530FFF7DFFF03B05DF804FB10B58F
:100710008A6809680446FFF7D6FF10B92046FFF73C
:100720002DFF204610BD826808B53AB921B108787E
:10073000B0FA80F0400900E0012008BD006809B966
:100740000078F5E703F069FBF2E7884270B515D051
:1007500083688A6893420FD183B104680D68013CB5
:1007600014F8010F50B104F09BFB064615F8010B7D
:1007700004F096FB8642F3D0002070BD0120FCE718
:1007800083688B4201D9006818B9034800230370BD
:1007900070470844704700BF3808002083689342C0
:1007A00010B506D90468A01803F02AFB08B1001B95
:1007B00010BD4FF0FF30FBE70022FFF7EFBFF8B5A9
:1007C00083689342054602D84FF0FF30F8BD0368B6
:1007D000541C00221F5D1A550668304603F09AFB30
:1007E00037550028F0D02B68C01AEFE78268013A2D
:1007F000FFF7E5BF2DE9F0419A420E461F460F492B
:1008000088BF13461546804684BF3D461F46FFF706
:10081000F3FEB468AC420DD9BC4228BF3C463368F5
:1008200000221F5D1A55316840462944FFF741FFF9
:1008300033681F554046BDE8F08100BFE6950100D2
:10084000FEE700000A4B19680A4B30B5D3F80405DF
:100850000C060D0A44EA00024FF47A712B46A2FB03
:10086000014501FB0355E00B40EA454030BD00BFA8
:100870003C08002000100140094B1968094B30B5B5
:10088000D3F804050D0A0C06074944EA00022B467A
:10089000A2FB014501FB0355E00B40EA454030BD9A
:1008A0003C0800200010014040420F0038B50446CB
:1008B00048B1FFF7C7FF054600F01AF8FFF7C2FF7F
:1008C000401BA042F8D338BD074B0022C3F80421D7
:1008D00082B0D3F80431054A0193019B13680133B8
:1008E000DBB2136002B07047001001403C080020EA
:1008F000704770B58AB061B1931E222B20D801AB2E
:100900001D4648B9AB4207D00A46AB4213D8002374
:10091000137008460AB070BDB0FBF2F402FB140677
:10092000092E204603F10103F4B294BF303457344A
:1009300003F8014CE5E713F8010D02F8010BE4E7B9
:100940000021E6E77047000008B500F015F8FFF752
:10095000F9FF0120FFF7AAFFF5F72AF8034CF5F796
:1009600029F8002CFBD0AFF30080F8E7000000006E
:1009700002F086BA02F08CBA2A4BE02283F81123E7
:100980004FF40032C3F880211A604FF080430122F7
:10099000C3F818259A6003F588330021C3F80815B9
:1009A0000221C3F80413C3F844131A604FF0102354
:1009B000D3F80022002A03DBD3F80432002B2FDA0D
:1009C000194B0122C3F80425D3F80024002AFBD0D8
:1009D0004FF010221521C2F80012D3F80024002A8B
:1009E000FBD04FF010231522C3F804220E4B1A46F9
:1009F000D3F800140029FBD00021C3F80415D2F865
:100A00000034002BFBD0BFF34F8F0849084BCA6856
:100A100002F4E0621343CB60BFF34F8F00BFFDE7EA
:100A2000704700BF00E100E000E0014000ED00E0A1
:100A30000400FA05192837B50CD84B4B53F8203071
:100A4000052B00F0828007D8032B12D07BD8022B15
:100A500000F08180002074E01D2B78D003D81C2B7F
:100A6000F8D1052206E01E2B73D01F2BF2D10822ED
:100A700000E002223D4B196808296EDD0A296FDD6E
:100A80000D29B5BF0C240E24022303233848C0F8D7
:100A9000F0350123C0F8003500200546030103F1BD
:100AA000804303F5E04301300828C3F81455C3F828
:100AB0001055F3D12F4B18682F4B1B6800021B03F6
:100AC00003F4805300F4E0601843294BC3F8180581
:100AD000C3F81425C3F810250DF10602C3F82C261F
:100AE0000122C3F830261A60D3F80021002AFBD077
:100AF0000022C3F8002101225A601D4B1A46D3F888
:100B000004010028FBD00020C3F8040101209860F4
:100B1000D2F81431002BFBD00023C2F81431BDF9F8
:100B200006209A42124AB8BFADF80630A142C2F878
:100B30000035BDF9060004D035BF611A091BC84055
:100B4000884003B030BD032294E7042292E70622D6
:100B500090E707228EE701228CE70824002395E71F
:100B60000A24012392E700BF2096010028000020FC
:100B7000007000402C00002048080020192830B5E3
:100B80003CD8224B53F82000214B00221D4653F83D
:100B90002240B4F1FF3F32D11E4C45F822006FEAEB
:100BA00041411D4D1D4B246853F822306FEA5141DD
:100BB00025F81210012101FA04F4C3F86005013C84
:100BC000C3F8640505EB4202C3F86805C3F86C0579
:100BD0000020C3F80015C3F80C05C3F80405C3F8DA
:100BE0000845C3F81405C3F81005C3F82025C3F859
:100BF0002415C3F82815C3F82C05996030BD84422C
:100C0000CAD00132032AC2D1F8E700BF2096010002
:100C10001C0000203000002040080020D896010071
:100C200019280FD8114B53F8203003290AD8DFE8D0
:100C300001F002160A1003F5E0734FF0A042002104
:100C400042F82310704703F5E0734FF0A0420C21E7
:100C5000F6E703F5E0734FF0A0420421F0E703F557
:100C6000E0734FF0A0420321EAE700BF20960100A5
:100C700019280CD8064B53F82020012393404FF03D
:100C8000A04211B9C2F80C357047C2F80835704758
:100C90002096010019289FBF4FF0A043054AD3F8C2
:100CA000103552F820009ABF23FA00F000F001003E
:100CB000002070472096010038B50025057329B93A
:100CC0000B4B0C4A0C48252101F088FE01600B49B2
:100CD00051F82220027151F8233083719DF81030B1
:100CE00051F8233043710223C371856038BD00BFC2
:100CF000E496010047970100F2960100209601005A
:100D0000037B23B943738373036101230373704728
:100D100084B00DF1100C0CE90E009DF8081002686B
:100D200000230129C2F80035039B12D00BD30329FD
:100D30000CD0C2F85435019BC2F824350123C2F807
:100D4000003504B0704743F00203F2E743F00403B8
:100D5000EFE743F00603ECE710B5FFF7D1FF0368B8
:100D60008279C3F808254279C3F80C250279C3F8C3
:100D70001025034BBDE810400ECBFFF7C9BF00BFE5
:100D80006008002010B485B001AC84E80E0094E83F
:100D90000E0005B05DF8044BFFF7BABF704703685B
:100DA000C3F81C15D3F80821002AFBD0D3F8180586
:100DB0000022C3F80821C0B27047000007B5094BF4
:100DC00009490A484FF080421A6000229A600222C4
:100DD0001A710B2300930C220D23FFF76DFF03B054
:100DE0005DF804FB60080020003002404C08002041
:100DF0000B460146184601F01BBE0000C0F3C75366
:100E00007F3B162B024605DC002B04DB0348184110
:100E100022EA0000704700F000407047FFFF7F00AB
:100E20002DE9F04FDFF82C938DB006460F4614469F
:100E30001D4600F095F999F90080B8F1FF3FCDE922
:100E4000000136D022462B462046294601F018FDE7
:100E5000834670BB32463B463046394601F010FDB2
:100E60008246002840F0A280304639460022002306
:100E700001F0D4FC10B3002200232046294601F0E3
:100E8000CDFC8346002867D09FEDA77B0122AC4BA9
:100E9000CDF828A00292CDE90467CDE906458DED95
:100EA000087B0393B8F1000F41D09FEDA17B8DED3E
:100EB000007BDDE900010DB0BDE8F08FDDE9000148
:100EC00000F066FF8046002800F08D804FF0000A99
:100ED0004FF0000BDDE9000152465B4601F09EFC3D
:100EE0000028E6D03046394600F052FF0028E0D016
:100EF0002046294600F04CFF0028DAD099F900304E
:100F00008F4A039204210022022BCDE90467CDE928
:100F10000645CDE908AB02910A9203D002A800F081
:100F20003DFF50B901F092FD2223036005E002A8C5
:100F300000F034FF002800F09B800A9B1BB101F0F9
:100F400085FD0A9B03609DED087B8DED007BDDE94F
:100F500000010DB0BDE8F08F2046294600F018FFD3
:100F60000028A6D0002200232046294601F060FC7C
:100F700000289ED0724A99F90030CDF828B001219E
:100F8000CDE90467CDE90645CDE90212002B74D006
:100F90006C490020022BCDE9080172D101F056FD09
:100FA000212303600A9B002BCDD0C8E70022002339
:100FB0002046294601F032FC00283FF47AAF624B0C
:100FC0005F49CDF828B000220120B8F1020FCDE929
:100FD00004670290CDE90645CDE908230391A6D127
:100FE000CDE9002365E73046394600F0D1FE002800
:100FF0003FF46CAF2046294600F0CAFE00283FF4BB
:1010000065AFDDE900231046194601F039FC99F976
:1010100000A000286BD10323DFF824C10A902946E1
:10102000204602930022494BCDF80CC0CDE906457D
:10103000CDE9046701F08AF904460D46BAF1000FC4
:1010400025D1DFF814B14FF0604A0022002330466A
:101050003946CDE908AB01F0EBFB38BB02A800F044
:101060009DFE00289ED101F0F1FC2223036099E748
:1010700001F0ECFC212303605FE79FED2B7B8DEDFE
:10108000087B02A800F08AFE00288BD186E79FED3E
:101090002A7B00220023304639468DED087B01F083
:1010A000C7FBA0B9BAF1020FDDD0D7E72046294629
:1010B00000F07CFE22462B4601F0B0FBA0B9244B89
:1010C00099F900A04FF06042CDE90823EAE72046F5
:1010D000294600F06BFE22462B4601F09FFB18B913
:1010E000184B0022CDE9082399F900A0DAE7012284
:1010F000134BCDF828800292CDE90467CDE906456F
:101100000393BAF1000FB8D000220023104619460D
:1011100001F046FABAF1020FCDE908013FF43EAF03
:10112000AFE700BFAFF30080000000000000000048
:10113000000000000000F03F000000000000F07F11
:10114000849701000000F0FF0000F03F0000E03F46
:10115000FFFFEFC734000020FFFFEF470000000053
:101160002DE9F04F23F0004555EA020493B00DD06D
:101170006B4E21F00044B4420F4682460BDD04F171
:10118000404404F5801454EA0A0350D16549002014
:1011900013B0BDE8F08F9B46944647D0B542EEDCD5
:1011A0005F4EB5425DD0002F80468946CDE90023D1
:1011B0005BDB0026BCF1000F0ED1594B9D423FD0A6
:1011C000584B9D4200F08880BBF1804F00F09C801E
:1011D000554B9B4500F0B8834046494600F0D4FD8E
:1011E000BAF1000F06D1002C59D04E4B27F04042E7
:1011F0009A4254D0FF0F013F56EA070373D04B4B7E
:101200009D4240F39B8003F104739D4240F33E8472
:10121000474B9C4272DDBBF1000F72DD3EA3D3E968
:1012200000231046194601F091F8B1E728B1414872
:1012300013B0BDE8F04F00F0B3BDA542F7DCAFE757
:1012400004F1404303F5801353EA0A039ED0384B60
:101250009C4240F38383BBF1000F52DBDDE90001C8
:1012600096E7BCF1000F9ED089E7334B9D4231DCFD
:10127000A3F154739D429CDD2B15A3F2FF33142B75
:1012800040F3A583C3F134032CFA03F202FA03F30B
:1012900063458ED102F00102C2F102068AE7BBF17A
:1012A000000F05DA02460B4600201E4901F078F9CE
:1012B000002FBFF66DAF04F1404404F5801454EAEA
:1012C000060300F03F84012E7FF462AF01F100437A
:1012D00019465DE702266DE7BBF1000FC0F24883B7
:1012E0004046494654E742464B461046194600F0F0
:1012F00075FE02460B4601F053F949E7BBF1000FBA
:101300008CDB0020002143E742464B4640464946DD
:1013100001F01CF83CE700BF9C7500883CE4377E78
:101320000000F07F0000F03F0000E03F0000E041DF
:10133000FFFFEF3F88970100FFFF3F43B4F5801F99
:1013400080F261830022D24B01F000F86FF0340C80
:101350000C462315CF4DC4F31302A3F2FF3342F022
:101360007F546344AA420B9344F4401440F33F83F8
:10137000C94B9A4240F304849FEDAF7B8DED087B0F
:101380008DED107B9FEDAE7B0B9B8DED067B0133CE
:101390000B93A4F580140025DDE90623214682463F
:1013A00000F01CFEA346DDE9062380468946504630
:1013B0002146CDE90CAB00F013FE02460B4600209F
:1013C000B64901F0EDF80A460146CDE90E12134682
:1013D00049460246404600F0B9FF631043F000530F
:1013E00082468B4603F500238C46CDE904AB5919A0
:1013F000D3460023CDE902BC0293DDE902AB002015
:1014000004460D4602460B465046594600F09EFFE4
:1014100002460B464046494600F0E0FDDDE9062362
:10142000804689462046294600F0D8FD02460B46F4
:10143000DDE90C0100F0D2FD52465B4600F086FF6C
:1014400002460B464046494600F0C8FDDDE90E2342
:1014500000F07CFFDDE90445CDE9060122462B467C
:101460002046294600F072FF77A3D3E90023044603
:101470000D4600F06BFF76A3D3E9002300F0B0FD2A
:1014800022462B4600F062FF73A3D3E9002300F04D
:10149000A7FD22462B4600F059FF71A3D3E9002394
:1014A00000F09EFD22462B4600F050FF6EA3D3E9CC
:1014B000002300F095FD22462B4600F047FF6CA369
:1014C000D3E9002300F08CFD2246804689462B4656
:1014D0002046294600F03AFF02460B464046494660
:1014E00000F034FF524604460D465B46DDE9040138
:1014F00000F076FDDDE9062300F028FF22462B46AA
:1015000000F06EFD5246804689465B46504659467D
:1015100000F01CFF0022624BCDE90C0100F060FDE1
:1015200042464B4600F05CFD02980D4604462246BA
:101530002B465046594600F009FF002282468B4652
:10154000574B2046294600F049FDDDE90C2300F009
:1015500045FD02460B464046494600F03FFDDDE9A9
:10156000042300F0F3FE2246804689462B46DDE93F
:10157000060100F0EBFE02460B464046494600F0ED
:101580002FFD8046894602460B465046594600F0DC
:1015900027FD029838A3D3E9002304460D4600F046
:1015A000D5FE5246CDE904015B462046294600F0AF
:1015B00015FD02460B464046494600F00FFD30A39C
:1015C000D3E9002300F0C2FE2FA3D3E90023804615
:1015D00089462046294600F0B9FE02460B464046A1
:1015E000494600F0FDFCDDE9102300F0F9FC8046DF
:1015F0000B98894600F040FE424682468B464B4699
:10160000DDE9040100F0ECFCDDE9082300F0E8FC72
:1016100052465B4600F0E4FC029852465B460446A4
:101620000D4600F0DBFCDDE9082300F0D7FCDDE926
:10163000042337E0AFF3008000000000000000004A
:10164000000000000000F03FEF4E454A287ECA3FF0
:1016500065DBC9934A86CD3F01411DA96074D13F26
:101660004D268F515555D53FFFAB6FDBB66DDB3F38
:10167000033333333333E33F000000E009C7EE3F69
:10168000FD033ADC09C7EE3FF5015B14E02F3EBED7
:10169000000040438E98030079B60B000000F03F35
:1016A0000000084000F09AFC0B46024649464046BE
:1016B00000F094FC013E56EA070382468B4600F098
:1016C0005E819FEDD37B8DED047BDDE9001200236D
:1016D0000E461746CDE902670293DDE90267084628
:1016E0003B461146324600F079FC22462B4600F07C
:1016F0002DFEDDE90023804689465046594600F01C
:1017000025FE02460B464046494600F069FC32463B
:10171000804689463B4620462946CDE9008900F0AF
:1017200015FE0B46024606460F464046494600F067
:1017300057FCD14B994204460D468A4640F324811A
:1017400001F13F4303F5E003034340F0FF81B2A3FF
:10175000D3E90023DDE9000100F042FC3246804677
:1017600089463B462046294600F038FC02460B4697
:101770004046494601F07AF8002840F0E781A84643
:101780004FEA2853A3F2FE324FF48013134153441F
:10179000C3F30A52B94DA2F2FF321541C3F3130449
:1017A00023EA05010020C2F1140B44F48014BAF1BD
:1017B000000F02460B4644FA0BFB30463946B8BFD1
:1017C000CBF1000B00F00AFC06460F463246DDE97D
:1017D00000013B4600F004FC4FEA0B5A0D46002482
:1017E0008FA3D3E900232046294600F0AFFD3246FF
:1017F000804689463B462046294600F0EFFB0246DC
:101800000B46DDE9000100F0E9FB87A3D3E90023E3
:1018100000F09CFD86A3D3E9002306460F46204630
:10182000294600F093FD02460B463046394600F04B
:10183000D7FB06460F4602460B464046494600F097
:10184000CFFB42464B4604460D4600F0C7FB02461E
:101850000B463046394600F0C1FB22468046894699
:101860002B462046294600F071FD73A3D3E90023DF
:1018700006460F4600F06AFD71A3D3E9002300F08D
:10188000ADFB32463B4600F061FD6FA3D3E9002378
:1018900000F0A6FB32463B4600F058FD6CA3D3E9AE
:1018A000002300F09BFB32463B4600F04FFD6AA34D
:1018B000D3E9002300F094FB32463B4600F046FD9E
:1018C00002460B462046294600F088FB06460F4696
:1018D00002460B462046294600F038FD0022CDE99D
:1018E00000014FF080433046394600F077FB024656
:1018F0000B46DDE9000100F053FE424606460F4666
:101900004B462046294600F021FD42464B4600F05A
:1019100067FB02460B463046394600F05FFB224625
:101920002B4600F05BFB02460B460020544900F0BA
:1019300055FB8A44BAF5801FC0F232815146DDE979
:10194000042300F003FD23E4002FFFF645AC4046DE
:10195000494613B0BDE8F04F00F056B9BBF1000F97
:10196000BFF6CFACDDE90034184604F100410FE4C6
:1019700042464B460020424900F012FE08E49FED2B
:10198000387B8DED047BA0E63E4B21F00048984566
:1019900040F3EA803C4B0B4403430AD132463B46BA
:1019A00000F01CFBDDE9002300F056FF00283FF4A7
:1019B000E7AEDDE904012CA3D3E9002300F0C6FC67
:1019C00029A3D3E9002300F0C1FCFFF7E1BBBCF180
:1019D000000F40F0D280C3F1140345FA03F202FA7B
:1019E00003F3AB4200F0E0806646FFF7E9BB9FEDF2
:1019F000207B8DED087B8DED107B9FED057B002519
:101A00008DED067BC8E44FF0000CA2E4AFF300803C
:101A1000000000000000F03FFE822B654715973C58
:101A200000000000432EE63FEF39FAFE422EE63F6B
:101A3000396CA80C615C20BED0A4BE726937663ECA
:101A4000F16BD2C541BDBB3E2CDE25AF6A56113FBE
:101A500093BDBE166CC1663F3E5555555555C53FA5
:101A6000000000000000F0BF59F3F8C21F6EA5018E
:101A70000000000000000000FFFF8F40FFFF0F008C
:101A80000000F03FFFCB904000346F3F5A4B9C4228
:101A90007FF734AC594B9C423FF7BDAB0022574B0C
:101AA00000F09CFA44A3D3E9002304460D4600F05D
:101AB0004DFC43A3D3E9002382468B4620462946AA
:101AC00000F044FC0022CDE902014D4B204629469E
:101AD00000F03CFC02460B463BA1D1E9000100F0BE
:101AE0007DFA22462B4600F031FC02460B460020D0
:101AF000444900F073FA2246804689462B46204628
:101B0000294600F023FC02460B464046494600F0B9
:101B10001DFC2FA3D3E9002300F018FC02460B465E
:101B2000DDE9020100F05AFA02460B46804689467A
:101B30005046594600F054FA002004460D465246DD
:101B40005B46AFE502460B46FFF7CFBBDDE904017C
:101B500021A3D3E9002300F0F9FB1FA3D3E900235D
:101B600000F0F4FBFFF714BB264B98453FF708AE97
:101B7000DDE902239246934631E60026FFF72CBBAF
:101B80009FED177B8DED087B9FED177B8DED107B17
:101B90009FED177B4FF480258DED067BFFF7FCBB97
:101BA0005A4600F091F9CAE602F00102C2F10206BB
:101BB000FFF706BBAFF30080000000604715F73F5A
:101BC00044DF5DF80BAE543E555555555555D53F40
:101BD000FE822B654715F73F9C7500883CE4377EF5
:101BE0000000004003B8E23F06D0CF43EBFD4C3E7F
:101BF000000000000000F83FFEFFEF3F0000F03F54
:101C00000000D03F0000E03F5E4A8A432DE9F041EA
